:020000040800F2
:1000000000040020E1010008290E00082D0E000860
:10001000810E00082D0E0008550E0008E3010008AF
:10002000E3010008E3010008E3010008552F000880
:10003000E3010008E3010008E3010008E301000810
:10004000E3010008E3010008E3010008E301000800
:10005000E3010008E3010008B5310008E1310008C0
:100060000D3200083932000865320008E30100084B
:10007000E3010008E3010008E3010008E3010008D0
:10008000E3010008E3010008E3010008E3010008C0
:10009000E3010008E3010008E301000891320008D1
:1000A000E3010008E3010008E3010008E3010008A0
:1000B000D12F0008E3010008E3010008E301000874
:1000C000E3010008E3010008E3010008E301000880
:1000D000E3010008E3010008E3010008E301000870
:1000E000F9320008E3010008E3010008E301000819
:1000F000E3010008E3010008E3010008E301000850
:10010000E3010008E3010008E3010008E30100083F
:10011000E3010008E3010008E3010008E30100082F
:10012000E3010008E3010008E3010008E30100081F
:10013000E3010008E3010008E3010008E30100080F
:10014000E3010008E3010008E3010008A926000814
:10015000E3010008E3010008E3010008E3010008EF
:10016000E3010008E3010008E3010008E3010008DF
:10017000E3010008E3010008E3010008E3010008CF
:10018000E3010008E3010008E3010008E3010008BF
:10019000E3010008E3010008E3010008E3010008AF
:1001A000E3010008E3010008E3010008E30100089F
:1001B000E3010008E3010008E3010008E30100088F
:1001C000E3010008E3010008E3010008E30100087F
:1001D000E3010008E3010008E3010008E30100086F
:1001E00002E000F000F8FEE772B6394880F30888B4
:1001F000384880F3098838484EF60851CEF200019D
:10020000086040F20000CCF200004EF63471CEF2ED
:1002100000010860BFF34F8FBFF36F8F40F2000003
:10022000C0F2F0004EF68851CEF200010860BFF334
:100230004F8FBFF36F8F4FF00000E1EE100A4EF6C4
:100240003C71CEF200010860062080F31488BFF3F1
:100250006F8F01F0F1FE02F013FE4FF055301F4991
:100260001B4A91423CBF41F8040BFAE71C49194A6A
:1002700091423CBF41F8040BFAE71A491A4A1B4B5A
:100280009A423EBF51F8040B42F8040BF8E70020F5
:100290001749184A91423CBF41F8040BFAE701F0B4
:1002A000CFFE02F049FE144C144DAC4203DA54F870
:1002B000041B8847F9E700F03FF8114C114DAC42A0
:1002C00003DA54F8041B8847F9E701F0B7BE0000D1
:1002D000000400200024002000000008000000208E
:1002E00000040020083700080024002028240020F3
:1002F0002824002018300020E0010008E001000858
:10030000E0010008E00100082DE9F04F2DED108A12
:10031000C1F80CD0C3689D46BDEC108ABDE8F08FD3
:10032000002383F311882846A047002001F00AFB30
:1003300001F0BAFA00DFFEE71A4B7C2270B5002408
:100340001A700F225C709C70DC701C715C719C7167
:10035000DC711C725C729A72DC7201F03FFE064620
:1003600001F064FE054650B90F4B9E4217D0013391
:100370009E4241F2883412BF054600240125002028
:1003800001F036FE0DB100F0B5F800F021FD00F0EF
:10039000F5FB204600F00CF900F0ACF8F9E7044654
:1003A000EDE700BF28240020010007B008B500F0E9
:1003B00087FBA0F120035842584108BD07B5054B03
:1003C00002211B88ADF8043001A800F0C7FB03B080
:1003D0005DF804FBDC330008064991F8243033B1A2
:1003E00000230822086A81F8243000F0E9BB0120CC
:1003F000704700BF482400202DE9F84F234C94F8A3
:1004000024300546884617468BBB2E46DFF87C9085
:10041000002F38D094F824A0BAF1000F05D1202283
:10042000FF214846266200F0C1FCCAF10805BD4222
:1004300028BF3D465FFA85FBAD0041462A4604EBE6
:100440008A0000F089FC94F82430A7EB0B079B444A
:100450005FFA8BFBBBF1080F2E44A844FFB284F86F
:1004600024B0D5D1FFF7B8FF0028D1D108E0266A23
:1004700006EB8306B042C9D0FFF7AEFF0028C4D117
:100480000020BDE8F88F0120BDE8F88F4824002047
:1004900010B5202383F311881248C3680BB101F013
:1004A000D7FA0023104A0F484FF47A7101F094FAFA
:1004B000002383F311880D4C236813B12368013B9B
:1004C0002360636813B16368013B6360084B1B786A
:1004D00033B9636823B9022000F02CFC3223636037
:1004E00010BD00BF342400209104000878250020AE
:1004F0007024002010B5254B254953F8042F0132F4
:1005000000D110BD8B42F8D1224C234B22689A4275
:100510003AD9224B9B6803F1006303F580339A427A
:1005200032D2002000F044FB1D4B0220187000F076
:10053000F5FB1C4B1A6C00221A64196E1A66196EB0
:10054000596C5A64596E5A665A6E5A6942F0800262
:100550005A615A6922F080025A615A691A6942F056
:1005600000521A611A6922F000521A611B6972B6B0
:100570000D4A0E4B13601B682268202181F31188FD
:100580009D4683F30888104710BD00BFFCFF00089C
:100590001C00010804000108FFFF000828240020B7
:1005A000702400200038024008ED00E0000001083F
:1005B0002DE9F04F99B0B34C01902022FF2110A8F3
:1005C000A66800F0F3FBB04A1378A346A3B9AF487E
:1005D0000121C3601170202383F31188C3680BB11C
:1005E00001F036FA0023AA4AA8484FF47A7101F0C4
:1005F000F3F9002383F31188019B13B1A54B019AF2
:100600001A60A54AA349019F0292002313704B6010
:1006100099461C461D469846012000F07FFB002F9E
:1006200000F012829B4B1B68002B40F00D8219B02A
:10063000BDE8F08F0220FFF7B9FE002840F0FB81F3
:10064000019BB9F1000F08BF1F46944B1B88ADF802
:100650002C3002210BA800F081FADDE74FF47A700C
:1006600000F02EFA031E0393EADB0220FFF79EFE42
:1006700082460028E4D0039B581E042800F2DD8146
:10068000DFE800F0030E1114170018A8052340F846
:10069000343D042100F062FA54464FF0000856E061
:1006A00004217848F6E704217D48F3E704217D48DA
:1006B000F0E71C24204600F07DFA04340B9004215E
:1006C0000BA800F04BFA2C2CF4D1E5E7002DB7D0A5
:1006D000002CB5D00220FFF769FE0546002800F087
:1006E000AF8101206C4C00F063FA0220207000F012
:1006F00015FB4FF000095FFA89FA504600F068FADE
:10070000074658B1504600F073FA09F10109002874
:10071000F1D12C46A9460027634B97E7012302201D
:10072000237000F0EDFA3E46DBF808309E4206D218
:10073000304600F03FFA0130EBD10436F4E7029B7B
:1007400000261E70534BA9465E602C46374600F0CB
:1007500035FB15B1002C18BF0027FFF72FFE5BE714
:10076000002D3FF46DAF002C3FF46AAF029B0220D6
:10077000187000F0D3FA322000F0A2F9B0F1000AAC
:10078000C0F25E811AF0030540F05A81DBF80820C0
:1007900006EB0A03934200F25381BAF5807F00F220
:1007A0004F8155450DDA4FF47A7000F089F90490C5
:1007B000049B002BC0F244813C4A049BAB5401359E
:1007C000EFE7C820FFF7F2FD0546002800F038816A
:1007D0001F2E11D8C6F12004544528BF544610AB33
:1007E00026F0030022463149184400F0B5FA2246AB
:1007F000FF212E4800F0DAFA4FEAAA0A5FFA8AF2DD
:100800002A493046FFF7F8FD0446002800F01A8117
:1008100006EB8A0605469AE70220FFF7C7FD002887
:100820003FF40EAFFFF7D8FD00283FF409AF4FF0BB
:10083000000A5346DBF8082092451CD2BAF11F0F7C
:1008400012D8109A01320FD02AF0030218A90A44D4
:1008500052F8202C0B92184604220BA900F024FB1E
:100860000AF1040A0346E5E75046039300F0A2F9B3
:10087000039B0B90EFE718A8042140F84C3D00F0D3
:100880006DF964E72824002074250020342400201A
:10089000910400087825002070240020DE33000831
:1008A0002C24002030240020E03300087424002091
:1008B00018A8002340F8343D642100F02BF90028EB
:1008C0007FF4BEAE0220FFF771FD00283FF4B8AE02
:1008D0000B9800F09FF918AB43F8480D0421184617
:1008E000CDE718A8002340F8343D642100F012F948
:1008F00000287FF4A5AE0220FFF758FD00283FF442
:100900009FAE0B9800F094F918AB43F8440DE5E75F
:100910000220FFF74BFD00283FF492AE00F08EF965
:1009200018AB43F8400DD9E70220FFF73FFD002840
:100930003FF486AE0BA9142000F086F9824618A871
:10094000042140F83CAD00F009F951460BA896E7A8
:10095000322000F0B5F8B0F1000AFFF671AE1AF0DF
:10096000030F7FF46DAEDBF808200AEB0803934217
:100970003FF666AE0220FFF719FD00283FF460AE97
:100980002AF0030AC244D0453FF4E1AE404600F0ED
:1009900011F904210A900AA800F0E0F808F104080F
:1009A000F1E74FF47A70FFF701FD00283FF448AEFD
:1009B000FFF712FD00283FF4AFAE109B01330CD0BF
:1009C000082210A90020FFF717FD00283FF4A4AE6D
:1009D0002022FF2110A800F0E9F9FFF7EFFC3748CB
:1009E00000F0B6FF23E6002D3FF42AAE002C3FF4C2
:1009F00027AE18A8002340F8343D642100F08AF89F
:100A0000824600287FF41CAE0220FFF7CFFC0028AE
:100A10003FF416AE0390FFF7D1FC41F2883000F0AE
:100A200097FF0B9800F0FEF900F0C8F9039B5746BA
:100A30001C461D46F0E5054689E64FF00008FFE537
:100A40002546FDE52C4667E6002000F039F80490C5
:100A5000049B002BFFF6E3AD012000F051F9049B4D
:100A6000213B122B3FF6D8AD01A252F823F000BF74
:100A7000350600085D060008CD06000819060008C6
:100A80001906000819060008610700085109000846
:100A900019080008B1080008E30800081109000857
:100AA000190600082909000819060008A30900080A
:100AB0004F07000819060008E7090008A086010092
:100AC00037B5114B1A780132D2B20024012A0146FF
:100AD0008DF8074011D80D4803681D6A4FF47A73EA
:100AE0004B4301220DF10701A847012805D1084B0E
:100AF0009DF807001C7003B030BD4FF4FA7000F091
:100B000027FF4FF0FF30F6E70024002048260020A2
:100B10008425002038B50E4B1A780132D2B2012A52
:100B200005460ED80B4803681C6A4FF47A734B4392
:100B300004222946A047042803D1074B002018703F
:100B400038BD4FF4FA7000F003FF4FF0FF3038BDAE
:100B500000240020482600208425002030B4054CC5
:100B60002368DD69044B0A46AC460146204630BC8A
:100B7000604700BF48260020A086010070B501F044
:100B800031F9094C094E20700025306823788342E2
:100B900008D901F021F9336805440133B5F5803FE8
:100BA0003360F2D370BD00BF852500208025002072
:100BB00001F0C6B900F1006000F5803000687047B0
:100BC00000F10060920000F5803001F051B90000A2
:100BD000054B1A68054B1B789B1A834202D91044B7
:100BE00001F0FAB8002070478025002085250020FC
:100BF00038B5074D04462868204401F0F5F828B9B7
:100C000028682044BDE8384001F006B938BD00BF6F
:100C10008025002010F0030308D1B0F5007F05D82F
:100C200000F10050A0F508400068704700207047B0
:100C3000014BC058704700BF107AFF1F014B186866
:100C4000704700BF002004E070B52A4B1C68C4F355
:100C50000B03240C63B140F21342934231D040F2B3
:100C6000194293422FD040F2214293422DD10323C7
:100C7000214A0C2505FB03235D6893F9082042F205
:100C800001039C4224D0B4F5805F23D041F20103DC
:100C90009C4221D041F203039C421FD041F2070342
:100CA0009C4208BF3122441E0C44013D0B46A34226
:100CB0001ED215F9016F581C96B1034600F8016C5D
:100CC000F5E70123D4E70223D2E73F220B4DD6E715
:100CD0003322E3E74122E1E75A22E4E75922E2E73F
:100CE0002C2584421D7001D9981C5A70401A70BD81
:100CF0001846FBE7002004E0F0330008E433000866
:100D0000022804D14FF40012034B9A617047012866
:100D1000FCD14FF48012F7E700040240022803D10F
:100D20002022034B9A6170470128FCD11022F8E77A
:100D300000040240022805D1064A536983F02003CB
:100D4000536170470128FCD1024A536983F01003B4
:100D5000F6E700BF0004024010B50023934203D021
:100D6000CC5CC4540133F9E710BD000030B5441E1B
:100D700014F9010F0B4660B193F90050854201F15F
:100D8000010106D11AB993F90020801A30BD013A49
:100D9000EEE7002AF7D1104630BD000002460346B8
:100DA000981A13F9011B0029FAD17047024403462F
:100DB000934202D003F8011BFAE77047024B1A78FE
:100DC000024B1A70704700BF8425002000240020C9
:100DD00038B5104D104C284600F002F9214628463F
:100DE00000F02AF924680D48626DD2F8043843F007
:100DF0000203C2F8043800F0ABFD0949204600F0B8
:100E000027FA626DD2F8043823F00203C2F80438DE
:100E100038BD00BF48260020BC34000840420F0007
:100E2000E434000870470000FEE7000000B59BB006
:100E3000EFF3098168226846FFF78EFFEFF3058321
:100E4000034B9A6B9A6A9A6A9A6A9A6A9B6AFEE755
:100E500000ED00E000B59BB0EFF309816822684621
:100E6000FFF77AFFEFF30583044B9A6B9A6A9A6A4D
:100E70009A6A9A6A9A6A9B6AFEE700BF00ED00E0F0
:100E800000B59BB0EFF3098168226846FFF764FF65
:100E9000EFF30583034B5A6B9A6A9A6A9A6A9A6AC5
:100EA0009B6AFEE700ED00E030B5084D0A44914230
:100EB0000BD011F8013B09245840013CF7D040F316
:100EC00000032B4083EA5000F7E730BD2083B8EDE4
:100ED000002304491A465A50C8180833802B426030
:100EE000F9D17047882500200268436811430160EA
:100EF00003B118477047000013B5446BD4F894341D
:100F00001A681178042915D1217C022912D1197986
:100F1000128901238B4013420CD101A904F14C002A
:100F200001F028FED4F89444019B21790246206800
:100F300000F0DAF902B010BD143001F0ABBD0000D2
:100F40004FF0FF33143001F0A5BD00004C3001F02C
:100F50007DBE00004FF0FF334C3001F077BE000043
:100F6000143001F079BD00004FF0FF31143001F072
:100F700073BD00004C3001F049BE00004FF0FF325D
:100F80004C3001F043BE0000D0F8942438B513680B
:100F900019780429054601D0012038BD017C0229B9
:100FA000FAD112795C89012090400440F4D105F116
:100FB000140001F00BFD02460028EDD0D5F8945442
:100FC0004FF480732868697900F07CF9204638BDB9
:100FD000406BFFF7D9BF000000207047704700004A
:100FE0007FB5124B0360002343608360C36001251B
:100FF00002260F4B057404460290019300F184020F
:10100000294600964FF48073143001F0BBFC094B65
:101010000193029400964FF4807304F523722946DD
:1010200004F14C0001F082FD04B070BD40340008B2
:10103000D10F0008F90E00080B68202282F31188F6
:101040000A7903EB820290614A79093243F822005F
:101050008A7912B103EB8203986102230374C0F80A
:101060009414002383F311887047000038B5037F80
:10107000044613B190F85430ABB9201D012502216C
:10108000FFF732FF04F1140025776FF0010100F043
:1010900087FC84F8545004F14C006FF00101BDE866
:1010A000384000F07DBC38BD10B501210446043045
:1010B000FFF71AFF0023237784F8543010BD000097
:1010C00038B504460025143001F074FC04F14C00DE
:1010D000257701F043FD201D84F854500121FFF7CE
:1010E00003FF2046BDE83840FFF74EBF90F844307C
:1010F00003F06003202B19D190F84520212A0AD053
:10110000222A4FF000030ED0202A0FD1084A826312
:101110000722C26304E0064B83630723C3630023F3
:101120000364012070478363C363F9E700207047BD
:1011300001240020D0F8943437B51A6811780429B6
:1011400004461AD1017C022917D119791289012389
:101150008B40134211D100F14C05284601F0BEFD31
:1011600058B101A9284601F005FDD4F89444019B2B
:1011700021790246206800F0B7F803B030BD0000C6
:1011800000EB8103F7B59C6905460E46F4B12023B8
:1011900083F3118805EB8607201D0821FFF7A4FEC5
:1011A000FB685B691B684C3413B1204601F0F0FC0E
:1011B00001A9204601F0DEFC024648B1019B314600
:1011C000284600F091F8002383F3118803B0F0BDA6
:1011D000FB685A691268002AF5D01B8A013B13404C
:1011E000F1D105F14402EAE7093138B550F8214060
:1011F000DCB1202383F31188D4F894241368527946
:1012000003EB8203DB689B695D6845B104216018CC
:10121000FFF76AFE294604F1140001F0E1FB2046C5
:10122000FFF7B2FE002383F3118838BD704700003A
:1012300000F08CBF0123037000234360C36183620D
:101240000362C3624362036303814381704700000A
:1012500038B50446202383F3118800254160C5601A
:1012600005614561856100F081FF0223237085F3EC
:10127000118838BD70B500EB810305465069DA600E
:101280000E46144618B110220021FFF78FFDA06909
:1012900018B110220021FFF789FD31462846BDE82C
:1012A000704001F02DB80000028902F001020281B5
:1012B000428902F0010242810022026142618261A0
:1012C00001F0B2B8F0B400EB81044789E46801256D
:1012D000A4698D403D43458123600023A260636083
:1012E000F0BC01F0CDB80000F0B400EB8104078938
:1012F000E468012564698D403D4305812360002336
:10130000A2606360F0BC01F047B9000070B5022331
:10131000002504460370A0F84C5080F84E5080F829
:101320004F5005814581C56005614561856180F843
:10133000345000F081FF63681B6823B129462046C2
:10134000BDE87040184770BD436802781B6880F89C
:101350005020052202700BB104211847704700008D
:10136000436890F850201B6802700BB105211847A4
:101370007047000090F8343070B5044613B1002374
:1013800080F8343004F14402204601F06FF86368BD
:101390009B6863BB94F8445015F0600615D194F82F
:1013A000453005F07F0545EA032540F202339D42B2
:1013B00000F00E815BD8022D00F0DC803FD8002DBC
:1013C00000F08780012D00F0CF800021204601F041
:1013D000A5FA0021204601F097FA63681B6813B153
:1013E000062120469847062384F8343070BD2046F5
:1013F00098470028CED094F84B2094F84A3043EA1E
:101400000223E26B934238BFE36394F94430E56B07
:10141000002B4FF0200380F2FD80002D00F0EC80C7
:10142000092284F8342083F311880021E36BA26B36
:101430002046FFF759FF002383F3118870BDB5F5EF
:10144000817F00F0B180B5F5407F49D0B5F5807F50
:10145000BBD194F84630012BB7D1B4F84C3023F00F
:101460000203A4F84C30A663E6632664C3E740F2A7
:1014700001639D421ED8B5F5C06F3BD2B5F5A06F94
:10148000A3D1B4F84430B3F5A06F0ED194F8463030
:1014900084F84E30204600F027FF63681B6813B1C4
:1014A000012120469847032323700023A363E363AD
:1014B0002364A0E7B5F5106F32D040F602439D4299
:1014C00052D0B5F5006F80D104F14F03A36301231F
:1014D00024E004F14C03A3630223E36325648AE759
:1014E00094F84630012B7FF470AFB4F84C3043F0E1
:1014F0000203B6E794F84920616894F848304D68D3
:1015000094F8471043EA0223204694F84620A8475F
:1015100000283FF45AAF4368A3630368E363A4E77A
:101520002378042B10D1202383F311882046FFF762
:10153000BBFE86F31188636884F84F601B68032143
:1015400021700BB12046984794F84630002BACD060
:1015500084F84F300423237063681B68002BA4D0E9
:10156000022120469847A0E7374BA3630223E36399
:1015700000239DE794F8481011F0800F204601F0F9
:101580000F010ED000F064FF012806D002287FF47E
:101590001CAF2E4BA363E06367E72D4BA363E563AA
:1015A00063E700F047FFEFE794F84630002B7FF445
:1015B0000CAF94F8483013F00F013FF476AF1A06E1
:1015C000204602D501F0BEF96FE701F0B1F96CE7F2
:1015D00094F84630002B7FF4F8AE94F8483013F0BE
:1015E0000F013FF462AF1B06204602D501F096F9C9
:1015F0005BE701F089F958E7142284F8342083F37B
:1016000011882B462A4629462046FFF75BFE85F3C4
:10161000118870BD5DB1152284F8342083F31188E0
:101620000021E36BA26B2046FFF74CFE03E70B2281
:1016300084F8342083F311882B462A462946204615
:10164000FFF752FEE3E700BF70340008683400087B
:101650006C34000838B590F834300446152B29D87E
:10166000DFE803F03E28282828283E28280B2939BF
:1016700028282828282828283E3E90F84B1090F843
:101680004A20C36B42EA01229A4214D9C268128AE4
:10169000B3FBF2F502FB15356DB9202383F31188F6
:1016A0002B462A462946FFF71FFE85F311880A2399
:1016B00084F8343038BD142384F83430202383F385
:1016C000118800231A4619462046FFF7FBFD002328
:1016D00083F3118838BD036C03B198470023E7E713
:1016E000002101F01BF90021204601F00DF963688B
:1016F0001B6813B10621204698470623D8E700004F
:1017000090F83420152A38B5044622D80123934096
:1017100040F6416213421DD113F480150FD19B0294
:1017200017D50B2380F83430202383F311882B4600
:101730002A462946FFF7D8FD85F3118838BDC368CE
:101740009B695B682BB9036C03B19847002384F84D
:10175000343038BD002101F0E1F80021204601F0CD
:10176000D3F863681B6813B1062120469847062307
:10177000EDE70000024B00221B605B609A6070473F
:1017800008260020002303748268054B1B689968B3
:101790009142FBD25A680360426010605860704703
:1017A0000826002008B5202383F31188037C032B2F
:1017B00005D0042B0DD02BB983F3118808BD4369E4
:1017C00000221A604FF0FF334361FFF7DBFF002375
:1017D000F2E790E80C001A6002685360F2E700003C
:1017E000002303748268054B1B6899689142FBD8FB
:1017F0005A680360426010605860704708260020F5
:10180000054B19690874186802681A6053601861FA
:1018100001230374FEF778BD0826002030B54B1C69
:1018200087B005460A4C10D023690A4A01A800F087
:10183000D3F82846FFF7E4FF049B13B101A800F09A
:1018400007F92369586907B030BDFFF7D9FFF8E7FA
:1018500008260020A517000838B50C4D41612B69FA
:1018600081689A689142044603D8BDE83840FFF782
:1018700089BF1846FFF786FF01232C6101462374B8
:101880002046BDE83840FEF73FBD00BF08260020D7
:10189000044B1A681B6990689B68984294BF0020AB
:1018A000012070470826002010B5084C23682069E5
:1018B0001A6822605460012223611A74FFF790FFB6
:1018C00001462069BDE81040FEF71EBD0826002035
:1018D0008260022202740022427470478368A3F17E
:1018E0007C0243F80C2C026943F83C2C426943F813
:1018F000382C074A43F81C2CC26843F8102C0222EB
:1019000003F8082C002203F8072CA3F118007047F5
:101910002103000810B5202383F31188FFF7DEFFB1
:1019200000210446FFF798FF002383F31188204627
:1019300010BD0000024B1B6958610F20FFF760BF0C
:1019400008260020202383F31188FFF7F3BF00004F
:1019500008B50146202383F311880820FFF75EFFB6
:10196000002383F3118808BD49B1064B42681B6907
:1019700018605A60136043600420FFF74FBF4FF0B8
:10198000FF307047082600200368984206D01A6886
:101990000260506059611846FFF7F4BE70470000BE
:1019A00038B504460D462068844200D138BD03682E
:1019B00023605C604561FFF7E5FEF4E7054B03F14A
:1019C00014025A619A614FF0FF32DA6100221A6202
:1019D000704700BF08260020F8B503614FF0804330
:1019E000C2605C6A194B1A46022952F8145F38BF6C
:1019F0000221954206461F460AD1586198611C6231
:101A00000560456081600819BDE8F84001F088B9BB
:101A1000186AAB68241A0C1902D3E41A2D6804E082
:101A20009C4202D2204401F089F9AB689C42F4D870
:101A30006B68736035601E606E60B460A9684FF0BB
:101A4000FF33091BA960FB61F8BD00BF0826002019
:101A500010B41B4C234653F8141F814210D0416828
:101A600002680A60026851609A424FF00001C1604A
:101A700003D0936881680B4493605DF8044B704712
:101A80000A68626100209A425360C86003D15DF821
:101A9000044B01F04DB993688868034493604FF09C
:101AA0008042206A526A121A9342E6D9991A012991
:101AB00098BF931C18445DF8044B01F03FB900BF78
:101AC0000826002000207047FEE700007047000055
:101AD0004FF0FF3070470000022906D0032906D0DE
:101AE0000129064818BF0020704705487047032A9F
:101AF0009ABF044800EBC200002070474035000840
:101B0000F43400080824002070B59AB001AD0646F0
:101B100008462946144600F095F82846FFF73EF996
:101B2000C0B2431C5B0086E8180023700323637077
:101B3000002302341946DAB2904204F1020401D8BB
:101B40001AB070BDEA5C04F8022C04F8011C0133E1
:101B5000F1E7000008B5202383F311880348FFF75D
:101B6000E9FA002383F3118808BD00BF482600204E
:101B700010B50446052916D8DFE801F0161503163E
:101B8000161D202383F311880E4A0121FFF772FBF3
:101B900020460D4A0221FFF76DFB0C48FFF790FA33
:101BA000002383F3118810BD202383F31188074895
:101BB000FFF75CFAF4E7202383F311880348FFF76B
:101BC00073FAEDE7743400089834000848260020C2
:101BD00038B50C4D0C4C0D492A4604F10800FFF7AE
:101BE00093FF05F1CA0204F110000949FFF78CFFC9
:101BF00005F5CA7204F118000649BDE83840FFF740
:101C000083BF00BF102B002008240020C43400082C
:101C1000CE340008D934000870B5044608460D4695
:101C2000FFF7BCF8C6B22046013403780BB918465A
:101C300070BD32462946FFF799F80028F3D10120FC
:101C400070BD00002DE9F84F05460C46FFF7A6F8D9
:101C50002B49C6B22846FFF7DFFF08B10236F6B2BD
:101C600028492846FFF7D8FF08B11036F6B2632E90
:101C70000DD8DFF88C80DFF88C90234FDFF890A030
:101C8000DFF890B02E7846B92670BDE8F88F294667
:101C90002046BDE8F84F01F099BB252E2CD1072234
:101CA00041462846FFF762F858B9DBF80030236058
:101CB000DBF8043063609BF8083023720735093481
:101CC000E0E7082249462846FFF750F8A0B90F4B35
:101CD000A21C13F8011F09095345C95D02F8021C33
:101CE000197801F00F0102F10202C95D02F8031C2C
:101CF000EFD118340835C5E7267001350134C1E746
:101D000060350008D9340008723500080F7AFF1FCB
:101D10001B7AFF1F68350008BFF34F8F024AD36854
:101D2000DB03FCD4704700BF003C024008B5094B00
:101D30001B7873B9FFF7F0FF074B1A69002ABFBF82
:101D4000064A5A6002F188325A601A6822F48062A8
:101D50001A6008BD6E2D0020003C0240230167453B
:101D600008B50B4B1B7893B9FFF7D6FF094B1A69DF
:101D700042F000421A611A6842F480521A601A68EE
:101D800022F480521A601A6842F480621A6008BD18
:101D90006E2D0020003C02400B2870B513D80B4A72
:101DA0000B4C137863B90B4E4FF0006144F82310CD
:101DB00056F8235001330C2B2944F7D1012313701B
:101DC00054F8200070BD002070BD00BFA02D002081
:101DD000702D002084350008014B53F82000704717
:101DE000843500080C2070470B2810B5044601D933
:101DF000002010BDFFF7D0FF064B53F824301844E5
:101E0000C21A0BB9012010BD12680132F0D1043B97
:101E1000F6E700BF843500080B2810B5044621D82A
:101E2000FFF77AFFFFF782FF0F4AF323D360C30067
:101E3000DBB243F4007343F002031361136943F40C
:101E400080331361FFF768FFFFF7A6FF074B53F8D6
:101E5000241000F0DDF8FFF783FF2046BDE81040B6
:101E6000FFF7C2BF002010BD003C024084350008CF
:101E70002DE9F84312F00103154640D18218B2F162
:101E8000016F3CD22C4B1B6813F0010337D02B4C55
:101E9000FFF74CFFF323E360FFF73EFF40F201271B
:101EA000032D01D9830713D0244C0F46401A40F26A
:101EB0000118EB1B0B44012B00EB0706236924D808
:101EC00023F001032361FFF74BFF0120BDE8F883F6
:101ED000236923F44073236123693B43236151F851
:101EE000046B0660BFF34F8FFFF716FF03689E4237
:101EF00008D0236923F001032361FFF731FF00209D
:101F0000BDE8F883043D0430CAE723F4407323613D
:101F1000236943EA08032361B94637F8023B33805B
:101F2000BFF34F8FFFF7F8FE3688B9F80030B6B22E
:101F3000B342BED0DDE700BF00380240003C0240A3
:101F4000084908B50B7828B153B9FFF7EFFE012314
:101F50000B7008BD23B1BDE808400870FFF700BF53
:101F600008BD00BF6E2D002010B50244064B043999
:101F7000D2B2904200D110BD441C00B253F82000F0
:101F800041F8040FE0B2F4E750280040104B30B5A0
:101F90001C6F240407D41C6F44F400741C671C6F6E
:101FA00044F400441C670B4C236843F480732360A3
:101FB0000244094B0439D2B2904200D130BD441CD6
:101FC00000B251F8045F43F82050E0B2F4E700BFDC
:101FD00000380240007000405028004007B5012240
:101FE00001A90020FFF7C0FF019803B05DF804FBD2
:101FF00013B50446FFF7F2FFA04206D002A9012262
:1020000041F8044D0020FFF7C1FF02B010BD0000F1
:1020100070470000034B1B689B0042BF024B01222C
:102020001A70704774380240A12D0020014B1878B7
:10203000704700BFA12D002070470000FEE70000A0
:10204000084A094B09498B4204D3094A00219342AB
:1020500005D3704752F8040F43F8040BF3E743F835
:10206000041BF4E72C37000818300020183000203B
:1020700018300020836D30B500229D68446D1146F4
:102080004FF0FF3004EB421301329542C3F80019C0
:10209000C3F81019C3F80809C3F8001BC3F8101BD4
:1020A000C3F8080BEED24FF00113C4F81C3830BD52
:1020B000890141F02001016103699B06FCD41220D3
:1020C00000F0C4BE204B03EB80022DE9F047D2F8AC
:1020D0000CE05D6DDEF81420461CD2F800C005EB64
:1020E000063605EB4018516861450BD3D5F8342806
:1020F000012303FA00F022EA0000C5F8340818466C
:10210000BDE8F087BEF81040ACEB0103A34228BF46
:102110002346D8F81849A4B2B3EB840F10D89468BA
:102120001F46A4F1040959F804AFC6F800A0042F13
:1021300001D9043FF7E71C440B4494605360D2E795
:102140000020BDE8F08700BFA42D002010B5054C8D
:102150002046FFF76FF84FF0A0436365024BA3657D
:1021600010BD00BFA42D0020D83500080378012B36
:1021700070B5054650D12A4B446D98421BD1294B6E
:102180005A6B42F080025A635A6D42F080025A65DF
:102190005A6D5A6942F080025A615A6922F08002EF
:1021A0005A610E2143205B6900F0D6FB1E4BE360B1
:1021B0001E4BC4F800380023C4F8003EC02323603F
:1021C0006E6D4FF40413A3633369002BFCDA012313
:1021D00033610C2000F03AFE3369DB07FCD4122097
:1021E00000F034FE3369002BFCDA0026A660284696
:1021F000FFF740FF6B68C4F81068DB68C4F8146828
:10220000C4F81C684BB90A4BA3614FF0FF336361FC
:10221000A36843F00103A36070BD064BF4E700BF61
:10222000A42D00200038024040140040030020028A
:10223000003C30C0083C30C0F8B5446D0546002174
:102240002046FFF735FFA96D00234FF001128F687C
:10225000C4F834384FF00066C4F81C284FF0FF3043
:1022600004EB431201339F42C2F80069C2F8006BCD
:10227000C2F80809C2F8080BF2D20B686A6DEB6568
:10228000636210231361166916F01006FBD1122049
:1022900000F0DCFDD4F8003823F4FE63C4F8003805
:1022A000A36943F4402343F01003A3610923C4F856
:1022B0001038C4F814380A4BEB604FF0C043C4F830
:1022C000103B084BC4F8003BC4F81069C4F800394F
:1022D000EB6D03F1100243F48013EA65A362F8BDCD
:1022E000B435000840800010426D90F84E10D2F8CE
:1022F000003823F4FE6343EA0113C2F80038704744
:102300002DE9F0410EB200EB86080D46D8F80C100E
:102310000F6807F00303022B50D0032B50D03D4A27
:102320003D4F012B18BF1746446D4FEA451E04EB85
:102330000E030022C3F8102B8A6905F1100C002A45
:1023400040D04A8A05F158035B013A43E250012329
:10235000D4F81C2803FA0CF31343A6444A69C4F8C2
:102360001C380023CEF8103905F13F03002A39D07C
:102370000A8A898B9208012988BF4A43C16D04EB00
:102380008303561841EA0242C66529465A60204630
:10239000FFF78EFED8F80C301B8A43EA85531F43A3
:1023A00005F148035B01E7500123D4F81C2803FA28
:1023B00005F51543C4F81C58BDE8F081174FB3E785
:1023C000174FB1E704EB4613D3F8002B22F4004279
:1023D000C3F8002BD4F81C28012303FA0CF322EADB
:1023E0000303BAE704EB83030E4A5A6004EB461674
:1023F00029462046FFF75CFED6F8003923F4004357
:10240000C6F80039D4F81C38012202FA05F523EA8F
:102410000505CFE700800010008004100080081040
:1024200000800C1000040002826D1268C265FFF784
:1024300021BE00005831436D49015B5813F4004040
:1024400004D013F4001F14BF0120022070470000C5
:102450004831436D49015B5813F4004004D013F434
:10246000001F14BF012002207047000000EB810113
:10247000CB68196A0B6813604B68536070470000A3
:1024800000EB810330B5DD68AA691368D36019B920
:10249000402B84BF402313606B8A1468426D1C4438
:1024A000013CB4FBF3F46343033323F0030302EB77
:1024B000411043EAC44343F0C043C0F8103B2B68CB
:1024C00003F00303012B09B20ED1D2F8083802EB56
:1024D000411013F4807FD0F8003B14BF43F08053C9
:1024E00043F00053C0F8003B02EB4112D2F8003B2E
:1024F00043F00443C2F8003B30BD00002DE9F04139
:10250000244D6E6D06EB40130446D3F8087BC3F8E8
:10251000087B38070AD5D6F81438190706D505EB15
:1025200084032146DB6828465B689847FA072FD565
:10253000D6F81438DB072BD505EB8403D968CCB962
:102540008B69488A5E68B6FBF0F200FB12628AB9BA
:102550001868DA6890420DD2121A83E8140020231A
:1025600083F311880B482146FFF78AFF84F3118813
:10257000BDE8F081012303FA04F26B8923EA020328
:102580006B81CB6823B121460248BDE8F041184772
:10259000BDE8F081A42D002000EB810370B5DD685B
:1025A000436D6C692668E6604A0156BB1A444FF4D5
:1025B0000020C2F810092A6802F00302012A0AB2B8
:1025C0000ED1D3F8080803EB421410F4807FD4F83E
:1025D000000914BF40F0805040F00050C4F80009DA
:1025E00003EB4212D2F8000940F00440C2F800099F
:1025F000D3F83408012202FA01F10143C3F8341878
:1026000070BD19B9402E84BF4020206020682E8AFA
:10261000841940F00050013C1A44B4FBF6F440EA3F
:10262000C440C6E7F8B504461E48456D05EB4413A3
:10263000D3F80869C3F80869F10717D5D5F8103839
:10264000DA0713D500EB8403D9684B691F68DA6891
:10265000974218D2D21B00271A605F60202383F3B1
:1026600011882146FFF798FF87F31188330617D5A5
:10267000D5F834280123A340134211D02046BDE8E9
:10268000F840FFF71FBD012303FA04F2038923EA90
:10269000020303818B68002BE8D021469847E5E7C9
:1026A000F8BD00BFA42D002096482DE9F84F456DD8
:1026B0006E69AB691E4016F4805F6E61044605D0FA
:1026C000FEF724FEBDE8F84F00F054BC002E12DAED
:1026D000D5F8003E8B489B071EBFD5F8003E23F07F
:1026E0000303C5F8003ED5F8043823F00103C5F80C
:1026F0000438FEF735FE370502D58248FEF724FE82
:10270000B0040CD5D5F8083813F0060FEB6823F4A5
:1027100070530CBF43F4105343F4A053EB603107E4
:1027200004D56368DB680BB176489847F2025AD447
:10273000B3020CD5D4F85480DFF8C8A100274FF0BD
:102740000109A36D9B68F9B28B4280F08780F70680
:1027500019D5616D0A6AC2F30A1702F00F0302F479
:10276000F012B2F5802F00F0A180B2F5402F0AD10F
:1027700004EB830301F58051DB68186A00231A46D5
:102780009F4240F087803003D5F8184813D5E10305
:1027900002D50020FFF7B2FEA20302D50120FFF709
:1027A000ADFE630302D50220FFF7A8FE270302D582
:1027B0000320FFF7A3FE750384D5E00702D50020B0
:1027C000FFF730FFA10702D50120FFF72BFF6207BB
:1027D00002D50220FFF726FF23077FF573AF032002
:1027E000FFF720FF6EE7D4F85480DFF818A1002728
:1027F0004FF00109A36D9B685FFA87FB5B4597D398
:1028000008EB4B13D3F8002902F44022B2F5802FD5
:1028100022D1D3F80029002A1EDAD3F8002942F089
:102820009042C3F80029D3F80029002AFBDB59465F
:10283000606DFFF73DFC228909FA0BF322EA0303DE
:10284000238104EB8B03DB689B6813B15946504628
:1028500098475846FFF736FC0137CBE708EB4112A3
:10286000D2F8003B03F44023B3F5802F10D1D2F807
:10287000003B002B0CDA628909FA01F322EA030318
:10288000638104EB8103DB68DB680BB1504698473A
:10289000013756E79C0708BF0A68072B98BF0270EC
:1028A00003F101039CBF120A013069E7023304EB14
:1028B000830201F58051526890690268D0F808C01F
:1028C0004068A2EB000E0022104697420AD104EBAA
:1028D000830463689B699A683A449A605A6817440B
:1028E0005F6050E712F0030F08BF0868964588BF85
:1028F0008CF8000002F1010284BF000A0CF1010C07
:10290000E3E700BFA42D0020436D03EB4111D1F894
:10291000003B43F40013C1F8003B7047436D03EBE9
:102920004111D1F8003943F40013C1F80039704760
:10293000436D03EB4111D1F8003B23F40013C1F8C0
:10294000003B7047436D03EB4111D1F8003923F48C
:102950000013C1F80039704700F1604300F01F0216
:10296000400903F5614309018000C9B200F16040EC
:1029700083F8001300F5614001239340C0F88031D3
:102980000360704730B5039C0172043304FB0325D8
:10299000C361049B03630021059B00604060C1602C
:1029A000426102618561046242628162C162436385
:1029B00030BD00000022416A41610161C260826253
:1029C000C2626FF00101FEF7EBBF000003694269CC
:1029D000934203D1C2680AB100207047181D7047A6
:1029E00003691960C2680132C260C2691344826916
:1029F0000361934224BF436A03610021FEF7C4BF11
:102A000038B504460D46E3683BB16269131D126890
:102A1000A3621344E362002038BD237A33B9294608
:102A20002046FEF7A1FF0028EDDA38BD6FF0010067
:102A3000FBE70000C368C269013BC36043691344FC
:102A400082694361934224BF436A436100238362E6
:102A5000036B03B11847704770B52023044683F316
:102A60001188866A3EB9FFF7CBFF054618B186F399
:102A70001188284670BDA36AE26A13F8015BA3625D
:102A8000934202D32046FFF7D5FF002383F311883A
:102A9000EFE700002DE9F84F04460E4690469946B0
:102AA000202787F311880025AA46D4F828B0BBF167
:102AB000000F09D149462046FFF7A2FF20B18BF352
:102AC00011882846BDE8F88FA16AE36AA8EB050BD8
:102AD0005B1A9B4528BF9B46BBF1400F1BD9334671
:102AE00001F1400251F8040B43F8040B9142F9D173
:102AF000A36A40334036A3624035A26AE36A9A4231
:102B000002D32046FFF796FF8AF311884545D8D2B5
:102B100087F31188C9E730465A46FEF71DF9A36AC4
:102B20005B445E44A3625D44E7E7000010B5029C8D
:102B30000172043303FB0421C36100238362C36277
:102B4000039B0363049B00604060C46042610261B8
:102B5000816104624262436310BD0000026AC26088
:102B6000426A4261026100228262C2626FF0010128
:102B7000FEF716BF436902699A4203D1C2680AB1DF
:102B800000207047184650F8043B0B607047000067
:102B9000C368C2690133C3604369134482694361F6
:102BA000934224BF436A43610021FEF7EDBE00005B
:102BB00038B504460D46E3683BB123691A1DA2628D
:102BC000E2691344E362002038BD237A33B9294611
:102BD0002046FEF7C9FE0028EDDA38BD6FF001008F
:102BE000FBE7000003691960C268013AC260C2696C
:102BF000134482690361934224BF436A0361002343
:102C00008362036B03B118477047000070B520233F
:102C100004460E4683F31188856A35B91146FFF7DD
:102C2000C7FF10B185F3118870BDA36A1E70A36A37
:102C3000E26A01339342A36204D3E1692046043976
:102C4000FFF7D0FF002080F3118870BD2DE9F84F09
:102C500004460D4691469A464FF0200888F31188A5
:102C60000026B346A76A4FB951462046FFF7A0FF9A
:102C700020B187F311883046BDE8F88FA06AE76A73
:102C8000A9EB06033F1A9F4228BF1F46402F1BD9BE
:102C900005F1400355F8042B40F8042B9D42F9D16F
:102CA000A36A4033A3624036A26AE36A9A4204D31D
:102CB000E16920460439FFF795FF8BF311884E45F3
:102CC000D9D288F31188CDE729463A46FEF744F871
:102CD000A36A3B443D44A3623E44E5E7026943697D
:102CE0009A4203D1C3681BB9184670470023FBE71B
:102CF000836A002BF8D0043B9B1AF5D01360C3689D
:102D0000013BC360C3691A44836902619A4224BFCC
:102D1000436A0361002383620123E5E700F06CB995
:102D20004FF08043002258631A610222DA60704734
:102D30004FF080430022DA60704700004FF080437C
:102D400058637047FEE7000010B5174CFEF712FD00
:102D5000FEF734FE802215492046FEF7B9FD012317
:102D600044F8180C0374124B124AD96821F4E0613C
:102D70000904090C0A431049DA60CA6842F08072FB
:102D8000CA600E490A6842F001020A601022DA772E
:102D9000202283F82220002383F3118862B608489A
:102DA000BDE81040FEF7B6BD30260020E43500082F
:102DB00000ED00E00003FA05F0ED00E0001000E097
:102DC000EC3500082DE9F84F1F4C4FF000086569FD
:102DD00004F11407C1464FF08043266A5B6AAA6873
:102DE0009E1B96421DD34FF0200AAA68236AD5F88D
:102DF0000CB0134423622B68BB425F60A6EB020653
:102E00006361C5F80C8001D1FFF792FF89F3118847
:102E10002869D8478AF311886569AB689E42E4D275
:102E2000D9E76269BA420CD0916823628E1B966022
:102E3000A86802282CBF1818981CBDE8F84FFFF7A7
:102E40007DBFBDE8F88F00BF08260020034B5968FE
:102E50005A68521A9042FBD8704700BF001000E039
:102E60004B6843608B688360CB68C3600B694361C8
:102E70004B6903628B6943620B6803607047000013
:102E800008B5224B22481A6940F2FF110A431A6121
:102E90001A6922F4FF7222F001021A611A691A6B90
:102EA0000A431A631A6D0A431A651A4A1B6D1146C2
:102EB000FFF7D6FF184802F11C01FFF7D1FF1748B2
:102EC00002F13801FFF7CCFF154802F15401FFF77A
:102ED000C7FF144802F17001FFF7C2FF124802F168
:102EE0008C01FFF7BDFF114802F1A801FFF7B8FF01
:102EF0000F4802F1C401FFF7B3FF0E4802F1E001F1
:102F0000FFF7AEFFBDE8084000F0E0B8003802402F
:102F1000000002400C360008000402400008024095
:102F2000000C024000100240001402400018024051
:102F3000001C02400020024008B500F037FAFFF7FD
:102F400003FFFFF767F8BDE80840FEF741BE000049
:102F500070470000064A536823F001035360EFF303
:102F60000983683383F30988002383F3118870474A
:102F700030EF00E010B5202383F31188104B5B681D
:102F800013F4006318D0F1EE103AEFF309844FF018
:102F9000807344F84C3C0B4BDB6844F8083CA4F1CC
:102FA000680383F30988FEF773FC18B1064B44F8F5
:102FB000503C10BD054BFAE783F3118810BD00BFEC
:102FC00000ED00E030EF00E03103000834030008BA
:102FD0004FF0804310B51A69920708D500241C6190
:102FE000202383F31188FFF7EDFE84F31188BDE8F9
:102FF0001040FFF7BFBF0000104B1A6C42F00102F7
:103000001A641A6E42F001021A660D4A1B6E93682A
:1030100043F0010393604FF0804353229A624FF0D4
:10302000FF32DA6200229A615A63DA605A60012242
:103030005A6108211A601C20FFF78EBC003802403C
:10304000002004E01F4B1A696FEAC2526FEAD252A5
:103050001A611A69C2F308021A614FF0FF301A6947
:103060005A69586100215A6959615A691A6A62F0AD
:1030700080521A621A6A02F080521A621A6A5A6AF6
:1030800058625A6A59625A6A1A6C42F080521A643B
:103090001A6E42F080521A661A6E0B4A106840F49B
:1030A00080701060186F00F44070B0F5007F1EBF94
:1030B0004FF4803018671967536823F40073536026
:1030C00000F054B90038024000700040304B4FF01F
:1030D00080521A642F4A4FF4404111601A6842F03E
:1030E00001021A601A689207FCD59A6822F003025E
:1030F0009A60274B19469A6812F00C02FBD11868A7
:1031000000F0F90018609A601A6842F480321A6080
:103110000B689B03FCD54B6F43F001034B671C4BC3
:103120005A6F9007FCD51C4A5A601A6842F08072A8
:103130001A60184A53685904FCD5154B1A68920155
:10314000FCD5164A9A60164B1A68164B9A42164BD3
:103150001BD1164A1168164A914216D140F2051247
:103160001A600B4B9A6842F002029A609A6802F069
:103170000C02082AFAD15A6C42F480425A645A6E00
:1031800042F480425A665B6E704740F20572E7E790
:10319000003802400070004008544007009488380E
:1031A000002004E011640020003C024000ED00E03B
:1031B00041C20F41084A08B5536911680B4003F03A
:1031C0000103536123B1054A13680BB15068984756
:1031D000BDE80840FFF7CEBE003C01408825002036
:1031E000084A08B5536911680B4003F002035361A4
:1031F00023B1054A93680BB1D0689847BDE80840F1
:10320000FFF7B8BE003C014088250020084A08B5F9
:10321000536911680B4003F00403536123B1054A5D
:1032200013690BB150699847BDE80840FFF7A2BE8B
:10323000003C014088250020084A08B55369116800
:103240000B4003F00803536123B1054A93690BB1A6
:10325000D0699847BDE80840FFF78CBE003C0140AC
:1032600088250020084A08B5536911680B4003F00F
:103270001003536123B1054A136A0BB1506A984792
:10328000BDE80840FFF776BE003C014088250020DD
:10329000174B10B55C691A68144004F478725A61CF
:1032A000A30604D5134A936A0BB1D06A9847600607
:1032B00004D5104A136B0BB1506B9847210604D507
:1032C0000C4A936B0BB1D06B9847E20504D5094AC1
:1032D000136C0BB1506C9847A30504D5054A936C49
:1032E0000BB1D06C9847BDE81040FFF743BE00BF5C
:1032F000003C0140882500201A4B10B55C691A6813
:10330000144004F47C425A61620504D5164A136DD8
:103310000BB1506D9847230504D5134A936D0BB13B
:10332000D06D9847E00404D50F4A136E0BB1506E70
:103330009847A10404D50C4A936E0BB1D06E984700
:10334000620404D5084A136F0BB1506F98472304E9
:1033500004D5054A936F0BB1D06F9847BDE8104074
:10336000FFF708BE003C014088250020062108B573
:103370000846FFF7F1FA06210720FFF7EDFA0621CC
:103380000820FFF7E9FA06210920FFF7E5FA0621F0
:103390000A20FFF7E1FA06211720FFF7DDFA0621E0
:1033A0002820BDE80840FFF7D7BA000008B5FFF7AE
:1033B00049FEFDF78DFDFDF73BFFFDF70FFEFFF723
:1033C000C7FDBDE80840FFF7A9BC0000034611F89F
:1033D000012B03F8012B002AF9D1704712101213A8
:1033E0001211000053544D3332463F3F3F0000005E
:1033F00000000000E43300083F0000001304000058
:10340000203400083F000000190400002A3400089E
:103410003F00000021040000343400083F00000099
:1034200053544D3332463430780053544D33324682
:103430003432780053544D333246343436585800C1
:1034400000000000550F0008410F00087D0F000824
:10345000690F0008750F0008610F00084D0F000884
:10346000390F0008D90F000800000000010000001B
:1034700000000000020000000000000081110008B0
:10348000E911000840004000E02A0020F02A002056
:103490000200000000000000030000000000000027
:1034A0002D1200080000000010000000002B00207A
:1034B000000000000100000000000000A42D00201A
:1034C000010102004172647550696C6F74002542FD
:1034D0004F415244252D424C002553455249414C01
:1034E00025000000711B0008D91A0008ED10000823
:1034F000551B000843000000FC340008090243008B
:10350000020100C03209040000010202010005248A
:103510000010010524010001042402020524060014
:1035200001070582030800FF09040100020A0000E8
:10353000000705010240000007058102400000006D
:10354000120000004835000812011001020000407E
:10355000091241570002010203010000040309049B
:1035600025424F41524425007265766F2D6D696E7C
:1035700069003031323334353637383941424344CB
:1035800045460000004000000040000000400000F0
:1035900000400000000001000000020000000200E6
:1035A0000000020000000200000002000000020013
:1035B0000000020000000000751300085516000806
:1035C0000117000840004000042E0020042E0020B7
:1035D00001000000142E00208000000040010000C7
:1035E000030000006D61696E0000000004360008F1
:1035F000202E00201830002001000000452D00087A
:103600000000000069646C65000000000001800299
:1036100000000000AAAAAAAA00010000FFFF000003
:103620000000000000A00A004005000000000000AB
:10363000AAAAAAAA40000000CFFF000000000000D4
:10364000000000000000000000000000AAAAAAAAD2
:1036500000000000FFFF000000000000000000006C
:103660000000000000000000AAAAAAAA00000000B2
:10367000FFFF00000000000000000000000000004C
:1036800000000000AAAAAAAA00000000FFFF000094
:10369000000000000000000000000000000000002A
:1036A000AAAAAAAA00000000FFFF00000000000074
:1036B000000000000000000000000000AAAAAAAA62
:1036C00000000000FFFF00000000000000000000FC
:1036D00000000000000000000A00000000000000E0
:1036E00003000000000000000000000000000000D7
:1036F00000000000000000000000000000000000CA
:103700000000000000000000FF009600000000081C
:10371000040000005C35000800000000000000000C
:103720000000000000000000000000000000000099
:10373000FFFFFFFFFFFFFFFFFFFFFFFFFFFFFFFF99
:10374000FFFFFFFFFFFFFFFFFFFFFFFFFFFFFFFF89
:10375000FFFFFFFFFFFFFFFFFFFFFFFFFFFFFFFF79
:020000040801F1
:100000000006002089120108958E0608F18D060869
:100010005D8E0608F18D0608298E06088B120108F0
:100020008B1201088B1201088B1201082963080842
:100030008B1201088B1201088B1201088B12010828
:100040008B1201088B1201088B1201088B12010818
:100050008B1201088B120108C16E0808E96E0808AE
:10006000116F0808396F0808616F080889210808AE
:10007000B1210808DD2108080922080835220808EE
:100080005D220808892208080D2108088B12010842
:100090008B1201088B1201088B120108896F080866
:1000A0008B1201088B1201088B1201088B120108B8
:1000B00085700808997008088B120108152808082F
:1000C000BD2908088B1201088B1201088B12010848
:1000D0008B1201085D7008088B1201087170080806
:1000E000ED6F08088B1201088B120108BD7008081B
:1000F000C1700808D5700808D9700808B52208082A
:100100008B1201088B120108AD7008088B120108D0
:100110008B1201088B1201088B1201088B12010847
:10012000E122080809230808352308086123080884
:100130008D2308088B1201088B1201088B1201080D
:100140008B1201088B1201088B120108556A0808EE
:10015000B5230808E12308080D2408088B120108BC
:100160008B1201088B1201088B1201088B120108F7
:100170008B1201088B1201088B1201088B120108E7
:100180008B1201088B1201088B1201088B120108D7
:100190008B1201088B1201088B1201088B120108C7
:1001A0008B1201088B1201088B1201088B120108B7
:1001B0008B1201088B1201088B1201088B120108A7
:1001C0008B1201088B1201088B1201088B12010897
:1001D0008B1201088B1201088B1201088B12010887
:1001E0008125010855AD0108E1CD020889500408B8
:1001F000056D0408F5BE040839C8040881CB04085D
:10020000DD330508DD3805089D50050851CB05088C
:10021000698706083524070871AA07084DD1070821
:1002200095DB07089D0A080865100808FFFFFFFF17
:1002300081F0004102E000BF83F0004330B54FEA97
:1002400041044FEA430594EA050F08BF90EA020F04
:100250001FBF54EA000C55EA020C7FEA645C7FEA97
:10026000655C00F0E2804FEA5454D4EB5555B8BFBA
:100270006D420CDD2C4480EA020281EA030382EA2B
:10028000000083EA010180EA020281EA0303362DBD
:1002900088BF30BD11F0004F4FEA01314FF4801C90
:1002A0004CEA113102D0404261EB410113F0004FA2
:1002B0004FEA03334CEA133302D0524263EB430359
:1002C00094EA050F00F0A780A4F10104D5F1200EF7
:1002D0000DDB02FA0EFC22FA05F2801841F1000152
:1002E00003FA0EF2801843FA05F359410EE0A5F126
:1002F00020050EF1200E012A03FA0EFC28BF4CF057
:10030000020C43FA05F3C01851EBE37101F000450C
:1003100007D54FF0000EDCF1000C7EEB00006EEB19
:100320000101B1F5801F1BD3B1F5001F0CD34908A3
:100330005FEA30004FEA3C0C04F101044FEA4452FA
:1003400012F5800F80F09A80BCF1004F08BF5FEA81
:10035000500C50F1000041EB045141EA050130BD61
:100360005FEA4C0C404141EB0101013C28BFB1F573
:10037000801FE9D291F0000F04BF01460020B1FABE
:1003800081F308BF2033A3F10B03B3F120020CDA91
:100390000C3208DD02F1140CC2F10C0201FA0CF06F
:1003A00021FA02F10CE002F11402D8BFC2F1200CD4
:1003B00001FA02F120FA0CFCDCBF41EA0C0190408A
:1003C000E41AA2BF01EB0451294330BD6FEA0404D3
:1003D0001F3C1CDA0C340EDC04F11404C4F12002BE
:1003E00020FA04F001FA02F340EA030021FA04F3D0
:1003F00045EA030130BDC4F10C04C4F1200220FA27
:1004000002F001FA04F340EA0300294630BD21FA64
:1004100004F0294630BD94F0000F83F4801306BF2A
:1004200081F480110134013D4EE77FEA645C18BF1E
:100430007FEA655C29D094EA050F08BF90EA020FB5
:1004400005D054EA000C04BF1946104630BD91EAAD
:10045000030F1EBF0021002030BD5FEA545C05D1B0
:100460004000494128BF41F0004130BD14F58004EF
:100470003CBF01F5801130BD01F0004545F0FE4163
:1004800041F470014FF0000030BD7FEA645C1ABF98
:10049000194610467FEA655C1CBF0B46024650EACF
:1004A000013406BF52EA033591EA030F41F40021FB
:1004B00030BD00BF90F0000F04BF0021704730B581
:1004C0004FF4806404F132044FF000054FF0000156
:1004D00050E700BF90F0000F04BF0021704730B517
:1004E0004FF4806404F1320410F0004548BF4042EC
:1004F0004FF000013EE700BF42004FEAE2014FEA41
:1005000031014FEA02701FBF12F07F4393F07F4F1B
:1005100081F06051704732F07F4208BF704793F01E
:100520007F4F04BF41F40021704730B54FF4607431
:1005300001F0004521F000411CE700BF50EA010234
:1005400008BF704730B54FF000050AE050EA0102DD
:1005500008BF704730B511F0004502D5404261EB4D
:1005600041014FF4806404F132045FEA915C3FF48E
:10057000D8AE4FF003025FEADC0C18BF03325FEA2B
:10058000DC0C18BF033202EBDC02C2F1200300FADC
:1005900003FC20FA02F001FA03FE40EA0E0021FA01
:1005A00002F11444BDE600BF70B54FF0FF0C4CF4EF
:1005B000E06C1CEA11541DBF1CEA135594EA0C0FA1
:1005C00095EA0C0F00F0DEF82C4481EA030621EADC
:1005D0004C5123EA4C5350EA013518BF52EA033517
:1005E00041F4801143F4801338D0A0FB02CE4FF0C9
:1005F0000005E1FB02E506F00042E0FB03E54FF0F9
:100600000006E1FB03569CF0000F18BF4EF0010EF0
:10061000A4F1FF04B6F5007F64F5407404D25FEAEC
:100620004E0E6D4146EB060642EAC62141EA55519F
:100630004FEAC52040EA5E504FEACE2EB4F1FD0CE1
:1006400088BFBCF5E06F1ED8BEF1004F08BF5FEA5F
:10065000500E50F1000041EB045170BD06F0004611
:1006600046EA010140EA020081EA0301B4EB5C04BE
:10067000C2BFD4EB0C0541EA045170BD41F48011B6
:100680004FF0000E013C00F3AB8014F1360FDEBFDB
:10069000002001F0004170BDC4F10004203C35DAB7
:1006A0000C341BDC04F11404C4F1200500FA05F33A
:1006B00020FA04F001FA05F240EA020001F00042DB
:1006C00021F0004110EBD37021FA04F642EB060151
:1006D0005EEA430E08BF20EAD37070BDC4F10C047B
:1006E000C4F1200500FA04F320FA05F001FA04F23F
:1006F00040EA020001F0004110EBD37041F100012B
:100700005EEA430E08BF20EAD37070BDC4F1200535
:1007100000FA05F24EEA020E20FA04F301FA05F29D
:1007200043EA020321FA04F001F0004121FA04F245
:1007300020EA020000EBD3705EEA430E08BF20EA15
:10074000D37070BD94F0000F0FD101F0004640004F
:1007500041EB010111F4801F08BF013CF7D041EAD1
:10076000060195F0000F18BF704703F000465200D5
:1007700043EB030313F4801F08BF013DF7D043EAA6
:100780000603704794EA0C0F0CEA135518BF95EA5C
:100790000C0F0CD050EA410618BF52EA4306D1D1E3
:1007A00081EA030101F000414FF0000070BD50EA02
:1007B000410606BF1046194652EA430619D094EA8C
:1007C0000C0F02D150EA013613D195EA0C0F05D176
:1007D00052EA03361CBF104619460AD181EA0301CA
:1007E00001F0004141F0FE4141F470014FF0000082
:1007F00070BD41F0FE4141F4780170BD70B54FF01D
:10080000FF0C4CF4E06C1CEA11541DBF1CEA13559C
:1008100094EA0C0F95EA0C0F00F0A7F8A4EB05047E
:1008200081EA030E52EA03354FEA013100F0888075
:100830004FEA03334FF0805545EA131343EA12633E
:100840004FEA022245EA111545EA10654FEA0026F3
:100850000EF000419D4208BF964244F1FD0404F5AC
:10086000407402D25B084FEA3202B61A65EB030508
:100870005B084FEA32024FF480104FF4002CB6EBC5
:10088000020E75EB030E22BFB61A754640EA0C0045
:100890005B084FEA3202B6EB020E75EB030E22BF85
:1008A000B61A754640EA5C005B084FEA3202B6EBC6
:1008B000020E75EB030E22BFB61A754640EA9C0085
:1008C0005B084FEA3202B6EB020E75EB030E22BF55
:1008D000B61A754640EADC0055EA060E18D04FEA13
:1008E000051545EA16754FEA06164FEAC30343EAB3
:1008F00052734FEAC2025FEA1C1CC0D111F4801F80
:100900000BD141EA00014FF000004FF0004CB6E778
:1009100011F4801F04BF01430020B4F1FD0C88BF17
:10092000BCF5E06F3FF6AFAEB5EB030C04BFB6EB22
:10093000020C5FEA500C50F1000041EB045170BD15
:100940000EF0004E4EEA113114EB5C04C2BFD4EB42
:100950000C0541EA045170BD41F480114FF0000EC6
:10096000013C90E645EA060E8DE60CEA135594EA42
:100970000C0F08BF95EA0C0F3FF43BAF94EA0C0F45
:100980000AD150EA01347FF434AF95EA0C0F7FF4BA
:1009900025AF104619462CE795EA0C0F06D152EA0E
:1009A00003353FF4FDAE1046194622E750EA4106F2
:1009B00018BF52EA43067FF4C5AE50EA41047FF403
:1009C0000DAF52EA43057FF4EBAE12E74FF0FF3C68
:1009D00006E000BF4FF0010C02E000BF4FF0010C39
:1009E0004DF804CD4FEA410C7FEA6C5C4FEA430CB2
:1009F00018BF7FEA6C5C1BD001B050EA410C0CBF01
:100A000052EA430C91EA030F02BF90EA020F002062
:100A1000704710F1000F91EA030F58BF994208BFC9
:100A200090422CBFD8176FEAE37040F00100704786
:100A30004FEA410C7FEA6C5C02D150EA013C07D1DD
:100A40004FEA430C7FEA6C5CD6D152EA033CD3D028
:100A50005DF8040B704700BF8446104662468C4622
:100A60001946634600E000BF01B5FFF7B7FF002855
:100A700048BF10F1000F01BD4DF808EDFFF7F4FF7E
:100A80000CBF012000205DF808FB00BF4DF808ED09
:100A9000FFF7EAFF34BF012000205DF808FB00BF2C
:100AA0004DF808EDFFF7E0FF94BF012000205DF84E
:100AB00008FB00BF4DF808EDFFF7CEFF94BF012003
:100AC00000205DF808FB00BF4DF808EDFFF7C4FFFC
:100AD00034BF012000205DF808FB00BF4FEA410C45
:100AE0007FEA6C5C02D150EA013C0AD14FEA430C28
:100AF0007FEA6C5C02D152EA033C02D14FF0000065
:100B000070474FF0010070474FEA410212F50012A2
:100B100015D211D56FF47873B3EB625212D94FEA44
:100B2000C12343F0004343EA505311F0004F23FA2E
:100B300002F018BF404270474FF00000704750EA83
:100B4000013005D111F0004008BF6FF00040704740
:100B50004FF00000704700BF4A0011D212F500129A
:100B600011D20DD56FF47873B3EB62520ED44FEA05
:100B7000C12343F0004343EA505323FA02F0704785
:100B80004FF00000704750EA013002D14FF0FF30C3
:100B900070474FF0000070474FEA4102B2F1E04366
:100BA00024BFB3F5001CDCF1FE5C0DD901F0004C54
:100BB0004FEAC0024CEA5070B2F1004F40EB8300A4
:100BC00008BF20F00100704711F0804F21D113F1D0
:100BD0003872BCBF01F00040704741F480114FEA09
:100BE0005252C2F11802C2F1200C10FA0CF320FA92
:100BF00002F018BF40F001004FEAC1234FEAD323AF
:100C000003FA0CFC40EA0C0023FA02F34FEA430318
:100C1000CCE77FEA625307D150EA01331EBF4FF0A1
:100C2000FE4040F44000704701F0004040F0FE40BC
:100C300040F40000704700BF80F0004002E000BFB9
:100C400081F0004142001FBF5FEA410392EA030FB7
:100C50007FEA226C7FEA236C6AD04FEA1262D2EB01
:100C60001363C1BFD218414048404140B8BF5B4206
:100C7000192B88BF704710F0004F40F4000020F09F
:100C80007F4018BF404211F0004F41F4000121F0B5
:100C90007F4118BF494292EA030F3FD0A2F10102FF
:100CA00041FA03FC10EB0C00C3F1200301FA03F13D
:100CB00000F0004302D5494260EB4000B0F5000F60
:100CC00013D3B0F1807F06D340084FEA310102F11F
:100CD0000102FE2A51D2B1F1004F40EBC25008BFD1
:100CE00020F0010040EA03007047490040EB00009B
:100CF000013A28BFB0F5000FEDD2B0FA80FCACF19C
:100D0000080CB2EB0C0200FA0CF0AABF00EBC250C8
:100D100052421843BCBFD0401843704792F0000FB6
:100D200081F4000106BF80F400000132013BB5E709
:100D30004FEA41037FEA226C18BF7FEA236C21D07F
:100D400092EA030F04D092F0000F08BF08467047E4
:100D500090EA010F1CBF0020704712F07F4F04D1B2
:100D6000400028BF40F00040704712F100723CBFC5
:100D700000F50000704700F0004343F0FE4040F4EF
:100D8000000070477FEA226216BF08467FEA2363AD
:100D90000146420206BF5FEA412390EA010F40F498
:100DA000800070474FF0000304E000BF10F00043E4
:100DB00048BF40425FEA000C08BF704743F09643CB
:100DC00001464FF000001CE050EA010208BF7047E6
:100DD0004FF000030AE000BF50EA010208BF70476D
:100DE00011F0004302D5404261EB41015FEA010C82
:100DF00002BF84460146002043F0B64308BFA3F17A
:100E00008053A3F50003BCFA8CF2083AA3EBC2535B
:100E100010DB01FA02FC634400FA02FCC2F120027A
:100E2000BCF1004F20FA02F243EB020008BF20F0B1
:100E30000100704702F1200201FA02FCC2F1200217
:100E400050EA4C0021FA02F243EB020008BF20EA0C
:100E5000DC7070477BB972B90029BEBF00204FF02B
:100E6000004106E008BF00281CBF6FF000414FF0B2
:100E7000FF3000F007BAADF1080C6DE904CE00298F
:100E800009DB002B1ADB00F095F8DDF804E0DDE962
:100E9000022304B07047404261EB4101002B1BDB91
:100EA00000F088F8DDF804E0DDE9022304B04042F8
:100EB00061EB4101524263EB43037047524263EBE3
:100EC000430300F077F8DDF804E0DDE9022304B025
:100ED000404261EB41017047524263EB430300F033
:100EE00069F8DDF804E0DDE9022304B0524263EB67
:100EF0004303704753B94AB9002908BF00281CBFF3
:100F00004FF0FF314FF0FF3000F0BCB9ADF1080CED
:100F10006DE904CE00F04EF8DDF804E0DDE90223CF
:100F200004B07047430803F05533C01A830803F038
:100F3000333300F03330184400EB101000F00F3062
:100F400000EB002000EB0040000E704707EE900A17
:100F5000F5EEC07AF1EE10FA01D400F00BB8F1EE24
:100F6000677A08B517EE900A00F004F8404261EB8A
:100F7000410108BDD0B5FFF7BFFA0C4B0022064671
:100F80000F46FFF711FBFFF7E7FD0446FFF792FA64
:100F9000074B0022FFF708FB02460B463046394656
:100FA000FFF74AF9FFF7D8FD2146D0BD0000F03D1C
:100FB0000000F0412DE9F047089D04468E46002BC5
:100FC0004DD18A42944669D9B2FA82F252B101FAFD
:100FD00002F3C2F1200120FA01F10CFA02FC41EA0D
:100FE000030E94404FEA1C48210CBEFBF8F61FFA92
:100FF0008CF708FB16E341EA034306FB07F199422D
:101000000AD91CEB030306F1FF3080F01F819942DF
:1010100040F21C81023E63445B1AA4B2B3FBF8F0B9
:1010200008FB103344EA034400FB07F7A7420AD940
:101030001CEB040400F1FF3380F00A81A74240F268
:1010400007816444023840EA0640E41B00261DB1D3
:10105000D4400023C5E900433146BDE8F0878B4208
:1010600009D9002D00F0EF800026C5E900013046C7
:101070003146BDE8F087B3FA83F6002E4AD18B42A1
:1010800002D3824200F2F980841A61EB030301204B
:101090009E46002DE0D0C5E9004EDDE702B9FFDE37
:1010A000B2FA82F2002A40F09280A1EB0C014FEAE2
:1010B0001C471FFA8CFE0126200CB1FBF7F307FB3F
:1010C000131140EA01410EFB03F0884208D91CEBE2
:1010D000010103F1FF3802D2884200F2CB8043467F
:1010E000091AA4B2B1FBF7F007FB101144EA01445E
:1010F0000EFB00FEA64508D91CEB040400F1FF31ED
:1011000002D2A64500F2BB800846A4EB0E0440EADA
:1011100003409CE7C6F12007B34022FA07FC4CEAE3
:10112000030C20FA07F401FA06F31C43F9404FEAD6
:101130001C4900FA06F3B1FBF9F8200C1FFA8CFEEB
:1011400009FB181140EA014108FB0EF0884202FA3F
:1011500006F20BD91CEB010108F1FF3A80F0888000
:10116000884240F28580A8F102086144091AA4B2BD
:10117000B1FBF9F009FB101144EA014100FB0EFE3E
:101180008E4508D91CEB010100F1FF346CD28E456D
:101190006AD90238614440EA0840A0FB0294A1EBFE
:1011A0000E01A142C846A64656D353D05DB1B3EB5B
:1011B000080261EB0E0101FA07F722FA06F3F1408B
:1011C0001F43C5E9007100263146BDE8F087C2F132
:1011D0002003D8400CFA02FC21FA03F391400143AA
:1011E0004FEA1C471FFA8CFEB3FBF7F007FB1036E3
:1011F0000B0C43EA064300FB0EF69E4204FA02F48F
:1012000008D91CEB030300F1FF382FD29E422DD9E1
:10121000023863449B1B89B2B3FBF7F607FB163316
:1012200041EA034106FB0EF38B4208D91CEB010196
:1012300006F1FF3816D28B4214D9023E6144C91A16
:1012400046EA004638E72E46284605E70646E3E626
:101250001846F8E64B45A9D2B9EB020864EB0C0E30
:101260000138A3E74646EAE7204694E74046D1E73F
:10127000D0467BE7023B614432E7304609E76444ED
:10128000023842E7704700BF02E000F000F8FEE7D6
:1012900072B6374880F30888364880F309883648A4
:1012A0003649086040F20000CCF200004EF634717E
:1012B000CEF200010860BFF34F8FBFF36F8F40F293
:1012C0000000C0F2F0004EF68851CEF20001086036
:1012D000BFF34F8FBFF36F8F4FF00000E1EE100AA6
:1012E0004EF63C71CEF200010860062080F31488AF
:1012F000BFF36F8F75F076F876F0D6F94FF0553072
:101300001F491B4A91423CBF41F8040BFAE71D49B3
:10131000184A91423CBF41F8040BFAE71A491B4AAC
:101320001B4B9A423EBF51F8040B42F8040BF8E7FE
:1013300000201849184A91423CBF41F8040BFAE7D3
:1013400075F054F876F004FA144C154DAC4203DAFB
:1013500054F8041B8847F9E701F002F9114C124DCB
:10136000AC4203DA54F8041B8847F9E775F03CB83F
:1013700000060020002200200000010808ED00E027
:101380000000002000060020B04A0A0800220020C9
:101390009425002098250020B8030120E0010108D1
:1013A0002C0201082C0201082C0201082DE9F04F43
:1013B0002DED108AC1F80CD0C3689D46BDEC108A93
:1013C000BDE8F08F002383F311882846A047002052
:1013D00073F05AFFFEE773F0C1FD00DFFEE7000087
:1013E00001F0FF01102A2BDB10F0070F08D010F8D6
:1013F000013B013A8B422DD010F0070F42B3F6D1DA
:10140000F0B441EA012141EA014122F007047FF0F2
:1014100000070023F0E80256083C85EA010586EA49
:10142000010685FA47F5A3FA87F586FA47F6A5FA85
:1014300087F68EB9EED1F0BC01F0FF0102F0070291
:1014400032B110F8013B013A83EA010313B1F8D13C
:101450000020704701387047002D06BF354603381D
:10146000073815F0010F07D1013015F4807F02BF56
:10147000013015F4C03F0130F0BC0138704700BFA7
:1014800010F8012B11F8013B012A28BF9A42F7D02E
:10149000D01A7047034613F8012B002AFBD1181A03
:1014A0000138704738B50022002304460D46FFF787
:1014B000EDFA28B920462946BDE8384000F00AB8C0
:1014C000204605F1004100F005F8404261EB410182
:1014D00038BD00BFD0B50C4B002206460F46FFF7C3
:1014E00063F8FFF739FB0446FEF7E4FF074B0022E1
:1014F000FFF75AF802460B4630463946FEF79CFE87
:10150000FFF72AFB2146D0BD0000F03D0000F0416E
:10151000036800221B6818470120704737B5019106
:101520002021044655F02CFBD0B10E4B93F98612C6
:10153000A1B1B3F98812D3F8203A019AB3F90C504B
:1015400001F10A039D4203DD40F28D33994205DC2F
:101550002046054B202155F019FB002003B030BD7B
:101560000120FBE7A0450020D8E4080808B505F0F5
:10157000A9FDBDE80840012104F0E2BE2DE9F043D9
:101580008FB00E46054605F09DFD002780462E22B1
:10159000394602A8019778F049FE322301AA39465C
:1015A000404605F077F8044648B9184A01AB314681
:1015B000284655F02DFD20460FB0BDE8F083DFF83A
:1015C0005890D9F8980603689B6898470028F2D08D
:1015D000A9F5405003F0DEFC814630B90C4A314693
:1015E000284655F015FD4C46E5E76946404604F0AF
:1015F00099FE0028DFD09DF801305B06DBD5054A57
:101600003146284655F004FD3C46D4E7ECE4080892
:10161000F5E408080CE50808A055002008B5064BBD
:1016200093F8593C9B0704D5044A55F0F1FC00207F
:1016300008BD0120FCE700BFA04500201CE508080C
:1016400070B50C4C0546D4F898060368DB680E4666
:10165000984710B10124204670BDA4F5405003F016
:10166000B7FC04460028F5D1034A3146284655F018
:10167000CFFCF0E7A05500202CE508082DE97043C9
:10168000274BD3F85C3C1D7B814688465DB9254BD2
:101690001B68986A03685B6B984738B9224A4146D1
:1016A000484655F0B5FC2846BDE8708342F010F975
:1016B000202143F079F838B142F00AF91F2143F0B4
:1016C00073F808B1194AEAE7484655F051FA38B9B3
:1016D000D9F80030414648465B6BBDE87043184777
:1016E00041464846FFF71AFF41460646484656F02F
:1016F000F1F820210640484655F042FA4146484656
:10170000FFF78CFFF5B2054041464846FFF798FFCA
:1017100041460540484656F0ABFA0540C3E700BFD6
:10172000A0450020405D002040E5080857E5080876
:1017300008B5FFF7A3FF054A92F8481C60F3410182
:1017400082F8481C024A907108BD00BFA0450020E5
:10175000ED5D00202DE9F04106460F4655F046FAB2
:10176000044668B30221304655F00AFA40B305F04A
:10177000A9FC4FF48071804604F0E2FD0546F8B9FB
:101780004FF40071404604F0DBFDC8B10E4856F03E
:101790008BFC0E4BD3ED707AF8EEE77A30EE670AE9
:1017A000DFED0B7AB0EEC00AB4EEE70AF1EE10FA04
:1017B00006DD084B3A460221304655F0E7F92C4643
:1017C0002046BDE8F08100BF58580020A0550020F9
:1017D0000000C84274E50808F8B504460F4655F005
:1017E000A5FC10210546204655F0CAF958B12046FF
:1017F000FFF7BCFE064630B9044B3A46102120469E
:1018000055F0C4F935462846F8BD00BF88E50808FC
:1018100070B505460E4655F057FA044678B180215A
:10182000284655F0ADF950B1094B93F8BD3143B19D
:10183000084B32468021284655F0A8F9002420465E
:1018400070BD31462846BDE8704055F035BE00BF3A
:10185000A05500209CE508082DE9F04180460E4681
:10186000FFF78CFE1A4F044610B90024FC710AE001
:10187000184D05F54053D3F8980603689B689847C0
:1018800020B90123FB712046BDE8F08108214046C4
:1018900055F076F90028F4D095F8E433B02202FB35
:1018A000035305F50055B3F8EE21B5F984329A4299
:1018B00006DD094B32460821404655F067F9D4E76A
:1018C0003146404655F0D4FA0028DAD1CDE700BFC2
:1018D000ED5D0020A0250020B0E5080855F0EABE27
:1018E00070B505460E46FFF749FE084B0446D87111
:1018F00031462846FFF7A4FE31460028284608BF97
:10190000002456F071F8204070BD00BFED5D00204E
:101910002DE9F843414F3B788146002B7BD1404C69
:10192000D4F85C5C2D7B01263E701DB13B702846CF
:10193000BDE8F88356F05AFA054630B9394A38708E
:10194000137843F001031370F1E7DFF8F48037F008
:101950006FF8314636F092F988F804600B2630F0C3
:101960007DF8013E30F018F816F0FF06F7D12E4949
:10197000484656F051F905F0A5FBD0F80C22C4F802
:101980006C2C90F89432DA0733D404F0F1FE37F07F
:101990004FF83C2136F088FF04F6544300221A60C9
:1019A000224B1B68D86A036801211B689847D4F84A
:1019B0005C2C137B1BB90123137388F8043037F0B8
:1019C00037F894F84D2C94F84C1C36F047FB34F063
:1019D00003FB33F02DFE00233B7057F091FA144BBC
:1019E000C3F88C0694F8493C43F0200384F8493C42
:1019F0009DE79B07D4D431460E4802F071F90E489A
:101A000056F052FBDFED0D7A20EE270A04F6544320
:101A100083ED000AC4E7002589E700BF9825002070
:101A2000A04500200C5E0020C0E50808405D0020B5
:101A3000A0550020A0250020585800200AD7233C9C
:101A4000ED5D00202DE9F043364DD5F85C3C1B7B65
:101A500087B006460C46002B61D000294BD02146AA
:101A6000304656F07BFA0446002853D02E493046C3
:101A700056F0D2F805F026FB074609F02FFF804606
:101A8000384604F0C5F8D8B198F92430022B17D1A4
:101A900000264FF00009F1B203AA38460191CDF8B3
:101AA0000C90CDF81090CDF8149004F08FFC0199B3
:101AB00018B103AA404609F01DFC0136032EEAD1F5
:101AC000D5F85C2C137B1BB100231373174A1371D9
:101AD00036F0AEFF002136F0D1F8154B1B68D86AFE
:101AE000036800211B68984795F8493C6FF345133C
:101AF00085F8493C0FE005F580530192D3F898062C
:101B00000368DB689847019A0028A8D195F8483CFB
:101B1000DB06A4D40024204607B0BDE8F0830124EE
:101B2000F9E700BFA0450020D0E50808ED5D0020E2
:101B3000405D002008B500F5005090F8483CC3F324
:101B400080028A420BD061F3820380F8483C31B1B5
:101B500036F06EFFBDE808400F2136F0A5BE08BD87
:101B600010B500F500520C4692F8593C03F0010103
:101B7000A14209D064F3000382F8593CDB0704D486
:101B800002F0FAFA024B9C7210BD02F0A7FBF9E7D3
:101B9000ED5D002000F5005090F8593C61F34103E1
:101BA00080F8593C014B1973704700BFED5D002070
:101BB00000207047002070470020704700207047C9
:101BC00000207047002070470020704700207047B9
:101BD00000207047002070470020704700207047A9
:101BE000704700007047000000F50A50143070473D
:101BF00000487047B00F090800F5005090F84C0CF1
:101C000070470000034808601C21117008221A6008
:101C1000704700BF9CE8080834F02AB914F0C0B837
:101C200036F0AAB941F05EBA3FF016BC02F0C4BA71
:101C300002F0F6B902F01EB92FF0AEBE45F06CBC52
:101C400041F00EBD0EF040BF02F038B802F0FABC11
:101C500002F0AEB902F04ABC02F0C4BF14F0BCBB43
:101C600003F0CCB902F0DCBA02F094BB70B51F4BA4
:101C7000036000F500530446D3F8DC0B1C4AC3F89C
:101C8000842A08B109F078F81A4B236004F58053D0
:101C900093F87C2E42B9D3F8785E2DB1284612F025
:101CA00091FE284609F064F804F589500C3054F090
:101CB0007DFA04F58750103043F04AFE04F6C4451F
:101CC00004F66446B54204D0183D284612F0ACFA3A
:101CD000F8E7094BC4F8983804F6941038F000FF80
:101CE00004F5106038F0FCFE204670BDD8EA080804
:101CF00044B9090804990908DC6F090838B5474B4D
:101D0000044640F8043B43F0B9FF04F1100008F02A
:101D10001DFC04F1680033F039FE04F590700DF0FD
:101D20006FFB04F5866007F007FA04F2545009F0DF
:101D300057F804F6980013F0DDFE04F5446043F014
:101D400025FF04F5516033F03FFB04F58150183056
:101D500035F0E4FE04F58750103043F0E1FD04F562
:101D600089500C3054F00EFA04F58A50083034F0E3
:101D7000C9F904F58D500C3045F02EF904F5805367
:101D80000025274A83F8D05104F58E53103304F50B
:101D90008F5013602FF086FC04F5915029461030C7
:101DA00003F028FC04F5C65008304DF001F904F5A5
:101DB000E8500C3051F066FA04F5F150043053F05D
:101DC0003BFB04F5F450083053F070FF04F5F75076
:101DD00007F0B0F804F501504DF0E8FC04F50350AD
:101DE0004AF040F904F50750103043F027FA04F5A3
:101DF000005304F5095083F838520A4D103054F05E
:101E000099FD2B6813B1084857F048F82046074958
:101E100032F0D6FB2C60204638BD00BF049909087B
:101E2000B0680020C05E002024E608083C9809083D
:101E300010B502F0AFFF41F04BFD0368BDE8104064
:101E40005B681847FFF7F4BF38B500F531553035FA
:101E50000446284608F054FA09F040FD90F9213074
:101E6000D3B190F84033BBB12846002108F00EF8FA
:101E7000DFED0A7A04F2AC7393ED287A20EE270A9C
:101E8000DFED077AA7EE270A04F2545083ED280A03
:101E9000BDE8384009F032BC38BD00BFCDCCCC3DE8
:101EA0006666663FFFF7D0BF10B50121044603F018
:101EB000C9F810B1204601F0DBF84FF480512046FC
:101EC00003F0C0F820B12046BDE8104001F092B800
:101ED00010BD0000FFF7E8BF38B50221044603F04B
:101EE000B1F838B10121204603F0ACF810B9204612
:101EF00001F0BEF80221204603F0A4F858B32046B2
:101F000001F0C4F84021204603F09CF868B104F5C4
:101F100081551835284635F07DF904F5805393F93D
:101F2000F03013B1284635F0BFFA4FF480612046F7
:101F300003F088F820B104F58150183035F00CFA20
:101F40008021204603F07EF860B115F087FABDE8E5
:101F5000384013F0E3BB0121204603F073F800285A
:101F6000CDD1CFE74FF48021204603F06BF8002855
:101F7000EBD14FF40021204603F064F80028E4D1AF
:101F800038BD0000FFF7A8BF10B50121044603F0DB
:101F900059F810B1204601F079F88021204603F06D
:101FA00051F828B115F05AFABDE8104013F092BB71
:101FB00010BD0000FFF7E8BF38B54FF6FF710446CB
:101FC00003F040F804F5005528B1D5F8482C072156
:101FD000204601F063F843F05BF842F07FFE95F88D
:101FE000483C074A83F01003C3F30013537133F0E6
:101FF000F3FF33F045FCBDE8384002484CF0E4BA4A
:10200000ED5D0020445B0020FFF7D6BFF0B52DED5D
:10201000028B00F5915410349FB0054601212046F3
:1020200004F0D6FF05F547512031204604F03AFE72
:1020300005F547513831204603F0FEFE05F5AC5159
:1020400004F54B7017F0D6FF05F5405405F54850E0
:10205000D4F8E021D4F8E43184ED810A1CA90C30D5
:102060001C921D9338F05CFA05F5475105F549506F
:1020700028311030B0EE608AF0EE408A38F0E8F88F
:1020800005F5485105F54A500431C4ED7B8A84EDCD
:102090007C8A84ED7D0A043038F0DAF884ED820A17
:1020A00036F0C6FC054656F033FF2B4B0746186842
:1020B0000E46FEF721FACDE91801D4F80002FEF72A
:1020C0001BFACDE91601D4F8FC01FEF715FACDE9AB
:1020D0001401D4F8F801FEF70FFACDE91201D4F893
:1020E0000802FEF709FACDE91001D4F80402FEF760
:1020F00003FACDE90E01D4F8F401FEF7FDF9CDE9BC
:102100000C01D4F8E801FEF7F7F9CDE90A01D4F89B
:10211000F001FEF7F1F9CDE90801D4F8E401FEF78A
:10212000EBF9CDE90601D4F8EC01FEF7E5F9CDE9CC
:102130000401D4F8E001FEF7DFF9CDE90076CDE93E
:102140000201064B064A0749284636F0E3F91FB05C
:10215000BDEC028BF0BD00BFE839002038E608086E
:1021600046E6080873E60808FFF750BF10B50446B6
:1021700002F09AFE1021204602F064FF28B115F00B
:102180006DF9BDE8104013F097BB10BDFFF7EEBF2F
:1021900000F5805000F5936300F2A440D3ED005A9F
:1021A000D0ED006AD1ED017A91ED006A26EEE77A72
:1021B00067EEA57AA6EE257AE6EE267A81ED007A1C
:1021C000C1ED017A7047000000F5805000F593637F
:1021D00000F2A440D3ED005AD0ED006AD1ED017AAF
:1021E00091ED006A27EEA67A67EEA57AA6EE257A2B
:1021F000E6EE667A81ED007AC1ED017A7047000063
:102200002DE9F0412DED028B054686B0FFF776FDF6
:10221000BA4B2B6005F50B50083005F5005401F062
:1022200021FC05F50A530C3305F528563036C4F861
:10223000283A062384F82C3A304654F027FC04AFA1
:10224000AF4BC4F8303A3946301D4FF0010805F560
:102250002A568DF81080043632F082FFA94BC4F85C
:10226000843A06F1080056F007F80723C4F8E03B6B
:102270000023A4F8E43B84F8D88B4FF4D27008F024
:1022800075FDC4F8DC0B05F52F50283055F0F4FF30
:1022900005F530502C3055F0EFFF9B4B1A6802B912
:1022A0001E609A499FED9A8A304632F089F9994B1F
:1022B000C4F8843A05F531500123A4F84C3C0E30A3
:1022C00055F086FE944B0593944B0495009305F5C9
:1022D000315097E80C004FF40071303007F00CFDDE
:1022E00005F5475003A9F7EE008A0430CDED038AC7
:1022F00037F01AFD05F54750103008F00DFA05F5D6
:1023000040549FED872A84ED788A05F59153103368
:10231000B0EE083A05F54B50C4F8D032F0EE432A3F
:10232000F0EE420AB0EE430AF0EE481AB0EE481A58
:1023300084ED798A84ED7A8A84ED7B8A84ED7C8AC7
:1023400084ED7D8A84ED7E8A84ED7F8A84ED808AA7
:1023500084ED8C8A84ED8D8A84ED8E8A84ED8F8A5B
:1023600084ED908A84ED918A84ED928A84ED938A3B
:1023700084EDAE8A84EDAF8A84EDB08A84EDB18AB3
:1023800084EDB28A84EDB38A14304CF0C3FAB0EE17
:10239000083A05F54E50F0EE432AB0EE682AF0EE0A
:1023A000481AB0EE481AF7EE080AB1EE0C0A0830E7
:1023B0004CF05EFCB0EE083AF0EE432AB0EE430A71
:1023C0009FED572ADFED570AF0EE481AB0EE481A93
:1023D00005F550504CF04CFCB0EE083A05F5515064
:1023E000F0EE432A9FED502ADFED500AF0EE481A36
:1023F000B0EE481AB0EE680A38304CF08BFAB0EE06
:10240000083A05F55450F0EE432A9FED490AB0EE24
:10241000482AF0EE481AB0EE481AF0EE480A2C307E
:102420004CF026FCF0EE083A05F556509FED410AB7
:10243000B0EE485AF0EE684AB0EE484AB0EE633A61
:10244000F0EE632AB0EE002AF0EE481AB0EE481A19
:10245000F6EE000A24304CF067F8374B3748186026
:1024600005F55A521432002314279EB207FB0601C9
:102470000133097C0029F8D1314B1E80314B19689A
:1024800011B1314856F00AFD05F55A501C30C4F818
:1024900098061A6002F090F82C4BC4F89C3605F5AB
:1024A0005B500C3002F088F8294BC4F8CC3605F5A7
:1024B0005B503C3002F080F8264BC4F8FC3605F542
:1024C0005C502C3002F078F8234BC4F82C3705F51B
:1024D0005D5004F25C7383ED008A83ED018A83ED25
:1024E000028A2C3002F068F81C4BC4F86C3728467E
:1024F00006B0BDEC028BBDE8F08100BFD8EA080849
:10250000ECE5080844B90908E061002044B5090871
:102510000000000098EB0808691C0108CCEA0808D4
:10252000CDCC4C3ECDCCCC3ECDCCCC3DCDCC4C3D21
:102530003333333F9A99993F885E00203821090848
:10254000845E0020445E002078E60808802A09089E
:10255000C0290908342B0908202A0908D02A0908AB
:1025600038B5054B1C6823680A461D68034B0146B5
:102570002046A847002038BD405D0020A02500204F
:1025800010B556F0EDF8064C064B18602046FFF7E4
:1025900037FE2046044A0549BDE8104075F040B9B1
:1025A000A0250020405D00209CB700206D1C010884
:1025B00010B504460180024932F002F8204610BDF1
:1025C00060EB080810B500234FF07C52274C0365E0
:1025D0004FF07E51C0F88030C0F89030C0F8A03085
:1025E000C0F8C0304365C0F88430C0F89430C0F8FB
:1025F000A430C0F8C43083668367C0F89830C0F850
:10260000A830C0F8B830C366C367C0F89C30C0F8C3
:10261000AC30C0F8BC304FF03F430267C0F8B02088
:102620004267C0F8B420C0F88820C0F8C820C0F8BD
:102630008C20016644668465C165C0F8CC304FF4D7
:102640007A71212042F0D2FA4FF47A71222042F0BE
:10265000CDFA4FF47A71232042F0C8FABDE8104059
:102660004FF47A71242042F0C1BA00BF000080BF4D
:10267000F8B52DED068B037B044643B90023C0F863
:10268000D430C0F8D830C0F8E030C0F8DC30D4ED39
:10269000371A94ED381AD4ED360A94ED350A854888
:1026A000DFED858A00F03AFC5820B7EE001AFFEE05
:1026B000000A94ED350A15F093FB592084ED350A94
:1026C000B7EE001AFFEE000A94ED360A15F088FB0B
:1026D0005A2084ED360AB7EE001AFFEE000A94ED98
:1026E000380A15F07DFB5B2084ED380AB7EE001A3E
:1026F000FFEE000A94ED370A15F072FB84ED370AFD
:1027000056F0F2FB07EE900A9FED6C7AF8EE677ACE
:1027100004F1100567EE877A2126C4ED027A2F4670
:10272000F7EE009A94ED35AAD5ED100AB0EE680ADE
:102730006AEE200A75F020FA94ED368AD5ED140A77
:10274000B0EE409A68EE200AB0EE680A75F014FA0E
:10275000D4ED385AD5ED186A94ED376A95ED1C7AA8
:1027600065EEA66A79EE007AF0EEE66A26EE077A62
:1027700077EEA67AB0EEC77A77EE877AB5EEC09A92
:10278000E5EC017A95ED235AC5ED079A28EE058A06
:1027900095ED1F5AAAEE058A95ED275AA5EE858A72
:1027A000D5ED2B5AA6EE258AF1EE10FACCBF012307
:1027B0000023B5EEC00A85ED038AF1EE10FA84F825
:1027C000D030C8BF94F8D030F5EEC06AC4BF013332
:1027D00084F8D030F1EE10FAC8BF94F8D030B5EEDE
:1027E000C07AC4BF013384F8D030F1EE10FAC2BF12
:1027F00094F8D030013384F8D03094F9D030002BE5
:10280000C1BF07EE103AB8EEC77AC8EE076AC5ED49
:10281000036A95ED038AB0EEC87A77EE877AF4EE14
:10282000E97AF1EE10FAC4BF79EEC77A45ED017A84
:1028300094F9E83015ED019A83B1DFED217AB4EE19
:10284000E79AF1EE10FA09D8DFED1E7AB4EEE77AD6
:10285000F1EE10FAA4BF4FF08043EB6194ED390A1A
:10286000D5ED077A20EE270AD4ED027A20EE270A6A
:10287000DFED157A30EE000A20EE270A75F0F6F843
:10288000A9EE008A30B201369FED100A85ED0B8A61
:1028900028EE000AB6B242F085F9252E7FF442AF49
:1028A000BDEC068B04F1200239460248BDE8F84031
:1028B00000F066BBA025002000000000BD37863573
:1028C0009A99193FCDCCCC3EDB0F494000007A44A9
:1028D0000022C0F8D420C0F8D820C0F8E020C0F80A
:1028E000DC20FFF7C5BE00000020704700207047C5
:1028F0000120704790F82C308B4286BF0C3150F885
:10290000210000207047000090F82C308B4286BFD9
:102910000C3150F82100002070470000FA20704769
:10292000D0E9083242F4E0524262826A43F4F8434A
:1029300042F4E0528262036270470000014802F0F4
:102940009BBB00BFA025002013B54FF45870019128
:1029500008F006FA044620B101993FF099FC024BB9
:102960002360204602B010BDE0EB0808704700006D
:10297000704700000020704770470000002070473B
:102980007047000070470000032070470820704720
:10299000064BD3F85C3C3BB11B7B002B0CBF50209B
:1029A000D02040F0010070475020FAE7A0450020F9
:1029B000704700007047000010B52DED028B174BDB
:1029C000D3F85C4C3CB3D4ED360A94ED380AF0EE03
:1029D000E00AB0EEC00A75F0CFF8D4ED370AB0EED9
:1029E000408A94ED350AF0EEE00AB0EEC00A75F0C8
:1029F000C3F8F0EE400AB0EE480A75F0BDF8DFED1E
:102A0000087A20EE270ABDEEC00A10EE103A18B27E
:102A1000BDEC028B10BD2046FAE700BFA0450020A8
:102A20000000C8423AF098BD10B504463BF0A0FF44
:102A3000054802F021FB054A034606212046BDE871
:102A400010403BF07DBF00BFA0250020CCEB080864
:102A50003BF048B808B5084607F048FF00280CBF0F
:102A60000420002008BD0000162A01D03AF0ACBDB9
:102A700003220A70012070473EF0C0BE08B53AF04C
:102A800049FF40F41C6040F00D0008BD10B504463D
:102A900008F06EF9204610BD08B5094B93F8482C94
:102AA000D2060BD403F58053D3F898060368DB6A8B
:102AB000984700280CBF0220042008BD0120FCE735
:102AC000A0450020044B187820B9044B93F8490C1A
:102AD000C0F38010704700BF985D0020A045002023
:102AE0001FB5002301930293039304F0EBFA01A9AD
:102AF00004F0B4F828B101A817F0FEFD05B05DF8A8
:102B000004FB0EF01FF890F8C432B02202FB030061
:102B100090ED2F0AF2E700000C4B93F8BD218AB923
:102B2000A3F5805393F8592C51070BD193F8482CF7
:102B3000D20609D493F8493C13F0020F14BF0420C5
:102B4000012070470520704703207047A0550020E2
:102B50002DE9F04F354F97F84C3C012B8DB00446D2
:102B600052D9334EDFF8E8A0082516F9018BB7F9E2
:102B7000A03208F1FF3B43FA0BF3D90740D5207C84
:102B800039F012F88146207C39F0D8FF00F121039A
:102B9000994505D2207C0DB0BDE8F04F3AF036BC27
:102BA000BBF1070F2CD8DFE80BF03E043234363887
:102BB0003A3C204B186959695A6AD3F804B0D3F8E3
:102BC00018E0D3F80CC0D3ED007A1B6ACDF82520AD
:102BD000CDF8293062222123CDE9003207900891F7
:102BE000207CCDED037A192303AAC221CDF810B0C1
:102BF000CDF814E0CDF818C08DF8248039F03EF8F7
:102C0000013D15F0FF05B0D10DB0BDE8F08F0A4BC6
:102C1000D0E70A4BCEE70A4BCCE70A4BCAE753464C
:102C2000C8E7094BC6E7094BC4E700BFA045002031
:102C3000A4EC0808E058002058590020D059002082
:102C4000585A0020845A0020D85B0020B458002035
:102C5000FC5A0020084BD3F8CC22920701D43AF05A
:102C6000A5BC03F5805393ED750ADFED047AB8EE49
:102C7000C00A20EE270A7047A04500200AD7233C4F
:102C800010B594B0044603A807F046FD1A4BD3F8DC
:102C90009806036803A95B6B984750B3247C56F0F1
:102CA0002FF9059BDDED047A0893069B0993002319
:102CB000F8EEE77A9FED117A0B930C930D930E9338
:102CC0000F931093119312934FF6F853ADF84C30C5
:102CD0000023962267EE877A8DF84E303323CDE9B4
:102CE0000032079007AA57212046CDED0A7A38F026
:102CF000C5FF14B010BD00BFA05500200AD7233C6B
:102D0000F0B5254D0E4607460FCD95B003AC0FC468
:102D10002B682360731EDBB2042B29D814AA02EBA4
:102D2000830353F8445C2B6828461B6A98472B683A
:102D300004469B6A28469847002305223D7C08905C
:102D400009938DF828208DF829608DF82A3094B9E0
:102D5000232221460DF12B0077F068FA86222E23DC
:102D6000CDE9003240F2B31108AA284638F086FFB8
:102D7000052015B0F0BD20460DF12B0304F1200213
:102D800050F8041B43F8041B9042F9D102881A80C2
:102D900082789A70E2E700BFE8E30808014802F091
:102DA00069B900BFA0250020014B93F84C0C704777
:102DB000A0450020024B93F8490CC0F34000704737
:102DC000A045002030B52DED028B154B91ED018A09
:102DD0000546D3F89806036885B0DB690C4698472A
:102DE00028B9BDEEC88A18EE103ADB0712D5D4E92F
:102DF000040115F0C7F968B1684607F08DFC6A4612
:102E0000214628463EF020FC20B10649684607F0DE
:102E100079FD00B1022005B0BDEC028B30BD00BFD2
:102E2000A0550020705700208B8B162B05D0C02B8F
:102E300001D1FFF7C7BF3FF05BBE00207047000025
:102E400030B52DED028B8DB000230546039304931E
:102E5000059304F037F903A903F000FF58B304F019
:102E600031F900F5607393E8070006AC84E80700C9
:102E7000DDED060A9DED070A2D7CF1EE600AB1EE4C
:102E8000400A75F015F82046B0EE408A17F034FC81
:102E9000DFED0B7A089B0B93012228EE278A0C2387
:102EA000CDE90032A82109AA28468DED098A8DEDC9
:102EB0000A0A38F0E3FE0DB0BDEC028B30BD00BF56
:102EC000E02E6542242938B5054605D040290DD0AD
:102ED000BDE838403EF058BF0C213AF0A9FA04464C
:102EE00010B12846FFF7ACFF204638BD0124FBE7B0
:102EF00008B591ED007AF6EE007AB4EEE77AF1EEDD
:102F000010FA06DD044801220521FEF79BFD002092
:102F100008BD0420FCE700BFD04F00202DE9F041A0
:102F200088B080461B22002101A810EE107A10EE16
:102F3000906A11EE105A11EE904A77F077F9A323B8
:102F40008DF8043095238DF805300B238DF806306D
:102F500055F0DEFFCDF8070008F58150CDF80B10D5
:102F60001B2201A91830CDF80F70CDF81360CDF8F1
:102F70001750CDF81B4034F099FE08B0BDE8F08141
:102F800070B58CB00D46144606462B22002101A8D0
:102F900077F04CF9A3238DF8043095238DF8053094
:102FA0000C238DF8063055F0B3FF2B68CDF80F30A9
:102FB0002368CDF813306B68CDF817306368CDF80F
:102FC0001B30AB68CDF81F30A368CDF80700CDF8F3
:102FD000233006F58150EB68CDF80B10CDF8273083
:102FE0002B22E368CDF82B3001A9183034F05EFEB7
:102FF0000CB070BD70B500F58154183400F54C521A
:103000000546143220460E2134F010FD05F54D52D0
:1030100020460F2134F00AFD05F54E522046383285
:10302000102134F003FD05F55052204605F55156A8
:103030003032112134F0FAFC06F1780220466C217E
:1030400034F0F4FC06F1A40220466D2134F0EEFCCD
:1030500005F5555220461C320D2134F0E7FC05F5EC
:10306000585220463832BDE87040692134F0DEBC49
:103070001FB500F59150002301A910300193029370
:10308000039302F0B5F905B05DF804FB08B504F050
:1030900019F8BDE8084003F02DBD00007FB50E46CD
:1030A0004FF6FF710446154601F0CCFFE8B110223F
:1030B0000021684677F0BAF8A3238DF800309523F5
:1030C0008DF8013004238DF8023055F021FFCDF842
:1030D000030004F58150CDF807101022694618301E
:1030E0008DF80B60039534F061FE04B070BD0000F4
:1030F000A120704738B5044600F5815501F0BCFFAA
:10310000183502460B49284634F06CFF04F500538D
:10311000284693F84D2C93F84C1C34F09FFF04F58F
:103120009150103004F086F904F59070BDE83840F5
:103130000CF06CBDCCEB080837B5069D044600B911
:103140002C7801B9697802B9AA7803B9EB78002024
:1031500064F3070061F30F2062F3174063F31F600D
:1031600003B030BD2DE9F04F2DED0C8B9DB0E04C40
:103170000D93D4ED379ADFEDDF5A90ED006A04F538
:103180000054F7EE006AD4F85C3CD3ED367A93ED48
:10319000387AF0EEE77AB0EEC77A77EE877A924621
:1031A000F4EEE67AF1EE10FAC8BF86EEA78A06467C
:1031B0000F46DFEDD17AD8BFB0EE668A28EE277AC7
:1031C000A6EE257A80ED007AD4F85C3C93ED357A52
:1031D00093ED376AB0EEC77AB0EEC66A37EE067A7C
:1031E000B4EEE67AF1EE10FACCBFC6EE878AF7EEBF
:1031F000008A90ED017A68EEA77AE7EE257AC0EDB5
:10320000017A35F015FC054655F082FE814618EE30
:10321000900A8846FDF770F9CDE9080118EE100A0A
:10322000FDF76AF9CDE906017068FDF765F9CDE9AA
:1032300004013068FDF760F9B04BB14ACDE90201F5
:10324000CDE900982846AF49AF4D35F063F9AF4955
:1032500095ED00AA384616F03BFE8DED160A9AED64
:10326000000ACDED170A30EE4A0A8DED181A14F057
:10327000A3FD9DED167AD4EDB07AB0EEC77AB4EE28
:10328000E77AA5F58963F1EE10FA0C9300F10F824D
:10329000D4F85C3C1B7B002B00F00982B4F8BE9292
:1032A000C9F340099DED177AB0EEC77AF4EEC77AFC
:1032B000F1EE10FA00F3FE81D4F85C3C1B7B002B8E
:1032C00000F0F881B4F8BE3203F001039DED187AE6
:1032D0000B93B0EEC77AF4EEC77AF1EE10FA00F372
:1032E000EB81D4F85C3C1B7B002B00F0E581B4F84B
:1032F000BE32C3F38008B0EEC00AF4EEC07AF1EE3D
:1033000010FA00F3DC81D4F85C3C1B7B002B00F04E
:10331000D681B4F8BE32C3F3C00B0DAB00930B994A
:103320009FED7B8A5B4642464846FFF705FFC3B2E6
:103330000BEE103AC0F307230AEE903AC0F30743AE
:103340000CEE903A030E0DEE103A9DF834300F90CB
:10335000002B40F0B7819DF83530002B40F0B28152
:10336000F8EE4B7A694ACDED197AF8EE6A7AB0EE4A
:10337000690ACDED1A7AF8EE6C7A19AB394602F586
:103380002070CDED1B7A4BF051FC8DED140ACDED84
:10339000150AB0EE409AF0EE608A9DF836305D4C2A
:1033A000002B40F094811CEE901AD4ED800A97ED2A
:1033B000020AB0EE691A04F22C504BF055FDB0EE43
:1033C00040CA9DF83730002B40F084819AED000A06
:1033D00030EE4A0A14F0F0FC1DEE101A4E48F0EEE2
:1033E000690A4BF057FA04F5C763DAF800201A604F
:1033F00004F23C63F0EE40BA83ED00AA474D95ED30
:10340000A91A4720F1EE410AB0EE490A14F0E8FC8F
:1034100095EDA91AB0EE40AAF1EE410A4820B0EEAF
:10342000680A14F0DDFC95EDAA1AB0EE409AF1EEB0
:10343000410A4920B0EE4C0A14F0D2FC95EDAB1ACB
:10344000F0EE408A4A20B0EE6B0AF1EE410A14F029
:10345000C7FC96ED007AD6ED017A9DF834308DEDFB
:10346000148A6AEE076AF0EE40BACDED106A69EE92
:10347000276A8DED158ACDED116AD4ED7B6A27EEB2
:10348000267AD4ED7C6A8DED127A67EEA67ACDEDC0
:10349000137AB3B99DF835309BB9B8EE4BBAF8EE54
:1034A0006AAAB0EE690A1E488DED19BA19AB12AAC4
:1034B00010A9CDED1AAA4BF0A5FA8DED140ACDEDA9
:1034C000150A9DF83630002B40F0078196ED000A72
:1034D000D4ED7D0A134860EE200A1CEE901A28EE07
:1034E000800AB0EE691A4BF0BFFCF0EE40AA1BE078
:1034F000A0250020A4707D3F00D7233C11F20808CE
:10350000281E0908411E0908E839002098570020A4
:1035100000000000A0550020445B0020A0450020D2
:103520007458002028590020844814A9FEF74CFE46
:103530009DF83730002B40F0D38096ED010AD4ED92
:10354000820A7F4860EE200AB0EE691A1DEE101A5A
:1035500020EE2B0A4BF088FCF0EE409AD5F85C3C4C
:103560001B7B7BBB19A977488DED198A8DED1A8AD3
:103570004BF072FB9FED740A74484BF091FC9FED89
:10358000720A73484BF0B2F919A972488DED198A85
:103590008DED1A8A4BF060FB9FED6B0A6E484BF085
:1035A0007FFC67489FED680A4BF07AFC04F5FC73DA
:1035B00093E807000C9B87E8070003F589631B6805
:1035C000CAF80030B9F1000F00F08D80D5F85C3CEE
:1035D00083ED368A0B9B002B00F09080D5F85C3C85
:1035E00083ED358AB8F1000F00F09380D5F85C3C8C
:1035F00083ED388ABBF1000F00F09580D5F85C3C74
:1036000083ED378A9FED558A9FED4F4AD4ED7B2A93
:1036100094ED7E1AD7ED000A62EE882A2AEE082A77
:1036200021EE081A60EE880AF0EE443AB0EE443A11
:10363000F0EE441AB0EE440A54F086FD9FED424A83
:10364000D4ED7C2A94ED7F1AD7ED010A62EE882A28
:1036500029EE082A21EE081A60EE880AF0EE443AB4
:10366000B0EE443AF0EE441AB0EE440A54F070FD65
:103670009FED354AD4ED7D2A94ED801AD7ED020AEC
:1036800062EEC82A28EEC82A21EE481A60EEC80A5F
:10369000F0EE443AB0EE443AF0EE441AB0EE440A8A
:1036A00054F05AFD1DB0BDEC0C8BBDE8F08F4FF00F
:1036B0000109F7E5012309E64FF001081BE64FF089
:1036C000010B2AE6F0EE488AB0EE489A65E69FEDD7
:1036D0001ECA76E6DFED1CBA90E6DFED1BAA23E7F3
:1036E000DFED199A3AE79DF83430002B7FF472AF82
:1036F000D5F85C3C149AC3F8D8206BE79DF83530B8
:10370000002B7FF46FAFD5F85C3C159AC3F8D4203A
:1037100068E79DF83630002B7FF46CAFD5F85C3C41
:10372000C3ED38AA66E79DF83730002B7FF46AAF07
:10373000D5F85C3CC3ED379A64E700BFA0250020B4
:10374000A0590020185A002000000000CC5A002088
:10375000445B002074580020285900200000C84213
:103760002DE9F04F2DED068B8FB0B74C0393D4EDC0
:1037700037AA04F500548046D4F85C3C1B7B0D4608
:103780001746002B00F02E81B4F8BE62C6F3400B42
:1037900006F0010AC6F3800916F0080600D00126DB
:1037A00003AB4A465146009358463346FFF7C4FCE4
:1037B00094EDA91A95ED000A0590F1EE410A9A20C0
:1037C00014F00EFB94EDA91AF0EE409AF1EE410AC6
:1037D00095ED010A9B2014F003FB94EDAA1AB0EEBC
:1037E000409AF1EE410A95ED020A984D9C2014F0A2
:1037F000F7FA94EDAB1AF0EE408A9D2097ED000A9F
:10380000F1EE410A14F0ECFA98ED007AD8ED017A65
:103810009DF80C3069EE876A0027CDED066A69EEE7
:10382000276AB0EE408ACDED076AD5ED7B6A0A972C
:1038300027EE267AD5ED7C6A8DED087A67EEA67ABA
:103840000B97CDED097AFBB99DF80D30E3B99DF8E2
:10385000143007EE103A9DF8153007EE903AB8EEA6
:10386000477AF8EE677AB0EE6A0A0CAB08AA06A9A6
:1038700005F535708DED0C7ACDED0D7A4BF0C2F873
:103880008DED0A0ACDED0B0A9DF80E30002B40F0AD
:10389000AE8098ED000AD5ED7D0A9DF816106C48B3
:1038A00060EE200AB0EE6A1A28EE800A4BF0DCFACD
:1038B000B0EE40AA64480AA9FEF786FC9DF80F30D6
:1038C000002B40F0978098ED010AD5ED820A9DF813
:1038D0001710604860EE200AB0EE6A1A20EE080A5F
:1038E0004BF0C2FAB0EE408AD4F85C3C1B7B7BB94B
:1038F00059480C970CA90D974BF0AEF99FED570A5C
:1039000053484BF0CDFA9FED550A52484BF0C8FA98
:10391000BBF1000F71D0D4F85C3CC3F8D870BAF199
:10392000000F74D0D4F85C3CC3F8D470B9F1000F28
:1039300077D0D4F85C3CC3F8E070002E7AD0D4F88D
:103940005C3CC3F8DC709FED468A9FED444AD5EDA0
:103950007B2A95ED7E1A62EE882A29EE882A21EECE
:10396000081AF0EE443AB0EE443AF0EE441AF0EEA3
:10397000440AB0EE440A54F0E7FB9FED384AD5ED17
:103980007C2A95ED7F1A62EE882A29EE082A21EE1C
:10399000081AF0EE443AB0EE443AF0EE441AF0EE73
:1039A000440AB0EE440A54F0D3FB9FED2C4AD5ED07
:1039B0007D2A95ED801A62EEC82A28EEC82A21EEEB
:1039C000481AF0EE443AB0EE443AF0EE441AF0EE03
:1039D000440AB0EE440A54F0BFFB0FB0BDEC068BB6
:1039E000BDE8F08F4FF00109CA46CB46D7E69FED00
:1039F0001BAA5FE79FED198A76E79DF80C30002B34
:103A00008DD1D4F85C3C0A9AC3F8D82087E79DF89A
:103A10000D30002B8AD1D4F85C3C0B9AC3F8D4202B
:103A200084E79DF80E30002B87D1D4F85C3C83ED01
:103A300038AA82E79DF80F30002B84D1D4F85C3C83
:103A400083ED378A7FE700BFA0250020A055002026
:103A500028590020A05900207458002000000000C0
:103A60000000C84270B5044610303FF04FFD0B4EC9
:103A70000B4B2361382560193FF066FF66513035E6
:103A8000B5F54E7FF7D104F54E7041F0DBF92046D5
:103A9000044930F095FD204670BD00BF7C27090821
:103AA00090270908A820090837B500F50951012217
:103AB0003831044632F0D6FD1C4A1368D90705D4C4
:103AC0001B4904F501530B600123136004F50B50EF
:103AD00017490122083030F02DFB0125002304F5A1
:103AE0008151CDE90053134A1831FD2030F0B4FA6A
:103AF000114B1A68D20705D4104A1D6004F58A5488
:103B0000083414600D48012130F030FB30F05EFFC6
:103B10000B4A0C48138843F0400313800421002211
:103B200003B0BDE8304030F093BA00BF445D0020E0
:103B300000220020B09F0908485D00200C220020D0
:103B4000785E0020982509080069C0F3401070478E
:103B50000F299DBF302303FB010028300020704750
:103B6000014B93F992027047A0450020024B93F855
:103B7000590C00F001007047A0450020014BD3F81C
:103B8000240A7047A0450020002910B517DB104C0F
:103B900094F82C2ACBB29A4211D3D4F8283A0122B5
:103BA000595CA4F5005000F073FD94F8493C38B915
:103BB0009A0704D5074A137843F00403137010BD25
:103BC0009B07FCD5034A137843F00203F6E700BFD6
:103BD000A04500200C5E0020022A10B50F4C12D127
:103BE0003522A4F5005000F053FD94F8493C9B07A2
:103BF00005D50B4B1A7818B142F002021A7010BDAD
:103C000042F00402FAE794F84C2C8A42F7D13FF0D4
:103C10005FFEBDE810403FF05FBD00BFA045002043
:103C20000C5E0020064A92F8593C92F8582C03F09A
:103C30000103134301D13FF05FBC0020704700BF78
:103C4000A0450020332901D040F01CBC7047000083
:103C500008B50A68332A07D0382A08D10A7903211F
:103C6000FFF7BAFF012008BD0A790121F8E7BDE896
:103C7000084040F0ADB9000030B5044689B0684650
:103C800004F5915506F048FD103504A806F044FDF2
:103C90006946284602F0CAFF70B104A9284602F01E
:103CA000F5FF48B104A9684606F064FD23680022C8
:103CB0001B6D69462046984709B030BD00F580521B
:103CC00092F8C424D2070AD400F50052D2F85C2C32
:103CD000117B09B1FFF7D0BF0368DB6C1847704751
:103CE00010B586B0044602A8019106F015FD04F552
:103CF000915002A9103002F099FF28B12368019A6F
:103D00001B6D02A92046984706B010BDF0B50446C9
:103D100085B004F59156684610360F46154606F0F4
:103D2000FBFC6946304602F0B1FF10B9002005B037
:103D3000F0BD3946304602F0C9FD0028F6D0002D0E
:103D4000F5D004F58054284694F8C43443F00203B7
:103D500084F8C434EBE7000010B500F50054D4ED4E
:103D6000A77AF5EEC07AF1EE10FA8AB04FF00003B0
:103D700044D907930893099306AB019300F591503A
:103D800007AB03AA04A90093103005AB02F03CFE78
:103D9000DDED080A9DED070A73F0EEFEDDED090A80
:103DA00073F0EAFED4EDA77A9DED047A77EEA76A68
:103DB000B4EEE70AF1EE10FAF4EEC76AACBF0120E8
:103DC0000020F1EE10FA0CD802309DED037AF4EEEB
:103DD000C77AF1EE10FA0CD8003818BF01200AB0EB
:103DE00010BDF4EEC77AF1EE10FA9CBF0130C0B2FC
:103DF000EBE7012894BF00200120F0E70020EEE768
:103E000038B500F50055044695F8593C5A071AD4C0
:103E100043F0040385F8593C34F00AFE01221121D5
:103E200034F062FD084BD3F8980603689B68984706
:103E300018B995F99932032B05D120460621BDE822
:103E4000384000F023BD38BDA055002008B500F56E
:103E5000005090F8593C5A070BD56FF3820380F855
:103E6000593C34F0E5FDBDE808400022112134F052
:103E70003BBD08BD2DE9F043054685B005F59158D9
:103E8000684608F1100806F047FC6946404602F013
:103E9000FDFEC8B105F50053424CD3F85C2C424FEF
:103EA000127B32B1D3EDA77AF5EEC07AF1EE10FABB
:103EB0000DD8238823F4FF7323F0010323802846C1
:103EC0000023FB73FFF7C2FF05B0BDE8F08328466F
:103ED00001F076F8064618B9284601F035F806468E
:103EE0002846FFF739FF814640B93EB12378002BC1
:103EF00041D1637803F00103FB73E5E76378DB07E7
:103F0000F7D423780133DBB2082B237006D128467F
:103F1000FFF722FF10B1404602F0E2FD2378092BA3
:103F200002D1404602F0D4FD2378092BE1D9238841
:103F300023F4FF7323F0010343F48573238034F0EB
:103F400077FD0222102134F0CFFC54F0D9FF6368D2
:103F5000C01A47F23053984209D905F52A50134A3E
:103F60000221043039F048F854F0CAFF6060284656
:103F7000FFF746FFBDE7013B23702388C3F3080327
:103F8000B3F5807FB5D1637860F30003637034F0DC
:103F90004FFD4A46102134F0A7FC2846FFF756FF94
:103FA000A7E700BF4C5D0020ED5D0020AC270908AD
:103FB00037B5044600F5915001A9103004F50055BD
:103FC00002F0CEFBD5F8703A834206D0C5F8700AED
:103FD00034F02EFD3E2134F067FC04F5805395F952
:103FE000741A93F8582593F95835994213D0FF2A3B
:103FF00011D085F8743A34F01BFD95F8742A182115
:1040000034F072FC042104F52A5095F9743A034AFD
:10401000084438F0F1FF03B030BD00BFBC270908E9
:104020002DE9F04395B0064654F06AFF06F5915825
:1040300003AB019308F1100802AB0024009305467E
:104040000EAB0BAA08A94046089409940A940B9455
:104050000C940D940E940F94109402F0C3FCDFEDB9
:10406000437A9DED0A7AB4EEE77AF1EE10FA07464C
:1040700037DB9DED0D7AB4EEE77AF1EE10FAACBFC6
:104080004FF001094FF0000907AB019311AB00930A
:1040900004AA06AB05A9404611941294139402F0A9
:1040A000B3FC06F50054002894F90C3A08BF002729
:1040B00083B17FB1D4F85C3C1B7B5BB1B9F1000FDD
:1040C00008D09DED057AF7EE007AB4EEE77AF1EECE
:1040D00010FA09D594F8783A73B90023C4F87C3AF9
:1040E0000FE04FF00009CFE7D4F87C0A20BBC4F8FA
:1040F0007C5AC4F8800A04E0D4F8800A20B9C4F8D5
:10410000805A15B0BDE8F083281A43F698239842E8
:10411000E3D9002584F8785AC4F8805A34F088FC32
:104120002A461D2134F0E0FB06F52A50104A0221F0
:10413000043038F061FFD0E72D1AB5F57A7FE0D969
:1041400094F8783A002BDCD1012584F8785A34F0C1
:104150006FFC2A461D2134F0C7FB06F52A50054A9C
:104160000221043038F048FFCBE700BF00000034E4
:10417000D4270908EF27090810B5044634F058FC85
:104180000022052134F0B0FB04F52A500421BDE8DB
:104190001040024A084438F02FBF00BF0C2809081D
:1041A00000F5005090F8493C9B065ABF90F8480C27
:1041B000C0F300100120704738B5044602F082FFBA
:1041C0004FF4804102F0BCF804F50052054692F825
:1041D000493CC3F3001181421CD060F3041304F581
:1041E0002A5482F8493C043460B134F021FC0222A4
:1041F0000B2134F079FB084A20460221BDE8384003
:1042000038F0FABE34F014FC2A460B2134F06CFB73
:10421000024AF1E738BD00BF242809082F28090801
:1042200070B500F50055044695F98232B3B3D5F860
:10423000D46B9EB354F064FE05F6142393ED000A8C
:10424000DFED177A9FED171ADFED170A861B20EEB8
:10425000270A692013F0C4FDBCEEC00A10EE103A24
:104260009E4209D295F8593C9A0717D5204600215D
:10427000BDE87040FDF78EBC10D995F8593C9B07FE
:104280000CD420460121FDF785FC04F528500122BD
:10429000BDE8704012213030FDF7D4BB70BD00BFC7
:1042A00000007A440000804F000000000B46012B04
:1042B00010B4114604D0052B06D05DF8044B7047AE
:1042C0005DF8044B00F0E2BA00F528505DF8044BAD
:1042D000012214213030FDF7B5BB00002DE9F0417B
:1042E000044604F5005834F0A3FB0122052134F004
:1042F000FBFA98F986522046003D18BF0125FFF7CA
:104300004FFF04F52A56043698B11E4A0421304660
:1043100038F072FE04F52850012210213030FDF7EC
:1043200091FB0025294620460322BDE8F041FFF716
:10433000BDBF04F54057D7F898060368DB6A984775
:1043400068B197F8BD3153B197F9BC31012B06DC48
:104350000D4A0421304638F04FFE0125E2E7D7F838
:1043600098060368DB6A984718B1D8F8103A1B071B
:1043700005D4064A0421304638F03EFED2E7044A0E
:10438000E7E700BF442809085F2809088D280908C5
:104390009C28090870B50446154634F049FB0122F3
:1043A000062134F0A1FA2046FFF7FAFE04F52A565A
:1043B000043698B104F52850012207213030FDF76A
:1043C00041FB154A0421304638F016FE00252946E7
:1043D00020460422BDE87040FFF768BF04F5405353
:1043E000EDB2D3F898060368DB6A984768B104F524
:1043F0000053D3F8103A1B0707D535B1074A0421FB
:10440000304638F0F9FD0125E1E7054A0421304640
:1044100038F0F2FDDBE700BFC0280908672809086B
:10442000DD280908F8B5044654F05EFD284BB4F8C1
:10443000BE201988274E914205460ED01A80264B81
:1044400018603378A3B10024347034F0F1FA2246B6
:104450001321BDE8F84034F047BA33781F4FC3B991
:104460003B782BB11C4B1E4A1B68C31A934200D8E1
:10447000F8BD0123337004F50053D3F85C0C037BC3
:104480000BB1FEF725FA34F0D3FA0122132134F0F0
:104490002BFA3B78002BEBD03378002BE8D00E4A78
:1044A00010491368EB1A8B42E2D904F500541560E9
:1044B000D4F85C2C137B002BDAD0002313730A4A48
:1044C000D4F85C0C1371BDE8F840FEF7D1B800BF1A
:1044D000565D0020545D0020585D0020555D002091
:1044E00080841E0040420F00ED5D00207FB500F586
:1044F000005300F54A550446383593F8781A284693
:1045000004F5915653F07EFD1036684606F004F926
:104510006946304602F08AFB04F54053029AC3F81C
:10452000D821039AC3F8DC212021304601F008FF8E
:10453000D0B1284653F0B8FD04F54755FDEEC07ADA
:10454000103504F5805417EE901A0222284617EE13
:10455000906A06F0E5F894F8C434DB0706D401222B
:104560003146284606F0DCF804B070BD012128462B
:1045700006F07EF90028F2D0F6E70000012070472F
:1045800000207047002070470020704700207047CF
:104590000020704700207047002070479FED010AFF
:1045A000704700BF000000009FED010A704700BF88
:1045B0000000000070470000104A0260104A42608C
:1045C00002F15001816002F58251C1600D49016123
:1045D00002F6E411416102F6E811816102F5F4612D
:1045E000C16102F2A471016202F5F56102F2AC72DE
:1045F0008262054A4162C262704700BF68290908A9
:1046000018480020D0370020B8260020042917D8E9
:10461000DFE801F003070B0F130000F55B500C30CF
:10462000704700F55A501C30704700F55B503C3025
:10463000704700F55C502C30704700F55D50FAE78C
:104640000020704700F54050D0F8980603685B687A
:104650001847000038B500F540550446D5F89806CF
:1046600003685B699847094B04F50052187492F887
:104670004C2CD5F89806DA7003685B6A98470146B7
:1046800004F58F50BDE838402DF0D0B9ED5D002025
:104690002DE9F84F00F5005A06469AF84C3C8B423B
:1046A0000F46914605D18AF84D2C01252846BDE8D4
:1046B000F88FFFF7ABFF044620B9304632F078F9A7
:1046C0002546F3E7DAF85C3C1B7B06F52A5883F0B5
:1046D000010B08F10408EBB9236859461B68204612
:1046E0009847054680B306F5405306F58150C3F858
:1046F00098464A4639468AF84C7C8AF84D9C1830D0
:1047000033F0ACFC404600213EF0A2F93046FFF702
:10471000A1FFCBE703689B689847E0B11C4800F015
:1047200039FC0546B8B9236820461B6A9847194AE0
:1047300003460421404638F05FFC34F079F93A46EC
:104740000A2134F0D1F8B1E7236820461B6A984764
:10475000114A0346EDE70E4800F03AFC0028BBD1B1
:1047600006F54053D3F898060368DB68984700289D
:10477000B2D023682046DB68984705460028ABD1B5
:10478000236820461B6A9847044A0346D1E700BFC6
:10479000A0250020F028090842290908192909083C
:1047A0000148FFF775BF00BFA025002070B5234B5F
:1047B00093F8593CDB0705460C46164605D5002301
:1047C00063602360A360336070BD3FF081F8037FB6
:1047D000002BF4D0EB699FED1A7A1B68B3F90A300D
:1047E00007EE903AF8EEE77AC7EE876AC4ED016A01
:1047F0002B6A1B68B3F90A3007EE903AF8EEE77AB5
:10480000C7EE876AC4ED006A6B6A1B68B3F90A30A9
:104810005B4207EE903AF8EEE77AC7EE876AC4ED9E
:10482000026AAB6A1B68B3F90A3007EE903AF8EEF9
:10483000E77AC7EE876AC6ED006AC5E7A0450020A3
:1048400000007A4400207047012070470020704724
:104850000020704700487047587A090800487047A0
:10486000B02909080020704743691A680023C2F87C
:10487000D43042691268C2F8D83042691268C2F86E
:10488000DC3042691268C2F8E03070470A4608B569
:104890000021FFF7FDFE034A137843F0080313706D
:1048A00008BD00BF0C5E002001207047002070474B
:1048B000012070470020704700487047082A090807
:1048C00000487047102A09080320704730B5084B8C
:1048D00003F547523832044600F1300507CA85E82F
:1048E000070003F5A253083301201B68E36330BDC2
:1048F000A025002030B52DED028B044687B0574D22
:10490000002301AA03A995ED378A03930493059325
:10491000FFF74CFF63689DED037AD3ED0E7A68EEE6
:10492000277A27EE277A8DED037A9DED047A67EEDC
:10493000277ACDED047AD3ED0F7A28EE277ADDEDD4
:10494000057A67EE877ACDED057AD3ED107A93F983
:10495000443028EE278ADDED017A27EE888A8DED36
:10496000018A1BB903A92846FDF712FC3C4A94EDC5
:104970000C7AD2ED7E7A636894ED0F0AD3ED0E6A5D
:1049800077EE677AF0EEE77AF4EEE67AF1EE10FA77
:1049900044BFDDED037A77EE877A94ED0D7A48BF58
:1049A000C4ED0C7AD2ED7F7AD3ED0E6A77EE677A9A
:1049B000F0EEE77AF4EEE67AF1EE10FA44BFDDEDC0
:1049C000047A77EE877A94ED0E7A48BFC4ED0D7ABB
:1049D000D2ED807AD3ED0F6A236977EE677AF0EE35
:1049E000E77AF4EEE67AF1EE10FA42BFDDED057AF1
:1049F00077EE877AC4ED0E7AD3ED867A30EE670AC9
:104A000013F0DAF96368D3ED107AB0EEC00AB4EEB1
:104A1000E70AF1EE10FA09D594ED0F0ADDED017AFF
:104A200030EE270A13F0C8F984ED0F0A00230D4871
:104A30008DF808308DF809308DF80A308DF80B307C
:104A4000029BD0F8600C04F13C0204F13001FEF747
:104A500089FB07B0BDEC028B30BD00BFA025002054
:104A6000A0550020A045002000207047012070477D
:104A7000012070470020704700487047682A0908E5
:104A800000487047702A0908012070471FB5044686
:104A900000236A4601A9019302930393FFF786FE60
:104AA0006369029A1B68C3F8D4206369019A1B6882
:104AB000C3F8D8206369009A1B68C3F8DC206369D7
:104AC000039A1B68C3F8E02004B010BD01207047B2
:104AD0000020704701207047002070470048704751
:104AE000EAF6080800487047EAF60808042070470C
:104AF000012070477FB5002303930493059301932E
:104B0000094800238DF808308DF809308DF80A30F7
:104B10008DF80B30029BD0F8600C01AA03A9FEF7B8
:104B200021FB07B05DF804FBA04500200120704781
:104B300000207047012070470020704700487047F0
:104B4000182B090800487047242B090802207047D9
:104B500010B5044686B0002301AA03A90393049369
:104B60000593FFF723FE63689DED037AD3ED0B6A8F
:104B7000DDED047A93F9443027EE267A67EEA67AC3
:104B80008DED037ACDED047A1BB9144803A9FDF726
:104B9000FFFA6368DDED057A93ED0C7A104867EE55
:104BA000877A93ED0D7ACDED057ADDED017AD0F8B7
:104BB000600C002367EE877A8DF808308DF8093095
:104BC0008DF80A308DF80B30029BCDED017A01AAE9
:104BD00003A9FEF7C5FD06B010BD00BFA02500204B
:104BE000A045002038B5044640F082F940F050FA64
:104BF00004F50054054640F0E5F93FF0D7FED4F83F
:104C00005C0CFDF735FD2846BDE8384040F0E2B9C0
:104C100010B500F500541421D4F8180A3EF0A8FE8F
:104C2000D4F81C0A14213EF0A3FED4F8200A1E2159
:104C30003EF09EFED4F8240A1421BDE810403EF058
:104C400097BE000038B505463EF042FE3EF094FDAA
:104C500005F50054C4F8180A3EF03AFE3EF096FD01
:104C6000C4F81C0A3EF034FE3EF09AFDC4F8200A57
:104C70003EF02EFE3EF09EFD4FF47A71C4F8240AF9
:104C8000D4F8180A3EF070FED4F81C0A4FF47A717A
:104C90003EF06AFED4F8240A4FF47A713EF064FEC6
:104CA000D4F8200A4FF47A713EF05EFE2846FFF7F2
:104CB000AFFF94F8493C43F0080384F8493C38BD01
:104CC00008B540F0E5F940F009F8BDE808403FF0CC
:104CD000BBBF000000F50050D0F85C0CFDF7F8BD3C
:104CE00038B500F50054054694F986322BB90021F9
:104CF0002846BDE83840FCF733BFB4F888328B4211
:104D000019D994F8593CDA070FD43EF0E1FD037F3E
:104D10001BB9D4F85C3C1B7B3BB194F8583C013385
:104D20005BB2022B02DC84F8583C38BD032384F8C4
:104D3000583C0121DCE794F8583C013B5BB2002B66
:104D4000F1DC002384F8583C94F8593CDB07CED4BE
:104D5000EBE7000038B50D46044654F0D1F8002DBD
:104D60000B4B09DD04F50054186094F8493C6FF3CF
:104D7000C30384F8493C38BD1B68C01AB0F5C87F2E
:104D8000F9D904F5005494F8493C43F00803F0E7DE
:104D90005C5D0020F7B5044654F0B2F806463EF0DC
:104DA00097FD3EF069FD04F50055B0B395F8483C19
:104DB00043F0200385F8483CD5F8203A204619896D
:104DC000FFF78EFFD5F8203A04F54057B3F90A10E3
:104DD0002046FFF7BFFFD7F890369FED307AF31AE1
:104DE00007EE903AD5F8203AF8EE677AB3F90A3030
:104DF00067EE877A04F54750CDED007A07EE903ADA
:104E0000F8EEE77A6A4601A90430CDED017A34F074
:104E100099FFC7F8906603B0F0BD95F8593CDB07E1
:104E2000F9D404F54053D3F89006361A3EF006FC48
:104E300080BB3EF04DFD9FED1A7AD0ED067A67EE0D
:104E4000877A9FED187AF4EEC77AF1EE10FAD8BFA0
:104E5000F0EE477AFCEEE77A17EE903AB342DAD8F2
:104E600095F98632002BD6D03EF032FD037F23B970
:104E7000D5F85C3C1B7B002BCDD033F0D9FD022252
:104E8000114633F031FD0121204603B0BDE8F0406A
:104E9000FCF766BE4FF47A73E0E700BF6F12833A07
:104EA00000007A440000C84238B5044600F5866523
:104EB000284604F097FB94F841049FED087A2422D9
:104EC00002FB0055D5ED0B7A67EE877A04F5405367
:104ED000FDEEE77AC3ED707A38BD00BF0000C8422E
:104EE000FEF708B90148FFF79DBA00BFA0250020D2
:104EF00010B5838F044643B932F06AF892224FF41A
:104F0000801132F01DF8638FA387A08F10BD0000C1
:104F100038B500F5915510350446284600F0E2FCFE
:104F200004F58053022283F8502404F16800FFF74F
:104F3000DFFF014604F6980012F0F6FA2846BDE8B5
:104F4000384000F0C9BD000038B500F59154103468
:104F50000546204600F012FF08B9002038BD05F5CF
:104F60000055D5F85C3C1B7B63B91021204601F04D
:104F7000E7F90028F2D14FF400712046BDE838402F
:104F800001F0DEB98021204601F0DAF90028E4D1F1
:104F90001021F2E738B500F50053054693F8593C67
:104FA0005B070AD4FFF7D0FF044620B905F59150FE
:104FB000103000F0E3FE204638BD0024FBE700007F
:104FC00008B500F59150103000F0D8FE002008BD63
:104FD00010B500F591541034204600F0CFFE50B1CA
:104FE0000421204601F0ACF928B120462021BDE87B
:104FF000104001F0A5B9002010BD000038B500F543
:105000000055044695F8483C590719D5D5F85C3C3D
:105010001B7B2BB920460021BDE83840FCF78ABD38
:1050200000F54053D3F898060368DB68984738B119
:1050300095F8493C1A0703D595F8593CDB07E9D5A3
:1050400038BD000037B500F581551835044604F524
:1050500000542846019132F049FF94F8483C0199E8
:1050600060F3C303284684F8483C03B0BDE83040F1
:1050700033F0A8BC07207047004870477C2B090814
:1050800037B505461048FFF733FF0190EC2005F0D7
:1050900067FE044610B10199FDF78AFA05F5005044
:1050A000C0F85C4C24B990F9D412084805F0FEFA17
:1050B000074920462FF092FC01202EF0BBFE03B0E2
:1050C000BDE830402FF082BC08260020842B090860
:1050D00060EB080873B5044600F58F502CF05AFCBD
:1050E0002046FFF7B7FA04F53150303004F03AFEAD
:1050F00004F58750103004F5866640F031FC3046E8
:1051000004F010F904F52A5004303AF0ADFB2046C3
:10511000FFF798FD2046FFF7B3FF6048FFF7E8FE72
:10512000082005F01DFE18B14FF07E530360436068
:1051300004F50055C5F8600C3EF0CAFB9922292100
:105140003FF074FB3EF0C4FB3EF0E4FA2046FFF76C
:10515000B7FD95F8493C04F58D5043F0400385F8C0
:10516000493C0C3042F008F94D4B4E491B68986A97
:1051700003684FF47A72DB6A98470423C4F87431E9
:1051800004F590700AF0B8F906F0A8FB4FF400534C
:10519000036306F0A3FB06F035FC8023C4F8443417
:1051A0000121304604F02EFB3F4B00933F4B01930F
:1051B00004F5815002AB13E90600183032F042FDCD
:1051C0002046FFF7A5FE4FF40023C4F8A83BD5F80E
:1051D0005C0CFDF7F7F904F5285001213030FCF79D
:1051E0009BF910B12046FFF775FD04F168063046C3
:1051F000FFF77EFED5F85C3C07EE900A04F54850B8
:10520000D3ED390AB8EE670AF2EE0E1AB6EE001ABE
:105210000C3035F06DFA3046FFF76AFED5F85C3C8D
:1052200007EE900A04F54950D3ED390AB8EE670A43
:10523000F2EE0E1AB7EE001A103035F083F8304651
:10524000FFF756FED5F85C3C07EE900A04F54A508D
:105250000430D3ED390AB8EE670AF2EE0E1AB1EE59
:10526000041A35F06FF895F893121A222046FFF7CA
:105270000FFA60B9212201212046FFF709FA95F8BB
:10528000493C43F0020385F8493C02B070BD084A2E
:10529000137843F008031370F1E700BF08260020DD
:1052A000405D0020E54E0108A0250020E14E0108E8
:1052B0000C5E0020836833B9C36823B940680038A6
:1052C00018BF012070470120704700002DE9F04110
:1052D0002DED048B92B0044602AD284605F01CFA71
:1052E00094F8D433002B70D004F580630FCB85E89D
:1052F0000F0094F81034D4EDF28A94EDF38A94ED13
:10530000F49A002B61D094F8E833002B5DD0284646
:10531000D4F8D883D4F8DC73D4F8E063D4F8E44349
:10532000FFF7C8FF002855D12E4B01932D220021F5
:1053300006A874F07BFFA3238DF8183095238DF811
:10534000193046238DF81A3053F0E2FD9FED260AFE
:10535000DFED267ACDF81F1068EE808A28EE008AED
:1053600068EEA78A28EE278AFDEEE88ABDEEC88A95
:1053700018EE903A29EE000AADF8233018EE103AF4
:1053800020EE270ACDF81B00ADF8253012F0E8FC1E
:10539000BCEEC00ACDF8358010EE103AADF82730DB
:1053A000019BCDF82930049BCDF82D30059BCDF81D
:1053B0003130CDF83970CDF83D60CDF8414033F053
:1053C00037FB2D2206A932F071FC12B0BDEC048B24
:1053D000BDE8F08101AA0021284605F059FA00280D
:1053E000A2D0A3E75241C07FE02E65420000C84230
:1053F00030B52DED028B8BB0044624220D4601A85A
:10540000002174F013FFA3238DF8043095238DF849
:10541000053048239FED1F8A8DF8063053F078FD44
:10542000D4ED847A2B68CDF80F3067EE887A95ED4D
:10543000020ACDF80B1017EE903AD4ED857ACDF82C
:10544000133067EE887A6B68CDF8173017EE903A14
:10545000CDF80700CDF81B3012F058FC10EE103AD2
:1054600094ED860ACDF81F3020EE080A12F04EFCAB
:1054700010EE103ACDF8233094F824338DF827300D
:1054800033F0D6FA242201A932F010FC0BB0BDECA7
:10549000028B30BDE02E654230B5104689B00D4616
:1054A0001446FFF707FF28BB0023019318220021B1
:1054B00002A874F0BBFEA3238DF8083095238DF865
:1054C000093049238DF80A3053F022FDA368059373
:1054D000E3680693019BCDF80F100793CDF80B00FE
:1054E0008DF8135033F0A4FA182202A932F0DEFB33
:1054F00009B030BD01AA0021204605F05DF9002861
:10550000D2D0D3E710B590B0044604A805F004F952
:1055100004A9204601F08AFB002846D001F0D2FD04
:1055200001A901F07DF902A9204600F0C3FC002882
:105530003DD0DDED027AF1EE677A03AA002104A8DE
:10554000CDED027A05F0A4F908B91A4B03931F2296
:10555000002108A874F06AFEA3238DF8203095235B
:105560008DF821304A238DF8223053F0D1FC069B70
:10557000DDED017ACDF82B30079BCDF82F30F1EE21
:10558000677A039BCDF8333017EE903ACDF8373079
:10559000029BCDF82710CDF82300CDF83B3033F037
:1055A00047FA1F2208A932F081FB10B010BDDFEDD1
:1055B000027AC2E75241C07F5241C07F002303609C
:1055C00043608360C360036143618361C3610362BD
:1055D0007047000090F8C432B02202FB030390F839
:1055E000082393F8A13012B1012B28BF01231846DC
:1055F000704700002DE9F04F04468BB04FF0000AD1
:105600000D4618F08DFC84F820A204F509704FF0C7
:105610007E5752F031FE4FF47A73A4F87A3284F850
:10562000805204F52170C4F86072C4F86472C4F842
:105630006872002505F070F804F531790323C4F889
:10564000983204F53A76C4F8AC52C4F8B052C4F8B3
:10565000B452C4F8B852C4F8BC52C4F8C052484658
:10566000FFF7ACFF04F54E7B3046FFF7A7FFC4F809
:105670002C53C4F83053C4F834535846FFF79EFFF8
:10568000C4F85C53C4F86053C4F86453C4F8685356
:10569000C4F86C53C4F87053C4F87453C4F8785306
:1056A000C4F87C53C4F88053C4F88453C4F88853B6
:1056B000C4F8A453C4F8A853C4F8AC53C4F8C053F6
:1056C000C4F8BC53C4F8B853C4F8C853C4F8CC5396
:1056D000C4F8D053C4F8E453C4F8E053C4F8DC531E
:1056E00004F57B70C4F8B473C4F8D87305F014F8EB
:1056F00004F5806005F010F804F2144304F58660A8
:105700001D605D6004F5846304F27C481D605D608B
:105710009D6005F001F804F2444340461D605D6061
:105720009D606D4BC4F8543404F51073C4F85834BC
:1057300004F51173C4F85C3404F51273C4F86034D2
:1057400004F51373C4F8643404F25123C4F86834C4
:1057500004F51473C4F86C3404F58E6304F25442F7
:105760001D605D609D60FFF729FF04F59460FFF701
:1057700025FF04F59A6304F2BC501D605D609D60D6
:1057800004F2DC431D605D609D6004F59D631D6057
:105790005D609D6004F2F4431D605D609D6004F2F5
:1057A00004531D605D609D6004F214531D605D60D4
:1057B0009D6004F5A763C2F8D470C2F8D8701D606C
:1057C0005D609D6004F244531D605D609D6004F562
:1057D000AC631F605D6004F284531D605D609D607A
:1057E00004F5B2631D605D609D6004F5B5631D60E6
:1057F0005D609D6004F090FF04F2CC5324221D6094
:105800005D6004F2D45351461D605D6004F2DC53C8
:1058100040461D605D6074F009FD04F5C060C8F885
:105820002070C8F81070C8F80070FFF7C7FE04F2C7
:10583000246304F27C601F609D605D60DD6004F2A3
:1058400034631D605D609D6004F5C8631D605D602C
:105850009D6004F24C631D605D609D6004F5CB6348
:105860001D605D609D6004F264631D605D609D600D
:1058700004F052FF194B1A491C6020462EF0A0FE7E
:1058800051462422584674F0D1FCC4F85873C4F829
:105890004873C4F8387304F52B7207CA04F52E73E5
:1058A00083E80700484694EDB01AD4EDAF0A94EDB2
:1058B000AE0A12F06DFE3546494668466E4612F055
:1058C00089FD0FCE0FC50FCE0FC533682B60204664
:1058D0000BB0BDE8F08F00BF642E0908605D0020AA
:1058E000002D090810B5044688B001F057FC94F962
:1058F0003E32012B02D1274804F0F6FE022B0AD1DA
:10590000032384F83E3204A9012304F111008DF829
:1059100010302FF015FC94F83E3284F8A83204F2CF
:10592000544001F0F7FB94F93D32642B30D16523EC
:1059300004A904F23D208DF810302FF03FFC04A99B
:1059400020462EF0B7F818B304238DF81830002342
:10595000CDE9013303930F230593694604A82EF084
:105960007FFA059B28B108AA02EB8302009942F84E
:10597000581C0133112B0593EFD951F06DF89DEDB3
:10598000031ADDED020A9DED010A652151F022F8AE
:1059900008B010BD942B090870B500F52B7600F502
:1059A0002E758CB004463146284614F031FAE0B921
:1059B00096E8070085E8070004F5317194EDB01A08
:1059C000D4EDAF0A94EDAE0A0191084612F0E0FD65
:1059D00002AD019902A812F0FDFC0FCD04F53A7456
:1059E0000FC40FCD0FC42B6823600CB070BD000036
:1059F00013B540F2751200F50971044601A80EF0C6
:105A000057FD04F2544001F06FFD204618F0B4FC3D
:105A100001A80EF06FFD02B010BD0000F8B54B6894
:105A2000C0F810328B68C0F81432CB68C0F8183256
:105A300001F1100607460C4600F54E750FCE0FC556
:105A40000FCE0FC533682B6004F1440207CA07F577
:105A50004B7383E8070004F1500207CA07F5577338
:105A600083E8070004F15C0207CA07F55A7383E86C
:105A70000700683494E8070007F55D7383E80700C2
:105A8000384601F09FFC3846BDE8F84001F082BC82
:105A900013B5044600F25440019003F03DF904F5BB
:105AA000BE610198009102F025FD0099204602B0E8
:105AB000BDE81040FFF7B2BF4A78064BC2F3401270
:105AC0001A754A78C2F380125A750A78C2F3001226
:105AD0009A757047ED5D002013B540F24D320446D3
:105AE00000F5097101A80EF0E3FC002104F2544016
:105AF00001F028FF94F8783223B1204619F0BEF95E
:105B000084F8780201A80EF0F5FC02B010BD000088
:105B100038B590F8243305460C462BB1032B0BD037
:105B200095F88032DB070CD405F27C630FCB84E858
:105B30000F0095F88C0603E018F09EFC0028EFD0CB
:105B400038BD0020FCE7000000F2544090ED350A1B
:105B50007047000000F2544090ED360A7047000094
:105B600010B490F824230C462AB1032A0AD000204E
:105B70005DF8044B704700F5B56007C884E807007E
:105B80000120F5E75DF8044B18F034BC90F89C0355
:105B9000431E58425841704738B590F824330D469B
:105BA0008BB900F2544001F007FD044610B90024FF
:105BB000204638BD01F05EFCD5ED007A27EE800A64
:105BC00085ED000AF4E7D0EDE67AC1ED007A90F8B1
:105BD0009443002CEBD090EDE47ADFED086AB4EE4C
:105BE000E67AF1EE10FAF7EE006AB8BFB0EE667A28
:105BF00067EE877AC1ED007ADAE700BF0000003473
:105C000090F82433032B01D118F074BB00207047A7
:105C100090F82423032A01D118F0E6BC00F2544086
:105C200002F0EAB830B5054685B00C469AB1032AB1
:105C30001BD005F52B7014F025F901A920468DED38
:105C4000010ACDED020A8DED031A13F0C9FE0123FE
:105C5000184605B030BD90F8F035002BF8D000F2B2
:105C600024630FCB84E80F00E3E790F87832002B31
:105C7000EED018F093FCDCE790F82423FFF7D2BFB6
:105C80007FB590F8242332B1032A4FF0000309D0E6
:105C9000039304930CE000F2544007B05DF804EB6A
:105CA00001F0D4BC03A903930493059318F018FBE7
:105CB0009DED030ADDED040A07B05DF804FB00006A
:105CC00037B5044640F2C7520D4600F5097101A8E8
:105CD0000EF0EEFB2046294618F0F8FB94F824332A
:105CE000032B08BF044601A818BF00240EF002FCD5
:105CF000204603B030BD000010B52DED028BB0F88A
:105D000090361B0782B0044630D5D0F838349FED6A
:105D1000198A07EE903AB8EEE77A01A927EE087AD9
:105D200000F515708DED017A2FF0F6F9D4F83C34BA
:105D300007EE903AF8EEE77A01A967EE887A04F563
:105D40001670CDED017A2FF0E7F9D4F834349FEDD9
:105D50000A7A07EE903AF8EEE77A01A967EE877AB9
:105D600004F51770CDED017A2FF0D6F902B0BDEC35
:105D7000028B10BD95BFD6330AD7233C90F824037D
:105D8000003818BF0120704738B590F82423032A43
:105D90000C4604D118F0A4FA0125284638BD90F825
:105DA0007056002DF9D000F2646393E8070084E890
:105DB0000700F2E710B590F8242303460C461AB109
:105DC000032A0BD0002010BD90F878060028FAD0E6
:105DD00003F5BE63D3F884300B60F4E718F096FA4D
:105DE000012084ED000AEEE730B590F8243385B049
:105DF00005460C4623B1032B09D0002005B030BD69
:105E000000F2544005B0BDE8304002F075BA0023FE
:105E100002A90293039318F04BFA0028EDD001A9D0
:105E2000284618F051FA0028E7D0029B2360039B14
:105E30006360019BA360E1E71FB500230C4601A945
:105E4000019302930393FFF7CFFF28B1019B2360D7
:105E5000029B6360039BA36004B010BD90F82423F1
:105E60001AB1032A05D00020704700F2544002F016
:105E700077BA18F01DBA000013B500230C46694626
:105E800000930193FFF7EAFF18B1009B2360019B89
:105E9000636002B010BD000090F824231AB1032AF9
:105EA00005D00020704700F2544002F04BBA18F0C1
:105EB0000BBA000013B50C4601A9FFF7EDFF08B1BE
:105EC000019B236002B010BD90F93E323BB990F8BF
:105ED000803213F0010F14BF03200020704703200D
:105EE00070470000F7B50446FFF7EEFF05460028AF
:105EF00062D0032839D194F878326BB394F88032A9
:105F0000D8072BD501A9204618F0A6FBBDF8043010
:105F1000002B18BF002594F8206206F0FD06012E24
:105F20004AD10023032D019307D101A9204618F07F
:105F30009FFB204618F07CFB064604F2544002F01A
:105F40001FFB08B994F821039DF80430D90703D545
:105F50005A0701D59F0632D400252DE0204618F0BF
:105F60000DF9002808BF0025D5E70025D3E713F079
:105F7000020F2EE094F9503223B99DF80430DB096A
:105F80002FD0E9E7002EF8D00AF0DCFDFFF722FB66
:105F9000022807D99DF805309806DDD59DF8043014
:105FA000D906D9D5FB6A93F89C30002BE5D118E0CF
:105FB000DA0601D41B0718D5284603B0F0BD002827
:105FC000FAD094F82123B4F99036002ACFD013F0F8
:105FD000010FF1D1154B1F68FB6A93F89C30002B21
:105FE000C8D19DF804309C07E2D405F077FC05F099
:105FF00073FB0028B0D10AF0A5FDFFF7EBFA0228E9
:10600000AAD90AF09FFD90F8C432B02202FB030027
:1060100090ED2F7AF0EE007AB4EEE77AF1EE10FA16
:106020009AD59DF80530DB09C6D195E7405D002083
:106030002DE9F04790F8783292B00446002B00F03A
:106040009480204618F078FC2046FFF74BFF032889
:106050007BD104F54E7800274146204600970197F2
:10606000029718F071FA6946204618F063FA009B0F
:10607000C4F81032019BC4F81432029BC4F81832E1
:10608000204601F09FF9204601F084F911F0E6F96D
:106090000546204618F0FEF80028A8BFC6B203AA9D
:1060A0004FF0FF312046BCBF95F80A9395F80B637B
:1060B0000397A8BFB1460497059718F035F903A8D0
:1060C00013F0E0FE4FF00C0A0AFB095084EDD70AEA
:1060D000C4EDD80A84EDD91A04F5577100F5117092
:1060E00013F0E0FE04F55D770AFB065584EDCB0A5C
:1060F000C4EDCC0A84EDCD1A3A464FF0FF3120466C
:1061000005F5C47518F024F995E8070006AE86E891
:1061100007003946304613F02BFF04F53172414633
:1061200009A812F0E7F8314609A812F065F809A9A4
:10613000204684EDDA0AC4EDDB0A84EDDC1A18F09F
:1061400097FA09A92046FFF7B7FC94F89236002B7E
:106150003AD109A804F0E0FA09A9204618F098F904
:1061600090B3012384F892362EE0D0F87C321BB92C
:1061700052F0C6FEC4F87C02154B1B68D86A03684F
:106180005B68984788B152F0BBFED4F87C32C01AE5
:10619000B4F87A32984204D9204618F06FFE84F899
:1061A000780294F878327BB14BE752F0A9FED4F82C
:1061B0007C32C01A41F287339842E4D832F038FC7E
:1061C00032F01CFC0028DED112B0BDE8F08700BF21
:1061D000405D002090F8243323B1032B4FF00000E2
:1061E00007D0704790F93E22032A04D10A7001209B
:1061F00070470870FBE718467047000073B50D46FE
:106200000DF107010446FFF7E5FF064628B19DF8AA
:1062100007302BB1032B09D00026304602B070BDE9
:1062200004F27C630FCB85E80F00F6E72946204691
:1062300018F022F994F87862EFE7000037B50D46C0
:106240000DF107010446FFF7C5FF28B19DF80720AF
:1062500029462046FFF7E6FC03B030BD37B50D46B2
:106260000DF107010446FFF7B5FF28B19DF807308F
:1062700023B1032B11D0002003B030BD04F2F4533E
:106280001B682B6004F5BF631B686B6004F2FC5352
:106290001B68AB6094F8F005EEE72046294618F03D
:1062A00049F994F87802E7E710B50446FFF70CFEC9
:1062B00018B1032807D0002010BD04F25440BDE8F7
:1062C000104001F04DB994F87832002BF3D02046FD
:1062D00017F054FF0028EED094F8203203F0FD03AD
:1062E000012BE9D194F82403C31E58425841E3E737
:1062F00010B50446FFF7E8FD80B1032810D194F8EB
:10630000780250B152F0FCFDD4F87C32C01A44F649
:106310002063984294BF0020012010BD0120FCE7BB
:106320000020FAE708B50246FFF7CEFD032804D1A6
:10633000104618F09DF9012008BD0020FCE7000080
:1063400013B50C4601A9FFF7EDFF20B1019B1C42DC
:1063500014BF0120002002B010BD000030B585B090
:106360000446019102F0FEFD0199054610B9002096
:1063700005B030BD019102F0C7FD01990028F6D0AB
:10638000284602F0C5FD0028F1D0B4F89036590730
:10639000EED494F82133002BEAD00B4A1268D26A6B
:1063A00092F89C506DB103A92046FFF7BBFF30B1B6
:1063B0009DF80E309A07DBD5C3F38000D8E7284656
:1063C000D6E71846D4E700BF405D002010B504466C
:1063D000FFF77AFD032804D12046BDE8104018F0ED
:1063E00021B8002010BD00002DE9F04190F82433C1
:1063F0008CB00027032B06460C46154600970197E4
:10640000029719D117F046FF6A4680464FF0FF31D8
:10641000304617F09DFFB8F1FF3FA7606760276027
:106420000DD111F01BF82B4690F80B13224610F0FB
:10643000A3F80CB0BDE8F0814FF0FF38EBE711F0A6
:106440000DF82B4622465FFA88F110F095F895ED8D
:10645000000A684613F052FD03A920468DED051A87
:106460008DED030ACDED040A13F082FD06F53172BD
:1064700006F54E7103A811F03DFF214603A811F067
:10648000BBFE84ED021A84ED000AC4ED010A95ED0D
:10649000007ADFED037AA7EE271A84ED021AC8E727
:1064A0000AE81C411FB5DFED0B7A20EE270A0C46E7
:1064B0001946094BCDE90042BDEEC00A18688DEDC2
:1064C000020A064B9DF81820C06A0EF0EBF904B0E2
:1064D00010BD00BFE02E6542405D0020A82B0908DA
:1064E0002DE9F0472DED028B92B0002504460F46B2
:1064F0004FF07E5A00F54E7106A89046CDF818A0D0
:1065000009950895079512F00DFF05F0E7F905F0DC
:10651000E3F881462046FFF7D7FC032803D094F820
:106520002433032B4FD19FED558ADFED558A00268A
:106530002379F2B2934247D90AAA71B22046CDF824
:1065400028A00D950C950B9518F008F80AA906A837
:1065500013F0B8FAB4EEC80AF1EE10FA0DDD494AAC
:10656000CDF800803B4648492046FFF79BFF0020BE
:1065700012B0BDEC028BBDE8F0870AA906A803950E
:106580000495059513F088FA03A90EA88DED0E0A5F
:10659000CDED0F0A8DED101ACDED111A13F00AF89A
:1065A000B9F1000F0DD09DED050AB0EEC00AB4EEB2
:1065B000E80AF1EE10FA04DD344ACDF800803B46DB
:1065C000D1E70136B4E7002394F8806216F00100A9
:1065D00001D0012BCCD104F5C0610AA8CDF828A0C8
:1065E0000D950C950B9512F09DFE0AA906A813F0C7
:1065F00069FADFED227AB4EEE70AF1EE10FA05DD72
:10660000204ACDF800803B462149ADE72046FFF700
:106610005BFC03282DD1204617F0F2FF94F880325E
:10662000DB0728D438BB0AA906A80395049505956D
:1066300013F032FA03A90EA88DED0E0ACDED0F0A64
:106640008DED101ACDED111A12F0B4FFB9F1000F53
:1066500011D09DED050ADFED0A7AB0EEC00AB4EE66
:10666000E70AF1EE10FA06DD084ACDF800803B4655
:10667000CAE70020D2E701207AE700BFC2B8323E65
:10668000C2B8B23ED42B0908DF2B09086FE6080810
:10669000E42B09082DE9F743154604468846019383
:1066A000FFF702FE019A074638B92848284B0068D0
:1066B0002946C06A0EF0F6F8019A01922946204652
:1066C000FFF70EFF064668B32046FFF7FDFB94F97F
:1066D0003E12019A43B2994207D01E4B1B480068F4
:1066E0002946C06A0EF0DEF81CE094F82433834299
:1066F00007D0019205F0F2F804F0EEFF019A0028AD
:10670000EBD12046FFF7E0FB18B103280FD0124B66
:10671000E4E7134641462A4604F2544000F034FFB1
:1067200000B107B90026304603B0BDE8F08394F805
:106730007892B9F1000F01D1084BCFE713464146DB
:106740002A46204617F02AFDEAE700BF405D0020F8
:10675000E82B0908F42B0908242C0908132C090834
:1067600090F82433032B01D117F098BF0020704715
:1067700013B540F6783200F50971044601A80DF012
:1067800097FE204617F012FE01A80DF0B3FE02B0EE
:1067900010BD000008B50246FFF796FB10B10328B4
:1067A00006D008BDBDE8084002F2544000F0ACBE7F
:1067B000BDE80840104617F067BF00000B4610B454
:1067C00011462BB1032B09D000205DF8044B704714
:1067D0005DF8044B00F2544000F0A2BE5DF8044B9B
:1067E00017F056BE13B50446FFF76EFB0A46014686
:1067F00020460192FFF7E2FF70B9084B019A1B682F
:10680000DB6A93F89C0038B194F82413204602B058
:10681000BDE81040FFF7D2BF02B010BD405D0020C0
:1068200070B590F89432DB0786B004460D460CD460
:1068300003F03EF9437C242202FB0300D0ED0B7AE7
:10684000F1EE677AC5ED007A3BE002A803F064FF41
:1068500001A92046FFF720FBE8B90AF073F994F983
:106860005032022B0646E3D1FEF7B4FE0228DFD9F0
:1068700096F8C4029FED147AB02303FB0066D4F8A7
:106880008832D6F8B0209B1A07EE903AF8EEE77AF5
:1068900067EE877AD6E702A92046FFF7A3FF002814
:1068A000DBD0D4F88822039BDFED076A9DED017AE7
:1068B0009B1A07EE903AF8EEE77AA7EEE67A85EDB6
:1068C000007A06B070BD00BF0AD7233CF0B50C4675
:1068D00087B000F50971064640F6DD3201A80DF0DB
:1068E000E7FDA36853B9E36843B9636833B9002788
:1068F00001A80DF0FFFD384607B0F0BD204603F0BB
:10690000F5FF0028F3D094E80F0002AD85E80F00F2
:106910000021284603F0ACFF07460028E7D096F890
:106920009432DB0704D432F083F8192131F0BCFF34
:1069300095E80F0006F5217C8CE80F0096F894325C
:1069400043F0010386F89432304600F073FD3BF0CB
:1069500085FC46213CF07CF83BF080FC45213CF076
:1069600077F8084BA2681B68DB6A1A61E2685A6113
:1069700062689A6116F028FA0028B9D014F04AF932
:10698000B6E700BF405D002038B5144B1B68DD6AD8
:106990002B6804465B6828469847F0B12B690BB911
:1069A0006A69D2B1C4F88C326B69C4F89032A969B3
:1069B000002204F5217003F0B3FE94F8943223F022
:1069C000030343F0030384F894323BF047FCBDE833
:1069D0003840034A062136F00FBB38BD405D002029
:1069E000382C090813B504460193FFF76DFA032804
:1069F000019B05D1204602B0BDE8104017F0D8BD7C
:106A0000002002B010BD000010B588B00446059308
:106A1000FFF75AFA0328059B4FF000000AD10690B1
:106A2000079006A802900B9801900A9800902046C3
:106A300017F0CCFD08B010BD38B5044602F092FA4C
:106A40000546D0B194F82433032B03D095F8464182
:106A5000204638BD204617F0D9FCFF280446F5D063
:106A60000146284602F054FA0028EFD02146284675
:106A700002F04AFA0028E9D0EAE70446E8E7000015
:106A800008B590F82433032B05D010F0E7FC90F9FB
:106A90000A03C0B208BD17F0FDFB431CF9D1F4E7AF
:106AA00008B590F8243383B1032B03D1BDE8084027
:106AB00017F0E8BB30F08CFA40F64C524FF48011DE
:106AC00030F03EFA4FF0FF3008BD1846FCE70000FA
:106AD00090F82433032B01D118F0A4B870470000BC
:106AE00090F82433032B01D117F0CCBA7047000083
:106AF00017F02CBB10B504461AF01CFB2046FEF71D
:106B0000E5FB2046BDE81040FEF7FCBC90F82423CE
:106B10001AB1032A07D00120704790F950020038BB
:106B200018BF0120704717F077BD000030B590F80E
:106B300040348BB00446002B64D1B0F89036DB06AD
:106B400060D590ED957ADFED307AB0EEC77AB4EE8D
:106B5000E77AF1EE10FA11D590ED967AB0EEC77A99
:106B6000B4EEE77AF1EE10FA08D590ED977AB0EE30
:106B7000C77AB4EEE77AF1EE10FA43D42046FFF775
:106B8000C5FF00283ED1D4ED976ADFED207A9FED56
:106B9000206A94ED967A009066EEA76AD4ED957A15
:106BA00027EE067A67EE867AFDEEE66ABDEEC77AD4
:106BB000FDEEE77A16EE903A17EE901A17EE102ACD
:106BC00006A803F0C7FD06A92046FFF779F8C8B16B
:106BD0003BF044FB0546D4F85C02F9F78DFCCDE9A7
:106BE0000401D4F85802F9F787FCCDE90201D4F882
:106BF0005402F9F781FC074ACDE900010621284635
:106C000036F0FAF90BB030BD000000340000C84285
:106C10008096184B502C090890F824330BB1032BA5
:106C200001D118F06BB800207047000030B500F5B6
:106C30007B7304460D460FCB85E80F0094F8FC03E8
:106C400030BD0000D0F898330B6090F89403704783
:106C5000D0F8A0330B6090F89D03704710B500F595
:106C6000697203460C4607CA84E8070093F8B0032C
:106C700010BD000030B500F56D7304460D460FCB16
:106C800085E80F0094F8C40330BD000030B500F56E
:106C9000866304460D460FCB85E80F0094F8400448
:106CA00030BD000010B500F2444203460C4607CA4E
:106CB00084E8070093F8500410BD00002DE9F0436C
:106CC0002DED028B8BB005460E461746FFF7B4FE3E
:106CD000014680462846FFF741FB0446002848D07D
:106CE00002F040F9414602F015F986ED000A95F9E7
:106CF0003C32002B3ADD09F025FFFEF76BFC012842
:106D000034D909F01FFF90F8C432D5EDE47ADFEDF5
:106D10005D8A96ED000AB02202FB030095F93C3231
:106D2000D0ED2F0A07EE103AF4EEE87AB8EEC77A03
:106D3000F1EE10FAB7EE008AB8BFF0EE487A37EEFF
:106D4000201A20EE270A70EEC70A40F20E4011F01A
:106D500047F8D5EDE47AF4EEE87AF1EE10FAB8BF30
:106D6000F0EE487A80EE277A86ED007A01233B70B8
:106D700003E095F8203333B9387020460BB0BDECF2
:106D8000028BBDE8F08395F824334FF00009CDF86D
:106D90000490CDF80890CDF80C9043B1032B10D09F
:106DA000CDF81090CDF81490CDF818907CB902234E
:106DB0003B703246414605F2544001F027FB044641
:106DC000DBE701A9284617F015FB0446E8E795F82C
:106DD0002433002BEBD004A92846FFF763FF0446B9
:106DE0000028E4D001A904A813F072F807A8CDED9B
:106DF000080A8DED091A8DED070A13F07DFC04A831
:106E0000B0EE408A13F078FC95F93C32002B30DD6F
:106E100007EE903AF8EEE77A40F2544070EE670AD7
:106E200037EE801AF5EEC00AF1EE10FA48BFDFED3A
:106E3000160AF4EE410AF1EE10FAB0EE480AC8BFA5
:106E4000B0EE601A10F0CCFFB0EE408AD5EDE47AD7
:106E50009FED0C7AF4EEC77AF1EE10FAB7EE007AF5
:106E6000B8BFF0EE477A88EE277A032386ED007AE2
:106E70007DE7B5EEC08AF1EE10FA48BF9FED028AB9
:106E8000E4E700BF000000340000000038B504460D
:106E9000FFF7F6FD94F826338342054604D010F040
:106EA000DDFA29460FF0C8F92046FFF7E9FD84F81E
:106EB000265384F825032046FFF7E2FD84F82703D4
:106EC0002046FFF7EDFD04F5607184F828032046A5
:106ED000FEF746FE84F88C0300F0CCFA04F56772E6
:106EE00084EDE40A04F566712046FFF7E7FE04F539
:106EF000687184F894032046FEF74EFE04F569712C
:106F000084F89D032046FEF77BFE04F56D7184F83E
:106F1000B0032046FEF7B0FE04F5727184F8C40396
:106F20002046FFF79BF904F5767184F8D4032046D8
:106F3000FFF784F904F57B7184F8E8032046FEF737
:106F4000E7FD04F5806184F8FC032046FFF756F95D
:106F500084F810042046FEF793FE04F2144004F572
:106F6000836380ED000AC3ED000A12F0C7FE04F24D
:106F70001C4304F58461204683ED000A04F22C4290
:106F8000FFF732FA04F586612046FFF72BFC80B14B
:106F900094F840349BB9012384F84034204600F033
:106FA00049FA3BF05BF945213BF052FD2046FEF7E4
:106FB000A3FE94F8403413B92046FFF7B7FD04F25E
:106FC00044412046FEF7E0FE84F8500438BD00003E
:106FD00037B50D46044600F0E1F81DB910F03EFA51
:106FE0000FF0FAF94FF4EA7204F5097101A80DF0F7
:106FF0005FFA94F881322BB92046FFF7C5FC0123D4
:1070000084F88132224B1D68A86A03689B699847FF
:107010002046FEF7C1FC2046FEF73AFD204600F070
:107020003BFA2046FFF704F8286B30B10368D4ED33
:10703000D80ADB6894EDD70A9847D4F81C0208B147
:1070400052F0B6FE204600F065F82046FEF74AFFF3
:1070500094F8A83284F8240383420ED084F8A8025E
:1070600098B10C4D0C4B032808BF1D463BF0F6F8B9
:107070000A4A2B46062135F0BFFF2046FFF706FFE0
:1070800001A80DF037FA03B030BD054DEEE700BFA3
:10709000405D0020E6FB0808DF2B09087C2C09086E
:1070A000E42B0908D0EDE47A9FED057AF4EEC77A77
:1070B000F1EE10FAB7EE000AA8BFB0EE670A70470B
:1070C00000000034014B1868704700BF605D00206D
:1070D00070470000704700007047000000207047B4
:1070E000002070470120704703681B6E184700009E
:1070F0000020704700207047002070470020704734
:107100007047000000207047002070470020704743
:10711000704700007047000008B510F09FF990F824
:107120000A0308BD30B52DED028B9FED1A1ADFED75
:107130001A0A91ED000A87B005462D200C468DED08
:10714000011ACDED000A10F04BFE9DED011ADDEDA8
:10715000000AF0EE408A2E2094ED010A10F040FE65
:107160009DED011ADDED000AB0EE408A2F2094ED6E
:10717000020A10F035FE03A905F52B70CDED038A48
:107180008DED048A8DED050A2EF0FCF807B0BDECFC
:10719000028B30BDC2B8323EC2B832BE10B5044612
:1071A00051F0AEFED4F80C331BB1C21AB2F57A7F9F
:1071B00012D30A4A1268D26A92F89C2002B15BB9D3
:1071C000C4F80C0394F83D4210F048F980F80543E8
:1071D00004F084FB80F8254010BD00BF405D002016
:1071E0002DE9F0432DED028B91ED007AD1ED037A7C
:1071F00087B08DED047AB0EEC77AB5EEC07AF1EEC5
:1072000010FADDE91087DDF84C90CDED057A0C46DB
:1072100015461E4606DCF0EEE77AF5EEC07AF1EE92
:1072200010FA02DD04A812F0DDFD6B20B7EE001AA3
:10723000FFEE000A9DED050A10F0D2FD6C2089EDED
:10724000000AB7EE001AFFEE000A9DED040A10F0E6
:10725000C7FD04A888ED000A12F02AFDB7EE008AE7
:10726000002852D00023C9F8003088ED008AD4ED00
:10727000067A67EEA77AF4EEC87AF1EE10FA4ADBE6
:107280000023336085ED008ADFED3F0A96ED000AAA
:107290007C20B7EE001A10F0A3FD86ED000A95EDF4
:1072A000000A7D20B7EE001AFFEE000A10F098FDEC
:1072B00085ED000AD4ED067A129BDFED346AF1EE1B
:1072C000677AC3ED007A96ED007AF0EEC77AF4EEB5
:1072D000E67AF1EE10FA2BD503AB02AA01A92046FB
:1072E00011F0B6F99DED018AB0EE480A70F0BEFBD0
:1072F00085ED000AB0EE480A70F00EFD87ED000A39
:1073000007B0BDEC028BBDE8F08304A812F0BCFC12
:107310000028A7D1ABE738EE670A10F0BFFC86ED76
:10732000000A94ED087AC7EE007AC5ED007AABE763
:1073300094ED076AC6EE077AC7ED007A96ED007AFB
:10734000B0EEC77AB4EEE67AF1EE10FAC4D495ED59
:10735000007ADFED0F6AB0EEC76AB4EE666AF1EE4E
:1073600010FAB9DCB4EE477AF1EE10FAB4D6B0EE0A
:10737000E77AB4EE667AF1EE10FAADDCF4EE677AF5
:10738000F1EE10FABCD7A7E70000000000000034BF
:10739000FFFF7F7F1FB500F51D73039300F51C737E
:1073A000029300F51B73019300F51A73009300F527
:1073B000187200F5197300F54E71FFF711FF05B053
:1073C0005DF804FB9FED196AD0ED846ADFED187A51
:1073D00090ED860A66EE866A20EE060A26EEA77A09
:1073E00010B5BDEEC77AC0ED7E6A80ED817A90ED72
:1073F000857A27EE067A044667EE275A60EE277AEA
:10740000FDEEE55AFDEEE77AC0ED825A17EE903AAE
:10741000002BBCBF03F50C43A033C0F80C3280ED49
:107420007F7A10F073FC84ED800A10BDE02E654277
:107430000000C8421FB50E4B1B680446B3B1684636
:1074400003F06AF969462046FFF720FC20B16A463E
:1074500000212046FEF720F894F89432DB0705D58A
:1074600004F5217201212046FEF716F804B010BD84
:107470000860002008B502F01BFBBDE8084001F0E1
:10748000E3BD000010B580F81013044651F038FD3C
:10749000C4F8140310BD000010B590F81033044672
:1074A00053B151F02DFDD4F81433C01AB0F57A7FE2
:1074B00084BF002384F8103394F8183353B151F08B
:1074C0001FFDD4F81C33C01AB0F57A7F84BF0023A7
:1074D00084F8183310BD000000F5AA700B4607C8E9
:1074E00083E80700012070470023C0F89C30C0F8F3
:1074F0009830C0F89430C0F8A830C0F8A430C0F874
:10750000A030C0F8AC30704770470000024B0B60F1
:107510004FF07C53136070470000484270470000F2
:1075200010B500F5B4700C460FC884E80F00204673
:1075300003F0E6F830B1FFF7C5FD00F521700FC884
:1075400084E80F00204603F0DBF880F00100C0B2B1
:1075500010BD000010B5044603F00AFC204610BD23
:1075600010B5D0F8603104465BB151F0C9FCD4F8D5
:107570006031C01A41F28833984294BF0020012044
:1075800010BD0120FCE7000013B5009303680192D1
:10759000DB6D9847DDE90021044628B90448054B16
:1075A0000068C06A0DF07EF9204602B010BD00BF31
:1075B000405D0020E82B090813B50446019101F055
:1075C000D1FC2368019ADB6B014608B190F84611A3
:1075D000204602B0BDE810401847000090ED007A48
:1075E000DFED0F7AB0EEC77AB4EEE77AF1EE10FA7B
:1075F00014D590ED017AB0EEC77AB4EEE77AF1EEE9
:1076000010FA0BD590ED027AB0EEC77AB4EEE77AB5
:10761000F1EE10FA4CBF01200020704700207047A7
:107620000000003410B501F09DFC044658B190F8FC
:10763000461101F069FC30B194F846112046BDE8CE
:10764000104001F065BC002010BD00002DE9F043A2
:107650002DED028B8FB0036800259B6B039504957D
:1076600005950695029502A904469847064638B145
:10767000FFF700FFDDED027A27EE800A8DED020AAA
:1076800009F060FAFDF7A6FF0746002E50D0DDEDA9
:10769000027AD4ED646A94ED657A23680B9527EE3F
:1076A000877A67EEA67A8DED097ACDED0A7A0C9588
:1076B0000D955B6B0BA9204609AD98470BA9284691
:1076C00012F060FA012F8DED030ACDED040A40F2AD
:1076D000B38009F037FA90F8C432DFED5B7AB02559
:1076E00005FB030090ED308A28EE278AB0EE480AA9
:1076F00070F0BCF9F0EE408AB0EE480A70F00CFB76
:10770000CDED0B8A8DED0C0A09F01CFA90F8C4320D
:1077100005FB030090ED2F0A0BA812F053FA09ADF8
:107720008DED050ACDED060A05A896BB03C885E0D8
:107730000128CED89DED020AB5EEC00AF1EE10FA8E
:107740007FDD07AED4F89421D4F89031079230460B
:10775000089312F061FA23680B950C950D955B6BFD
:107760000BA920469847DDED077A9DED0B7A77EE61
:10777000877A9DED0C7ACDED077ADDED087A77EE0C
:10778000877A09ABCDED087A96E8030083E8030019
:1077900049E0236993ED000AB7EE008A38EE408A8B
:1077A00012F010FA04F5BC798DED090A4846B0EEE6
:1077B000480ACDED0A0A12F005FA0BA92846CDEDCC
:1077C0000C0A8DED0B0A12F0DDF904F5C47603AF57
:1077D000C4ED5F0A314684ED5E0A384612F0E2F9E4
:1077E00004F5C0788DED090A4046B0EE480ACDEDAB
:1077F0000A0A12F0E7F90BA928468DED0B0ACDED28
:107800000C0A12F0BFF997E8030084ED600AC4ED9A
:10781000610A86E803004946404612F0B3F98DED4F
:10782000090ACDED0A0A9DED090ADDED0A0A0FB03D
:10783000BDEC028BBDE8F083DDE9030185E80300C0
:10784000F1E709950A95EEE735FA8E3C10B590F808
:107850004213044603F068FC7C23C0B203FB0044DF
:10786000D4F8A00010BD0000044B026F1B68DB6A57
:107870005A60426F9A60826FDA607047405D002004
:10788000F0B58FB004460FF0E9FD00230293039397
:10789000049390F80A1301AB02AA05460EF012FEFB
:1078A00004F19407D8B39DED010AB5EEC00AF1EEDC
:1078B00010FA34DD02A812F031FB04F1B00684EDB9
:1078C0002C0AC4ED2D0A84ED2E1A3946304612F0EA
:1078D00035FB04F17C01304612F0E4FA04F1880132
:1078E00005A88DED050ACDED060A8DED071A12F0FB
:1078F000D9FA08A88DED080A9DED010ACDED090A17
:107900008DED0A1A12F0FAFA0BA904F128008DED98
:107910000B0ACDED0C0A8DED0D1A10F045FF95F810
:107920000A030C2303FB0050394600F5117012F0D6
:10793000B9FA84ED2C0AC4ED2D0A84ED2E1A0FB08D
:10794000F0BD00002DE9F0477E4B00251F682DEDAE
:10795000028BC0F89C50C0F89850C0F89450C0F802
:107960008450C0F88050C567C0F89050C0F88C5063
:10797000C0F88850C0F8B850C0F8B450C0F8B05043
:107980000446F86A03688AB05B680E46984704F1BB
:107990002809002854D051F0B3FA42F20F739842EC
:1079A0004ED8FB6A9FED688A93ED010A84ED1C0AAC
:1079B000D3ED020AC4ED1D0A93ED031A484684ED87
:1079C0001E1A10F0E5FD3AF049FCD4ED1E7A67EE80
:1079D000887A054617EE900AF8F78EFDD4ED1D7AE9
:1079E00067EE887ACDE9040117EE900AF8F784FD76
:1079F000D4ED1C7A67EE887ACDE9020117EE900A81
:107A0000F8F77AFD514ACDE900010621284635F004
:107A1000F3FA94ED1E8AB0EE480A70F027F884ED70
:107A2000650AB0EE480A70F077F984ED640A51F007
:107A300067FAC4F864010AB0BDEC028BBDE8F087B8
:107A4000A6B194ED1C0AB4EE400AF1EE10FA0DD680
:107A5000D4ED1D0AF4EE600AF1EE10FA06D694EDAC
:107A60001E1AB4EE411AF1EE10FA67D70FF0F6FCC9
:107A700090F80B334FF00C0A0AFB030303F5C473B1
:107A8000074693E8070007AE86E807004FF01508A1
:107A9000B2EE028AF2EE068A304612F02DFEB4EE05
:107AA000C80AF1EE10FA11D508F1FF3818F0FF08F6
:107AB00015D1304612F020FEF1EE047AB4EEE70A5A
:107AC000F1EE10FA1CDC2567656731E0304612F0F4
:107AD00013FEB4EEE80AF1EE10FAE5DCE9E7384609
:107AE0000EF0AEFB38460EF077FC97F80B330AFB2E
:107AF000037303F5C47393E8070086E80700CBE738
:107B0000DDED098A9DED088A9DED070A68EEA80A59
:107B1000E8EE080AF1EEE00A70F0CAF9F1EE680A40
:107B200084ED1D0AB1EE480A70F0C2F984ED1C0A1A
:107B30009FED071AD4ED1D0A94ED1C0A484610F07B
:107B400027FD66E7405D0020E02E6542F02D090824
:107B5000000000000021FFF7F5BE000037B5044625
:107B600008461546019112F0C7FDB7EE007AC7EE40
:107B7000007AB4F8D03001980133A4F8D03094EDF5
:107B8000337A37EE277A84ED337AB0EE007AF4EE6A
:107B9000C77AF1EE10FA06D5B6EE007AF4EEC77A9F
:107BA000F1EE10FA0DDC9FED0E7AF4EEC77AF1EEED
:107BB00010FA13D59FED0B7AF4EEC77AF1EE10FAB6
:107BC0000CDDB0EE670A12F099F9012085ED000A8C
:107BD000C5ED010A85ED021A03B030BD0020FBE7B8
:107BE00000247449BD37863570B52DED028B00F148
:107BF000280600F134058AB029460446304612F0C2
:107C0000F9F9B6EE008A20EE088A2846B0EE480A56
:107C100012F074F907A93046CDED080A8DED091A66
:107C20008DED070A12F054F930468DED010AB0EEE1
:107C3000480ACDED020A8DED031A12F05FF907A98B
:107C400028468DED070ACDED080A8DED091A12F0D0
:107C50003FF904A901A88DED040ACDED050A8DEDCB
:107C6000061A12F0DBF9324601A920468DED070A0B
:107C7000CDED080A8DED091AFFF770FF58B951F0E4
:107C80003FF90121C4F860012046FFF75BFE0AB00E
:107C9000BDEC028B70BD2A4604A92046FFF75EFFAB
:107CA0000028ECD004F1400207A92046FFF756FF58
:107CB0000028E4D0EBE7000030B52DED028B0D4637
:107CC00083B091F842130446284603F02DFAC1B25E
:107CD0007C2000FB0151903104F1280010F0E8FAFB
:107CE00068468DED000ACDED010A12F007F8DFEDD0
:107CF0001C7AB4EEE70AF1EE10FA05D59FED190AE9
:107D000003B0BDEC028B30BD684612F06BF86846DC
:107D100011F0CEFF0028F1D1284694ED428A03F0FD
:107D20006BFBF0EE400AB0EE480A0FF083FF80B91B
:107D3000284603F061FB84ED420AB0EE408A6FF002
:107D400095FE84ED430AB0EE480A6FF0E5FF84ED3E
:107D5000440A04F58671684611F088FFD0E700BF39
:107D600000000034000000009FED0C7AB4EEC70A5A
:107D7000F1EE10FA0BD4DFED0A7AB4EEE70AF1EE79
:107D800010FA07DCC0EE077AB0EE670A7047F7EE2C
:107D9000007AF9E7F2EE047AF6E700BFF3665F3F98
:107DA00058A00B4108B51C3011F0A8FFF1EE007A85
:107DB000B4EEE70AF1EE10FA9DBFF1EE027A37EE6B
:107DC000C00ADFED047A9FED040A98BF20EE270A6F
:107DD00008BD00BFCDCC4C3ECDCCCC3D08B58369B1
:107DE00093F9000038B108F0ADFEFDF7F3FB012870
:107DF00094BF0020012008BDF8B52DED028B05468B
:107E000003F06CFD03F068FC0446B8B3FFF75AF9C1
:107E100090F8213393B32846FFF7E0FF064668B396
:107E200008F090FE90F8C432B02707FB030090EDF5
:107E30002F7AF0EE087AB4EEE77AF1EE10FA1DD45C
:107E400095ED1E8A08F07EFE90F8C432DFED1E7AB2
:107E500007FB030090ED300A98EE270A0FF06CFF45
:107E6000DFED1A7AB0EEC00AB4EEE70AF1EE10FACE
:107E700008DC51F045F83446C5F85001BDEC028BE2
:107E80002046F8BD05F5AA7012F036FCB0EE408A27
:107E900008F058FE90F8C4329FED0D7A07FB0303FB
:107EA000D3ED2F7A67EE877AB4EEE78AF1EE10FA17
:107EB000DFD551F025F8D5F85041001BB0F5FA6F29
:107EC0008CBF00240124D9E7E02E65420000344233
:107ED000CDCC4C3F10B50A4B1B68DB6A93F89C3045
:107EE00004465BB951F00CF8D4F86431C01A44F67A
:107EF0001F6398428CBF0020012010BD0020FCE7CA
:107F0000405D0020F8B52DED068B044608F01AFE02
:107F1000054603F0E3FC064604F036F9002840F07D
:107F2000AA802046FFF768FF002800F0A7803046AF
:107F3000FFF78CFCD4F8DC30984200F01881304612
:107F4000FFF784FCD4F8DC30DFED8E7AC31A08EE3C
:107F5000903AF8EE688A304668EEA78AFFF776FC1A
:107F600094F8BC30C4F8DC00F3B9304603F0C6FB2B
:107F7000D0B104F1280796F842233946304603F081
:107F80003FFAD4ED1D0AB0EE401A384694ED1C0AB3
:107F900010F0FEFA0023C4F89030C4F88C30C4F816
:107FA0008830012384F8BC3020463146FFF784FE38
:107FB00095F8C40205EB0015B0EE408A2B6FC4F8AB
:107FC000E03004F1B000D4ED129A12F095FB636832
:107FD000DFED6D7A93ED007AB4EEE77AF1EE10FA08
:107FE00068EE299AB0EE40AA01D5C3ED007A20468A
:107FF000B0EE4A0AFFF7B8FE636820EE299A93EDC7
:10800000000A29EE009AFFF7CDFE29EE009A2046DD
:1080100084ED249AFFF75EFF38B1D4ED247AB2EEF6
:10802000007A67EE877AC4ED247AF0EE007AF4EEF7
:10803000E78AF1EE10FA10D5DFED547AB4EEE7AA34
:10804000F1EE10FA09D5DFED527A69EEA79AD4ED78
:108050002A7AE9EEA87AC4ED2A7A9FED4E0A94EDC9
:10806000367ADFED4D7AB0EEC88A28EE008AA7EEA8
:10807000278A84ED368ABDEC068BF8BDFFF722F81F
:1080800090F82133002B72D02046FFF7A7FE00287E
:108090006DD095F8C42205EB0213196FD4F8E030C7
:1080A0008B4264D0B02606FB025292ED2F7AF0EE9E
:1080B000087AB4EEE77AF1EE10FA58DBCB1AC4F87E
:1080C000E01008EE903A95F8C4329FED341A94ED22
:1080D0001E0ADFED337A06FB0353D3ED309A69EEC7
:1080E000819AF8EE688A39EEC00A68EEA78A0FF026
:1080F00063FEB0EE409A6FF00FFE94F8BC30B0EE25
:10810000408AF3B1F3EE047AF4EEE78AF1EE10FA66
:1081100017DC95F8C40206FB005595ED2F7AF2EEB8
:10812000027AB4EEE77AF1EE10FAFFF64AAFDFED2D
:108130001D7AB0EEC99AB4EEE79AF1EE10FAFFF6A6
:1081400040AF9FED198AD4ED1D0A94ED1C0AB0EEE4
:10815000691A04F1280010F01BFA012384ED248A27
:1081600084ED238A84ED228A84F8BC3029E7BDECB3
:10817000068B04F188009FED0D0ABDE8F84011F070
:1081800011BF00BFBD378635CDCC4C3DC2B8B23E25
:108190000AD7233CCDCC4C3ECDCC4C3F35FA8E3C5F
:1081A0006F12833A1904863F00000000EC51783FBB
:1081B00030B50C2303FB010101F1C003144693E821
:1081C00007008BB004AD85E8070094E8070083E85A
:1081D00007002846FFF702FA07AB58B194E80700FA
:1081E00083E807009DED070ADDED080A9DED091AF9
:1081F0000BB030BD95E80700F2E70000F0B52DEDBB
:10820000028BD0F818318B60D0F81C31CB6085B070
:1082100004460D4601F04CFC064608F093FCA369A9
:1082200093F90030022B07464BD1FDF7D3F9022812
:1082300047D997F8C432B02202FB0373D3F8B010C9
:108240000022284602F06CFAD4ED4A0A94ED490A5D
:10825000284602F079FD94F82C3163B350F050FEBB
:108260009FED228A97F8C4128DED018A01AA064675
:10827000384607F0E5FCD4F820019FED1D0A361AB8
:1082800007EE906AF8EE677A40F23C4027EE800AEB
:10829000B6EE001AF0EE480A0FF0A2FDDDED017A0D
:1082A00030EE270A04F1F0008DED010A11F08AFC8E
:1082B000284602F049FD94F82C0105B0BDEC028B74
:1082C000F0BD707C242303FB006696ED0B8AFEF75D
:1082D000F9FED0EDA27A9FED077AF8EEE77AE8EEA4
:1082E000077AFDEEE77A17EE901AA9E70000000082
:1082F0006F12833A0000C84230B589B00446684620
:108300000D4602F009FA69462046FFF709F918B947
:108310000024204609B030BD04A802F0FDF9204633
:1083200004A9FFF76BFF04460028F1D004A96846B2
:1083300002F012FC85ED000AC5ED010A85ED021A76
:10834000E7E700001FB500230C4601A90193029343
:108350000393FFF7D1FF08B1039B236004B010BD66
:1083600030B585B001AD00230C4629460193029338
:108370000393FFF7C1FF034618B195E8030084E8B3
:108380000300184605B030BDF8B52DED028B06464A
:108390000F46154600F0E6FD0446A0B1394600F050
:1083A000B3FD80B12046394600F0B2FD044650B11D
:1083B00000F0D8FD394600F0ADFD85ED000ABDECBA
:1083C000028B2046F8BDFEF77DFE90F82033B7EE15
:1083D000008A7BB13046FFF701FD044650B1D6ED6F
:1083E000538AFFF747F8C8EE007A67EEA87AC5ED22
:1083F000007AE4E7D6ED538AFFF73CF8C8EE007A3E
:10840000002467EEA87AC5ED007AD8E770B52DEDA7
:10841000048B1646FFF7B8FF054670B3FEF752FE11
:1084200090F93C424CB308F08DFBFDF7D3F80128DE
:1084300023D9E4B207EE904AB8EE678A08F082FBCF
:1084400090F8C43296ED009AB02202FB0300D0ED02
:108450002F8AFFF70FF838EE281A78EEC80A40F294
:10846000654029EE000A0FF0BBFCB0EE408AFFF732
:1084700001F8C8EE007AC6ED007ABDEC048B284600
:1084800070BD000038B50D4608F05CFB0446FDF7F2
:10849000A1F8022881BF94F8C402B02303FB004076
:1084A000D43089BF07C8002085E80700012038BD07
:1084B00030B585B000230D4601A9019302930393C3
:1084C000FFF7E0FF044620B1039B2B60204605B078
:1084D00030BD01F0EDFA417C00F0A4FF0446002815
:1084E000F4D001F0E5FA00F051FEB1EE400A85ED5E
:1084F000000AEBE7F8B5036F4B60436F8B60836F47
:10850000CB6000F14C070C46054601F110060FCF79
:108510000FC60FCF0FC63B68336005F1280104F189
:10852000340010F0FFFE2346012203F8442B05F12E
:10853000B00207CA83E8070005F1940207CA04F1F4
:10854000500383E8070005F11C0207CA04F15C032D
:1085500083E8070004F174012846FFF793FF04F154
:10856000840184F880002846FFF7A2FF04F18C0103
:1085700084F888002846FFF741FE84F89C00F8BD87
:1085800008B503F0ABF9BDE8084003F0A5B800005A
:1085900010B5044611F05EFD50B904F10C0011F065
:1085A00059FD28B904F11800BDE8104011F052BD82
:1085B000012010BD38B500F1280504462846FFF714
:1085C000E7FF28B120460121BDE83840FFF7BAB9DE
:1085D000D4ED107AB7EE007AF4EEC77AF1EE10FA25
:1085E00006D5BFEE007AF4EEC77AF1EE10FA12DC8F
:1085F0002046FFF7F9FA2846FFF7CAFF0028E1D125
:10860000D4ED107AB2EE047AF0EEE77AF4EEC77A9F
:10861000F1EE10FAD6DC38BD10B5044612F06CF855
:108620002046BDE8104011F0D1BC00002DE9F04F0C
:108630002DED048B9FEDCA8A95B00446F0EE408A7A
:108640008DED028A8DED038A8DED048AFFF75AFCC9
:108650000EF004FF0023054695F87921012AA8BFF2
:10866000012293423FD2002128460DF051FD012303
:108670000028F1D008AB0BAA002128468DED0B8A0B
:108680008DED0C8A8DED0D8A0DF076FF9DED080ABB
:10869000B5EEC00AF1EE10FA23DD0BA811F03EFC96
:1086A00011A904F128008DED110ACDED120A8DED0E
:1086B000131A0FF0A1FD0EA88DED0E0AB0EE680A98
:1086C000CDED0F0A8DED101A11F018FC11A904F16F
:1086D000E4008DED110ACDED120A8DED131A11F0A3
:1086E0002DFC0123B8E795F80B130C2303FB015174
:1086F00004F1280B01F5C47158460FF07DFD84ED9F
:10870000070A94ED3F0AC4ED080A70EE288A84ED4A
:10871000091AC4ED3F8A08F015FA0646FEF7D2FCA6
:1087200090F8213301932046FFF758FB80B1304683
:10873000FCF750FF02280BD996F8C4226169B023D8
:1087400003FB026391F9001093F8D200884263DAC8
:1087500094ED3F7ADFED837AB4EEE77AF1EE10FA2A
:1087600061D4D4ED538AFEF75DFF58B100F0FAFBF7
:1087700090F8461100F0CEFBF0EE408AFEF77AFE4C
:1087800060EE288A236C626BA16A1393B0EE680ACC
:1087900011A81292119111F0B1FB04F5AA7102A86F
:1087A0008DED020ACDED030A8DED041A11F0C6FB22
:1087B00050F0A6FB0023074684F814312046FFF74B
:1087C0000DFB002865D096F8C422B02302FB0332CB
:1087D00032445268C4F8182196F8C42202FB0333CD
:1087E00033449B68C4F81C3150F08AFB0123C4F861
:1087F000200184ED498A84ED4A8A84F82C31D4F82A
:108800000031002B58D102AB93E80700C4F8007187
:10881000F03484E8070006E006EB0212176FD4F884
:108820000021BA4204D115B0BDEC048BBDE8F08F35
:10883000D43393E8070094F814310DF1080C8CE858
:1088400007001BB904F1F00383E807000123604629
:1088500084F8143104F5AA7111F03AFB11A904F15E
:108860004C008DED110ACDED120A8DED131A0FF0AB
:10887000F1FCB5EEC00AF1EE10FA8DED110AD8BF89
:108880009FED370ACDED120A8DED131A84ED530AD0
:1088900094E794ED3F7AD4ED497ADDED026AE6EE95
:1088A000877ADDED036AC4ED497AD4ED4A7AE7EEC2
:1088B000267AC4ED4A7AA2E7D4ED3F7A254B8DEDB6
:1088C000058AF5EEC07AF1EE10FA8DED068A07936F
:1088D000A9D9214B9FED217A1B68DB6A67EE877A65
:1088E00093F89CA0B7EE007AC7EE279ABAF1000F72
:1088F0004AD094F8143113B9019B002B42D0E3689D
:1089000004F1F001D3ED008A02A811F0E1FA69EE5A
:10891000A88A8DED110A11A8B0EE680ACDED120AF1
:108920008DED131A11F0EAFA0EA905A88DED0E0AC5
:10893000CDED0F0A8DED101A11F000FB05A8FFF721
:108940006BFE05A811F0A0FBF0B150F0D9FAC4F805
:10895000600168E7000080BF405D00200AE81C411C
:1089600000000000CDCC4C3ECDCC4C3FCDCC4C3D9E
:10897000920A06BF920A063FC2B8B23E728A0E3C05
:108980005B821839DDF804A05FED0B8A0023CDE986
:108990000833CDE90A33CDE90C334FF0FF320092B2
:1089A00004F1E40895F87921012A1046A8BF0120B6
:1089B000834255D20123002AFAD095F82D130029BD
:1089C000F6D0B0EE690A404611F0ECFA0DF12C0930
:1089D000BAF1000F3FD0424600212046FFF7E8FBE6
:1089E0008DED0B0ACDED0C0A8DED0D1A4846FEF704
:1089F000F5FD70BB4846FFF70FFE484611F044FBFB
:108A000038BB05A9484611F009FB05A94846CDED3C
:108A1000090A8DED0A1A8DED080A11F0EBFA08A883
:108A2000B0EE409A11F068FE009B33B9F4EEC08AB4
:108A3000F1EE10FAD8BFB0EE680AB5EEC09AF1EECA
:108A400010FAF7EE008A4FF0000358BFF0EE408AAC
:108A500000930123A6E798E8070089E80700C5E727
:108A6000009B002B7FF471AF002384F80431204673
:108A7000FFF7C2F938B12046FFF7B0F9002840F0FF
:108A800025818DED0A8A95F80A3395F878219A4266
:108A900040F233812B4493F82C33002B00F02D81CE
:108AA00095F80B3395F879219A4240F226812B44B0
:108AB00093F82D33002B00F0208108A958460FF0C1
:108AC000C9FB8DED080ACDED090A8DED0A1A08A83B
:108AD00011F0C0FA002840F0178108A811F0D4FA6C
:108AE000002840F011815FED617A94ED357A68EEEF
:108AF000A78A5FED637AE7EE278A04F1B000C4ED40
:108B0000358A11F0F9FDA3685FED687A93ED007A7C
:108B1000B4EEE77AF1EE10FAF0EE408A00F1F88058
:108B20002046B0EE680AFFF71FF908A811F0E6F931
:108B3000A3688DED110ACDED120A8DED131A93ED98
:108B4000000A11A811F0DAF9204684ED1F0AC4EDDD
:108B5000200A84ED211AFFF7BDF928B1B2EE000A10
:108B600004F17C0011F01EFA019BB3B33046FCF710
:108B700031FD012831D996F8C402B02303FB006609
:108B800096ED2F7AF0EE087AB4EEE77AF1EE10FA6D
:108B900023D595F80B030C2303FB005595ED627A62
:108BA000F1EE0C7AB4EEE77AF1EE10FA15DBD4EDC3
:108BB0001D7A1FED917AF4EEC77AF1EE10FA0CDD12
:108BC0001FED947AF4EEC77AF1EE10FA05D5B6EE01
:108BD000000A04F17C0011F0E5F95FED997AF4EEFA
:108BE000E78AF1EE10FA22D51FED9C0A08A811F0D1
:108BF00085F90EA88DED0E0A94ED3F0ACDED0F0A12
:108C00008DED101A11F07AF911A904F1A0008DED83
:108C1000110ACDED120A8DED131A11F08FF9D4ED72
:108C20002B7A94ED3F7A77EE877AC4ED2B7A94ED28
:108C30002B7AF1EE047AB4EEE77AF1EE10FA3BDB30
:108C40000EF00CFC5FEDB27A94ED2B1A94ED280A2D
:108C500021EE271A40F2C930F1EE410A8DED011ADA
:108C6000CDED000A0FF0BCF89DED011ADDED000A14
:108C700084ED280A40F2CA3094ED290A0FF0B0F8CA
:108C80009DED011ADDED000A84ED290A40F2CB309A
:108C900094ED2A0A0FF0A4F804F1A00184ED2A0A49
:108CA00004F1940011F04AF984ED2A8A84ED298AAE
:108CB00084ED288A84ED2B8A0023C4F8E430C4F8BC
:108CC000E830C4F8EC3084ED3F8A9CE5E368F7EEC9
:108CD000000A93ED000A0EF0ADFF00283FF4D1AE7C
:108CE00094ED1C0AB0EEC00A6FF016F8DDED0A7ABA
:108CF00027EE800A8DED0A0AC5E68DED0A8A8DED14
:108D0000098A8DED088AE2E62046FFF753FC1CE64F
:108D1000C3ED007A04E700BF2DE9F04D2DED0E8B79
:108D2000A0B004460EF09AFBD0EDC67A90ED618AB1
:108D3000F4EE487AF1EE10FA48BFB0EE678ADFED44
:108D4000677AB4EEE78AF1EE10FA0EDD0023C4F87C
:108D5000E430C4F8E830C4F8EC300023C4F8FC3048
:108D600020B0BDEC0E8BBDE8F08D2046FEF788FDEF
:108D70002046FEF739FFB0EE480A2046FFF756FCC2
:108D80002046FFF717FCFEF79DF916AD00F53A7285
:108D900004F1280116A80FF0ADFA0FCD04F14C062E
:108DA0000FC60FCD0FC62B68336004F1740204F1B7
:108DB000780304F1700104F14C000FF049FC94EDCC
:108DC0001E8AB0EE480A6EF051FE84ED650AB0EEE0
:108DD000480A6EF0A1FF204684ED640AFEF744FDC8
:108DE000FEF770F904F5B471FDF750FF50F088F804
:108DF000D4F89831C31A632BB2D9C4F898012FF074
:108E000017FE9FED378A054650F082F8D4ED1C7AA4
:108E100067EE887A074617EE900A0E46F7F76CFB66
:108E2000D4ED1D7A67EE887A41EC1D0B17EE900A9F
:108E3000F7F762FB94ED1E0A20EE080A41EC1C0BCA
:108E40000EF064FFD4F8D40010EE108AF7F754FB4C
:108E50008246D4F8D8008B46F7F74EFB41EC180B4E
:108E6000D4F85401F7F748FB41EC190BD4F858013A
:108E7000F7F742FB41EC1A0BD4F85C01F7F73CFB27
:108E800094ED53EA41EC1B0BFEF7F4FACEEE007AB8
:108E900017EE900AF7F730FBCDE9140140468DED4F
:108EA00012BB8DED10AB8DED0E9B8DED0C8BCDE9D6
:108EB0000AABF7F721FB0B4B01930B4B0093CDE96A
:108EC00008018DED06CB8DED04DBCDE90276074B75
:108ED000074A084928462FF033FB41E7CDCC4C3EEA
:108EE000E02E6542F50609084B0709081C2E090803
:108EF000272E0908E42B090870470000002070475E
:108F00007047000000207047002070470020704725
:108F1000002070479FED010A704700BF000000006D
:108F20009FED010A704700BF00000000002070475D
:108F30007047000010B50446143000F019F804F131
:108F40002C0000F015F804F1700050F0C1FF04F19E
:108F5000F00050F0BDFF4FF0FF33C4F84C31204615
:108F600010BD0000014B1868704700BF645D002011
:108F70007047000008B52DED048BB0EE609AF0EE5E
:108F8000408A00F00FF9B0EE408A89EE280A6EF0B0
:108F9000F9FFDFED0B7A20EE270A6EF08BFFDFED95
:108FA000097A38EE278ADFED087A28EE278AF7EE6D
:108FB000007A37EEC00A28EE000ABDEC048B08BD2B
:108FC00041D3423E33938843A1D81943FFF7D2BF20
:108FD00008B52DED048B9FED179AF0EEE07AF4EED4
:108FE000C97AF1EE10FAF0EE408AB0EE608A04D54C
:108FF000B7EE000ABDEC048B08BD00F0D3F8DFED3E
:109000000E7A9FED0E7ADFED0E6A70EE277A9FEDF5
:109010000D0AE8EEC77A27EE800A88EE007AC6EEDF
:10902000877AF4EEC97AF1EE10FAE1DBB1EEE70AE5
:10903000E0E700BF0000003433938843F4FDD43BE5
:10904000CDCC9C3F48A18F43427CD0ED257A242192
:1090500001FB020292ED0B0AD2ED090A30EE270A5B
:10906000FFF7B6BF38B52DED088BDFED21AA9FEDD8
:1090700021AA9FED21BA0546B0EE409AF0EE609A23
:10908000B0EE408A1524013CA4B25CB3F0EE490A6C
:109090002846B0EE480AFFF76DFFF0EE490A70EE81
:1090A000698A284638EE2A0AFFF764FFB0EEE87AAC
:1090B00070EE697AB4EECA7AF1EE10FA77EEE87AD9
:1090C00010D468EEAA8A40F2631088EEA70AB0EEC8
:1090D0004B1A38EE400AF0EE4A0A0EF081FEB0EE6E
:1090E000408AD0E7B0EE480ABDEC088B38BD00BF1F
:1090F000CDCCCC3D0AD7233C0024744900234360E7
:109100008360C360036143618361C361002380F8AE
:109110002030704790F82020531CDBB2062B80F8DB
:10912000203000EB820288BF002382ED010A88BF55
:1091300080F82030704700004FF0FF3310B54361D6
:109140000E4BC0F8A8300023044680F8C830A83081
:10915000FFF7D4FF0A4BC4F8A83004F586704FF02F
:109160008BF8084B08491C6020462BF029FAD4F8EC
:109170009030C4F89430204610BD00BF403009083C
:1091800050300908685D0020E830090808B5A830AB
:1091900030F07CFCDFED027A20EE270A08BD00BF2C
:1091A00000007A4490ED3C0ADFED057AB0EEC07A1B
:1091B000B4EEE77AF1EE10FA48BF90ED3D0A704741
:1091C0000000003473B5D0F8A43004460E4663B1F5
:1091D0004FF096FED4F8A430C01A42F20F739842B2
:1091E00003D894ED280A02B070BD114B1D687DB103
:1091F00095F846112846FFF78BFE48B195F84611C1
:1092000001AA2846FFF77AFE10B19DED010AEAE7B0
:10921000242101FB064494ED0A0ADFED067AB4EE40
:10922000E70AF1EE10FA58BFB0EE670ADBE700BFBD
:10923000645D002000000C4208B561B10378022B88
:1092400002D906484FF02AFE5A1C027000EB830038
:109250004160012008BD0846FCE700BF082F09084F
:109260002DE9F84305460E469146002400F13C08DE
:109270002B7CA34211DD00234A46314601200AF02F
:1092800093FF242363430746002158F803000AF0A4
:109290009BFF874204D00134EAE70020BDE8F88351
:1092A0000120FBE770B50B46064614469AB11146FD
:1092B0009847054628B9236820465B68BDE870409A
:1092C000184701463046FFF7B7FF20B92B682846FC
:1092D0005B689847EFE770BDF0B50D4685B0114665
:1092E0001A46CDE902130446FFF7BAFF034698B9C0
:1092F0000A480068406804270668CDE90037DDE9C0
:1093000002123668064BB04702462946204605B091
:10931000BDE8F040FFF7C6BF0022F6E7405D002041
:10932000801A06007FB5D0ED247A9FED347AF0EEF6
:10933000E77AF4EEC77A0123F1EE10FA04460376D9
:1093400009D49030002303A9019003932BF0CCFEA5
:1093500001982BF00DFB002277232949E263226656
:10936000C4F884202046FFF7B7FF2378032B28D0CA
:10937000237C032B25D094F99D20002A15DAD4F8FC
:109380000031DA041FD40025637EEB40DB07EAB22C
:109390001FD40135082DF7D123781BB1237C0BB1E5
:1093A000636873B9174801F09FF977231449D2B263
:1093B0002046FFF791FF2378032B02D0237C032B59
:1093C000DDD104B070BD637E002BDCD10123637658
:1093D000D9E73820019201F0C3FC064618B1019A82
:1093E000214651F0A5F931462046FFF725FF2378A5
:1093F000032BE6D0237C032BCBD1E2E70000003423
:1094000091A40608242F0908054B1B682BB141695C
:109410004A1C02D018462FF0D5BA0020704700BF72
:109420000860002002290BD8242303FB010191F8D6
:10943000390030B191F83A0018B191F83B0070470B
:10944000002070472DE9F04704464FF059FDD4F84D
:10945000F86042F21073861B9E4288BFC4F8F80081
:1094600000274FF0240942F2107A237CFDB2AB4270
:109470001CD929462046FFF7D5FF70B109FB0548E6
:1094800098ED0D0AD8ED097AD4ED250A30EE270AB9
:109490002046FFF7E7FD88ED0C0A564504D909FB85
:1094A000054030302BF064FA0137DEE7617C20465E
:1094B000FFF788FE84ED3D0ABDE8F08770B52DED1D
:1094C000028B044686B04FF01BFDD4F89830C31AC7
:1094D000B3F57A7F05463FD33C4B94ED257A1B6864
:1094E0009FED3B8ADB6AD4ED247A93F89C60F0EE22
:1094F000C76AF4EEC86AF1EE10FA22D5F0EEE76A18
:10950000F4EEC86AF1EE10FA1BD502A801F004F9D6
:1095100016BBFDF7D7FD02A9FDF7B8FBE0B1DDED05
:10952000037A9FED2C7AF8EEE77A67EE877AB0EE51
:10953000E77AB4EEC87AF1EE10FA11D4C4ED257AC8
:1095400011E077EE676AB7EE006AF0EEE66AF4EED5
:10955000C66AF1EE10FA1EDC06B0BDEC028B70BDDF
:109560001D4BC4F89430C4F89850FDF7ABFDFDF7DF
:10957000FFF82046FFF766FF38F070FE0546D4F886
:109580009400F6F7B9FF154ACDE9000106212846F7
:1095900033F032FDE0E7F0EEE76AF4EEC86AF1EE90
:1095A00010FAD9D4002EC9D02046903080ED007A30
:1095B0002BF0DEF938F052FE094A012106B0BDEC6D
:1095C000028BBDE8704033F017BD00BF405D002046
:1095D000000000340AD7233C6F12833A6D2F09082C
:1095E000482F0908F0B52DED048B85B0044640F2F4
:1095F000723200F5867103A80AF05AFFD4ED227A80
:10960000D4ED236A9FED796A637C37EEE67A2422F3
:10961000B0EEC77AB4EEC67AF1EE10FAC1BF9FED94
:10962000747A67EE877A9FED737AE6EE877A02FBAB
:1096300003430025C4ED237A93F839602378E9B217
:109640008B4206D904EB81030135586800F09EFA7D
:10965000F4E7DFED698A9FED698A9FED699A00273B
:10966000237CFDB2AB4264D9242303FB054393F86A
:109670003920002A5BD0D3ED0C7AF4EEE87AF1EED3
:1096800010FA0BDBF4EE677AF1EE10FA06D6F0EE84
:10969000E77AF4EE487AF1EE10FA04DD242303FBB6
:1096A00005435A6A1A63242303FB0543D3ED090AD1
:1096B000D3ED0D7A93F8382070EEA70AA2B993ED96
:1096C0000C0A2046FFF782FCD4ED257A30EE670ABB
:1096D000B4EE400AF1EE10FA16D7242303FB054539
:1096E000002385F83A3022E0012A09BFD3ED0C7A35
:1096F00093ED0B0A77EEE00AD4ED3B7A04BF80EEDF
:10970000897A87EE270AE3E7F0EEC07AF4EE487A2A
:109710002423F1EE10FA03FB0545E1DC012385F873
:109720003A30D4ED237A37EE800A85ED0B0A013703
:1097300096E7627C20461146FFF774FE48B124216B
:1097400001FB024292ED0B0AD16904F1A80030F04E
:109750007DF994F99C10277C002907DBB94205DAD2
:10976000CAB211462046FFF75DFE68B90022627456
:10977000D5B2AF4209D929462046FFF753FE013240
:109780000028F5D0657400E062742046FFF796FE6D
:109790002046FFF739FE10B1204650F015FC637CDF
:1097A000242505FB034393F83930B34216D02FF03C
:1097B0003FF94FF6FF712FF005F978B1607C05FB9A
:1097C000004494F83930002B14BF00220422019287
:1097D0002FF02EF9019A12212FF086F803A80AF033
:1097E00089FE05B0BDEC048BF0BD00BF0AD7233C59
:1097F0000AD7A33C48E17A3F00000034FFFF7F7F97
:10980000002019462DE9F04F0446007C0F4687B032
:1098100004F13A0300220121D5B2A84203F1240346
:1098200005D903F8231C03F8241C0132F4E76F4B1D
:109830001E68F06A03685B68984740B138F00EFD17
:109840006B4A062107B0BDE8F04F33F0D5BB38F0C6
:1098500005FD684A062133F0CFFB002303A904F17C
:10986000880003932BF040FC0A254FF049FB80460B
:109870002046FFF7B7FE4FF043FBA0EB0800B0F522
:10988000FA7F02D95C4800F02FFFB06A03680A2112
:109890005B689847617C2046FFF7C4FD0028E7D04D
:1098A000B06A036864215B68013D984715F0FF05C5
:1098B000DBD1524B05951B888DF80650CDE9035539
:1098C000ADF8043005254FF01BFB80462046FFF71E
:1098D00089FE4FF015FBA0EB0800B0F5FA7FD1D858
:1098E000617C2046FFF79EFD0028EFD094F810B071
:1098F0000DF10C08A14601AA4FF0000A5FFA8AF1A7
:109900008B4516D92046FFF78DFD50B1D8ED007A72
:1099100099ED097A137877EE877A0133C8ED007AEA
:1099200013700AF1010A08F1040809F1240901324F
:10993000E4E7B06A036864215B68013D984715F06D
:10994000FF05C0D1A9464FF02408237C5FFA89F6B1
:10995000B34226D906AB334413F8143C33B908FBA1
:10996000064686F83B3009F10109EEE7002FFAD0F0
:1099700007EE903A06AA02EB8602F8EEE77A12EDBD
:10998000030AD4ED250A204680EE270AFFF76AFB7A
:1099900008FB064002A930308DED020A2BF0A4FB33
:1099A000E1E7617CDFF85C902046FFF70BFC0026C6
:1099B00084ED3D0A4FF02408237CF7B2BB420FD957
:1099C00008FB074393F83B3043B138F047FC7B1C5E
:1099D0004A46062133F010FB0135EDB20136EBE7C4
:1099E0000DB907484FE707B0BDE8F08F405D002094
:1099F000882F0908B32F0908C92F0908FCE30808B4
:109A000005300908E32F090808B5037C022B02D9A9
:109A100003484FF043FA5A1C0274184608BD00BFB1
:109A20002430090838B5057C02460024E1B28D4295
:109A300006D91046FFF7F6FC01340028F6D138BDF0
:109A4000281E18BF0120FAE770B50D4609780729CE
:109A5000044606D8027E437E22B901228A4013437F
:109A6000437670BD002BFCD000262278F3B29A42D8
:109A7000F7D904EB8303294658680368DB689847E5
:109A80000136F2E737B50D460192FFF7CBFF01999A
:109A9000044630B90448054B00682A46C06A0AF0FB
:109AA00001FF204603B030BD405D00201B130A08B3
:109AB000014B1868704700BF685D002070470000C8
:109AC00073B543681B7C8B4205460C4642D900F1B6
:109AD0000801212201A80AF0EBFC4FF011FA6A6894
:109AE000242303FB0423D969411AB1F5FA7F33D249
:109AF000196A401AB0F5FA6F2ED2D3ED097A9FEDAC
:109B0000177AF0EEE77AF4EEC77AF1EE10FA54BF66
:109B100001200020242606FB04F31A449FED107A4E
:109B200082F8390069680B44D3ED0A7AF4EEC77AFB
:109B3000F1EE10FA06D49FED0B7AF4EEC77AF1EE4F
:109B400010FA04DD06FB0411002381F8393001A866
:109B50000AF0D0FC02B070BD0020DBE7000000344A
:109B6000000048C30000484310B5044B0446C0E958
:109B7000003108304EF080FB204610BDE03109086E
:109B80004368242000FB0131CA63704713B50368A2
:109B9000019104469B689847236801991B692046F8
:109BA00002B0BDE810401847F8B52DED028B4368B0
:109BB0001B7C8B4205460C46F0EE408AB0EE608A74
:109BC0001FD94FF09DF924276B6867433B4493ED01
:109BD000090AF0EE680A06460EF02CF8A0B96B6888
:109BE000242202FB04331E626B6824214C4323446D
:109BF000C3ED098A6B68234483ED0A8A69680C44C3
:109C0000E661BDEC028BF8BD6B683B4493ED0A0A3C
:109C1000F0EE480A0EF00EF80028E0D0E4E700006D
:109C2000DFED2A7AB0EEC07AB4EE677AF1EE10FA80
:109C300049DCB4EE400AF1EE10FA44D6436893F9D9
:109C4000FC3063B190ED087ADFED217AF0EEC76A5F
:109C5000F4EEE76AF1EE10FA03D580ED080A01236D
:109C60002BE077EE407A37EE006AF0EEE77AC7EE47
:109C7000866ADBB29FED176A07EE903A26EE866A97
:109C8000F8EE677AB4EEE76AF1EE10FA9FED126A29
:109C900015DDF2EE047A66EEA76A436AC6EE267A0E
:109CA000013343620023F7EE006A76EEE76A27EE9F
:109CB000800AA7EE260A80ED080A18467047F0EEE3
:109CC000467A0123EFE70023F7E700BFFFFF7F7F1E
:109CD0000000003400004843CDCCCC3D90F83C352A
:109CE000934207D900EB8200D0F8140510B1036845
:109CF0009B6A1847002070472DE9F34105466E46E0
:109D000086E80C00134B45F8043B04460F4600F56B
:109D1000C87828462C3500F00FFCA845F9D196E804
:109D2000030004F5A863C4F8387583E80300089BB2
:109D3000C4F84835084920462AF042FC074B1A6807
:109D400012B107484FF0AAF820461C6002B0BDE8E7
:109D5000F08100BFC8330908903209086C5D00200B
:109D6000F43109082DE9F74F90F83C650446002EC0
:109D70004DD17F2380F84C3500F5C87500F214589A
:109D8000071D5FFA86F91822FF21284670F04EFA67
:109D900085F8589097F924A0BAF10A0F4DD039DC14
:109DA000BAF1040F0FDCBAF1020F0FDD442000F00E
:109DB000D7FF834620B13B462A46214650F056FD48
:109DC000C8F800B002E0BAF1090F2AD0D8F80000B4
:109DD00050B1296EC5F85CA031B1254B43F826106F
:109DE0002AF0FCFD2AF0F2FD58F8040B09F10109F4
:109DF0005FFA89F920B103689B68984784F83C951D
:109E00000136092E05F1640507F12C07B9D103B01D
:109E1000BDE8F08FBAF1190F1DD0BAF11F0FC5D0F0
:109E2000D4E7382000F09CFF83460028C8D03B468A
:109E30002A46214651F092F9C2E7302000F090FF07
:109E400083460028BCD0CDF800903B462A462146E8
:109E500051F01EFBB4E7482000F082FF8346002843
:109E6000AED03B462A46214651F084FBA8E700BF0E
:109E7000705D002090F83C358B4283BF642303FB68
:109E8000010090F8D50100207047000090F83C35A3
:109E90008B4283BF642303FB010090ED6A0A9FEDB0
:109EA000010A70470000000090F83C358B4206D94B
:109EB00000EB8100D0F8140508B150F089BE9FED89
:109EC000010A70470000000010B490F83C458C4235
:109ED0000A4614D900EB8104D4F814457CB1E46837
:109EE000246A640603D55DF8044BFFF7DDBF6421E7
:109EF00001FB020393ED6A0A5DF8044B70479FED86
:109F0000010AF9E70000000090F83C358B420BD9BC
:109F100000EB8100D0F8140538B1C3681B6A1A42FF
:109F200014BF0120002070470020704770B590F8E2
:109F30003C35934204460E46154601D8002070BDBC
:109F400000EB8203D3F814050028F7D003689B695F
:109F500098470028F2D0642202FB0544D4F8AC31C3
:109F60003360ECE770B590F83C35934204460E46FA
:109F7000154601D8002070BD00EB8203D3F814050C
:109F80000028F7D003689B6998470028F2D0642224
:109F900002FB0544D4ED6C7AF4EE677AF1EE10FA28
:109FA000E8D6C6ED007AE6E770B590F83C35934206
:109FB00004460E46154601D8002070BD00EB820312
:109FC000D3F814050028F7D003685B699847002888
:109FD000F2D0642202FB0544D4F8B4313360ECE7DC
:109FE00090F83C3593420ED900EB8203D3F8143538
:109FF0005BB1642303FB020292F8E40130B1D2F8B2
:10A00000E0310B6070470020704718467047000031
:10A0100008299DBF2C2303FB0100406800207047E6
:10A020002DE9F04F4B4B2DED028B1B68DB6A93F84B
:10A030009C3089B00446002B00F08680DFF82CB1FC
:10A040009FED458A4FF0000994F83C355FFA89F599
:10A05000AB4279D904EB8503D3F8140500285DD011
:10A0600003685B6B9847642303FB0543074693F83B
:10A07000D431834252D2032861D8DFE800F04F0286
:10A080005259364E4FF0000838F0E8F894F83C2565
:10A09000AA4284BF642202FB05424FF0640105F12D
:10A0A000010301FB05458CBFD2F8A82118EE102A48
:10A0B0008246D5F8B001CDE90632F6F71DFA079AC7
:10A0C000CDE904011046F6F717FA069B0096CDE994
:10A0D00002015A460421504632F08EFF0123204AE5
:10A0E00084F84D3585F8D471D372D4F848354BB324
:10A0F000002255B25957481C03D0414502F10102D4
:10A10000F7D194F94C35AB4208DBD4F84435D4F898
:10A11000400542463146984784F84C5509F10109FB
:10A1200092E72C2303FB05430E4E93F92B80ABE7FC
:10A130002C2303FB05430C4E93F92C80A4E7002647
:10A14000B046A1E71D46DCE709B0BDEC028BBDE8D7
:10A15000F08F00BF405D00200000000021320908A0
:10A16000ED5D0020A61E0A081832090830320908E1
:10A1700090F83C358B4207D900EB8100D0F81405EC
:10A1800010B10368DB6918470020704708299CBF9D
:10A19000642303FB010000F5C870704790F83C355C
:10A1A000934207D900EB8200D0F8140510B1036880
:10A1B0005B6A1847002070472DE9F04F002493B0E8
:10A1C00005460E46174621462F2206A8059405F29D
:10A1D000145970F02BF805F1280A4FF02C0B05F5F7
:10A1E000F6730BFB04F259F8040B1AF90210E5B2EE
:10A1F00030B951B90134092CF3D14FF0010813E003
:10A20000642262439A58914212D01548154B006857
:10A2100001930135EDB20095134BC06A32463946C1
:10A220000AF040FB4FF00008404613B0BDE8F08F45
:10A2300005A93322039350F0ADFD039B804605A989
:10A240000028D7D1064801910135EDB2006800958C
:10A25000054BC06A324639460AF024FBE4E700BFEA
:10A26000405D00204D3C0908583209082DE9F04FA7
:10A27000DFF88090DFF880A0DFF880B08DB0064670
:10A28000002796F83C35FCB2A3422ED9642505FB85
:10A29000046595F8DC3133B395F8DD1119BB4FF047
:10A2A00001082022444404A889F819806FF0BEFFF9
:10A2B00007EE904A4AF21043F8EEE77A03AA4C21DF
:10A2C000ADF8283050462423CDED037A32F0A6FCB9
:10A2D00037F0C4FF9BF80030054A0094042132F0A7
:10A2E0008BFE85F8DD810137CBE70DB0BDE8F08F3F
:10A2F00068320908ED5D002089600020CD22002031
:10A300002DE9F04F2F4B1E6885B0044646B1D0F8BA
:10A31000381530462EF056FB10B130462DF0F4F9CA
:10A320004EF0EEFD4FF0000801904FF02C0A4FF078
:10A33000640B94F83C355FFA88F5AB4239D904EBED
:10A340008507D7F8140588B30AFB05430BFB0549BD
:10A3500093F92820D9F8EC118A4227D132B3026848
:10A36000D2689047D7F814050268126B904799F8A5
:10A37000D52112B1019BC9F8D831BEB1D4F8381536
:10A3800030462EF01FFB88B14EF0C2FDCDE9021021
:10A3900002460B46D7F81405294650F0F3FEDDE9D6
:10A3A0000232D7F81405294650F062FF08F101087F
:10A3B000BFE72046FFF734FE204605B0BDE8F04F6A
:10A3C000FFF754BF086000202DE9F0474FF0000868
:10A3D0002DED028B04468946B0EE408A47460126A1
:10A3E0004FF0640A94F83C355FFA88F5AB421AD90D
:10A3F00029FA05F3DB070AD504EB8503D3F8140526
:10A4000078B10368B0EE480A9B6B984706400AFB98
:10A41000054508F1010895F8D4319F4238BF1F4621
:10A42000E0E70646F3E727B97F23A4F84C35034B52
:10A43000DF72BDEC028B3046BDE8F087ED5D002099
:10A4400090F83C358B4207D900EB8100D0F8140519
:10A4500010B10368DB6B1847002070470B461146AC
:10A4600090F83C259A4207D900EB8300D0F81405F8
:10A4700010B103681B6C18477047000070B50446A4
:10A480000E46002594F83C35E9B28B4205D9324698
:10A490002046FFF7E3FF0135F4E770BD2DE9F843EF
:10A4A00090F83C550246002400F128062C2700F5C0
:10A4B000F6784FF06409E1B28D420FD907FB04F33F
:10A4C00009FB04F0F35658F80000834209D11BB190
:10A4D0001046FFF7CFFC10B10134ECE70120BDE8D6
:10A4E000F8830020FBE7000010B590F83C258A4275
:10A4F000044617D9642202FB010393F8D431022BDE
:10A5000003D004D9032B18BF0023184610BDFFF752
:10A5100097FF48B92046FFF7C1FF00280CBF06236C
:10A520000123F2E70023F0E70623EEE7014B18686A
:10A53000704700BF6C5D002010B5034904462AF047
:10A540003FF8204610BD00BF4834090810B5044646
:10A55000203041F043FC044B04491C6020462AF0A3
:10A560002FF8204610BD00BF945D0020C0350908BB
:10A57000F7B5B7EE000A00220221044629F010FECA
:10A58000204651F05FF841F017FD144B1D68064658
:10A59000E86A03685B6A98470B460221024600910D
:10A5A000304641F031FCB4F94E60002E14DDEF6A04
:10A5B0003B6838465B68B4B2984728B197F84D308D
:10A5C00013B1C92EA8BFC824A86A03685B682146D6
:10A5D00003B0BDE8F040184703B0F0BD405D002077
:10A5E00010B5044650F0E4FF2046BDE8104051F09D
:10A5F0000FB800002DE98048284BDFF8A490DFF861
:10A60000A4A0DFF8A4B01446012293B005460E467C
:10A610001A704FF000084EF073FCD9F80030039325
:10A62000A0EB080241F287339A4207461FD9CDE9D1
:10A63000005603985346342205A9C06A0AF032F93D
:10A64000214605A804944DF095FECDE900560398E7
:10A650005B46342205A9C06A0AF024F9049437F055
:10A66000FDFD049B05AA022132F0AEFCB84637F08E
:10A67000F5FD36F0F1FE37F0F1FD38F033FD0A213B
:10A6800005A809F0FBFE039B986A036805215B6837
:10A69000984705A809F0FEFEBDE700BF985D0020C1
:10A6A000405D0020383509080D340A080FB400B5A4
:10A6B00095B016AA002152F8043B039205A83C224B
:10A6C000019304916FF0B2FD054A019B402104A85B
:10A6D0004DF0F8FD039A034804A9FFF78BFF00BF74
:10A6E00040350908563509080FB407B504AA0348D0
:10A6F00052F8041B0192FFF77DFF00BF683509087F
:10A7000008B5044910226FF037FDB0FA80F0400917
:10A7100008BD00BF9C5D0020102200216FF086BDA7
:10A720000378416023F00D03022A037008D0032A46
:10A730000AD0012A03D1DBB243F001030370704752
:10A74000037843F00803F9E7037823F0050343F0A7
:10A750000503F3E773B504460E4615460193FFF76C
:10A76000DBFF2046C4E90265069A0199FFF7D8FF8E
:10A7700002B070BD4B6843600A78037862F300034F
:10A7800003700B780278C3F3800363F382020270D4
:10A790000B78D2B2C3F3C00363F3C30202707047F5
:10A7A0000078420704D4030704D400F00100704786
:10A7B0000320704702207047F0B585B00546164665
:10A7C000FFF7EEFF88420F4605D16B683360012426
:10A7D000204605B0F0BD032801D10024F8E7032985
:10A7E000FBD001280BD0022816D018BB6D68012FB2
:10A7F00022D0022F2ED0002FEFD13560E7E7FCF7F3
:10A8000061FC90F89432DB07E7D56D68FCF75AFCE1
:10A81000D0F888321D44EAE76846FFF77DFFFCF771
:10A8200051FC6946FCF732FA04460028D0D06D6826
:10A83000019BEFE70025DAE7FCF744FC90F894422F
:10A8400014F00104C9D0FCF73DFCD0F88832ED1AB1
:10A850003560BDE76846FFF75FFFFCF733FC6946EC
:10A86000FCF714FA04460028B2D0019BEFE7000081
:10A8700073B501AA05460E46FFF79EFF044620B1B8
:10A88000019932462846FFF74BFF204602B070BDC3
:10A8900013B5144601AAFFF78FFF48B1DDED017A29
:10A8A0009FED047AF8EEE77A67EE877AC4ED007AD6
:10A8B00002B010BD0AD7233C07EE900A9FED090AAB
:10A8C000F8EEE77A08B527EE800A6DF0CFF8DFEDF5
:10A8D000067AB4EEE70AF1EE10FAD8BFB0EE670AD6
:10A8E00008BD00BF50E0EF300AD7233C10B5044646
:10A8F00080680DF01FFC20B1E068BDE810400DF04D
:10A900002DBC10BD73B5856804460E461DBBC368DB
:10A9100023B98B688360CB68C3600125636873B912
:10A920002378DB070BD52046FFF73AFF01AA014643
:10A930003046FFF741FF10B1019B6360054620469A
:10A94000FFF7D4FF20B9B368A360F368E360012583
:10A95000284602B070BD0025E0E700000D4B8342A1
:10A960004FF000038B4106DA00F1255000F531105D
:10A9700000F5E0507047084B98424FF0FF3371EB01
:10A980000303BEBF00F1564000F5130000F524405C
:10A99000704700BF00D2496B002EB69490EA010FB9
:10A9A00001D4401A7047C317401A63EBE1710D4B95
:10A9B00083424FF000038B4106DA00F1255000F589
:10A9C000311000F5E0507047074B98424FF0FF33CD
:10A9D00071EB0303BEBF00F1564000F5130000F514
:10A9E0002440704700D2496B002EB69470B52DED0F
:10A9F000028B84B0044668460D46FFF78DFEFCF7D7
:10AA000061FB6946FCF742F9064608B3A368029A5F
:10AA1000DFED128A03999B1A07EE903AF8EEE77A77
:10AA200067EEA87AC5ED007AE068FFF7B7FF08EE99
:10AA3000100AA068024402EBD272B8EEC88A501025
:10AA4000FFF73AFF28EE288A28EE000A85ED010A72
:10AA5000304604B0BDEC028B70BD00BFF67C8E3F6B
:10AA600037B500230C4601AA022105460193FFF7E2
:10AA7000A3FE10B9002003B030BD21462846FFF7E1
:10AA8000B5FF0028F6D0DDED017AF8EEE77AC4EDE7
:10AA9000027AF0E710B52DED028B84688A680B46C8
:10AAA000111B08EE901AC168D868FFF777FF22449F
:10AAB00002EBD27208EE100A5010FFF7FDFEB8EE5E
:10AAC000C88AF8EEE88A28EE000A20EE000AA8EE0E
:10AAD000A80ABDEC028BB1EEC07A9FED020A27EE08
:10AAE000000A10BD8262363CF0B52DED028B0D469A
:10AAF00089B08C680646D0E90271E868FFF74EFF1E
:10AB000008EE100AE01900EBD0704010FFF7D4FEF9
:10AB100073686A689FED0E1A9B1A07EE903AE41B61
:10AB2000B8EEE77AF0EE400A07EE904A9FED090A88
:10AB3000B8EEC88AF8EEE77A28EE008A27EE011A06
:10AB400027EE800A68EE200A09B0BDEC028BF0BD4A
:10AB50000AD7233C8262363C84B004B0FFF7C4BFFE
:10AB600038B52DED028B0C460246C168E068FFF750
:10AB700015FF9568A46808EE100A601900EBD07004
:10AB80004010641BFFF798FE07EE904AF8EEE77A54
:10AB9000F8EEC80A87EE807ABDEEC70A10EE103ACA
:10ABA0005B4200EE103AB8EEC00A6DF081F9DFEDBD
:10ABB000087A30EE270ABDEC028BB5EEC00AF1EE42
:10ABC00010FA44BFDFED037A30EE270A38BD00BF2C
:10ABD000DB0FC93FDB0FC94030B52DED028B0B46B3
:10ABE00085B08C68D0E90251D868FFF7D7FE08EE2F
:10ABF000100A601900EBD0704010FFF75DFE641B77
:10AC000007EE904AF0EE400AB8EEC88A9FED060AB9
:10AC1000F8EEE77A28EE008A27EE800A68EE200A2E
:10AC200005B0BDEC028B30BD8262363C82B002B012
:10AC3000FFF7D2BFF0B52DED028B0B468F68D0E940
:10AC4000025185B0D868FFF7A9FE7B1903EBD373D7
:10AC500004465810FFF730FE781B10EE106AF5F727
:10AC600039FC14A3D3E90023F5F79EFCF5F794FF14
:10AC700008EE100A2046F5F72DFC0EA3D3E90023B9
:10AC8000F5F792FC044630460D46F5F735FC0246D2
:10AC90000B4620462946F5F787FCF5F77DFF00EEC9
:10ACA000900AB0EE480A05B0BDEC028BF0BD00BFC3
:10ACB000AFF300800000004050CC863F094B984223
:10ACC00006DDC0F1D64000F5930000F5A4407047C2
:10ACD000054B9842BEBFC0F1144000F5360000F5A8
:10ACE0003850704700E9A43500175BCAF8B52DED60
:10ACF000028BDFED148A076820EE280A0646FDEE77
:10AD0000C07A0D4617EE904A04EBD47007EB600052
:10AD1000B0EE608AFFF7D0FD28EE288A3819C8EE19
:10AD2000007AFFF7CBFF306017EE900AF6F70EF9C6
:10AD30002B68C01841EBE371FFF710FEBDEC028BEE
:10AD40002860F8BD02AAB34200F10C010830FFF7F9
:10AD5000CDBF00000148FFF7DFBC00BF9C5D0020B5
:10AD60000121884238BF08466AF0AEBFFFF7F8BF3E
:10AD700008B16AF0ADBF7047FFF7FABFF8B50646F5
:10AD80000F46144622B96AF0A3FF25462846F8BDAF
:10AD900010461EB9BDE8F8406AF066BF6AF064FF6D
:10ADA00005460028F2D0BC422246314628BF3A462A
:10ADB0006FF0F2F930466AF08BFFE7E737B50446EB
:10ADC0000846089D11461A46036801959DF81C50D7
:10ADD00000951D68069BA8472060204603B030BD43
:10ADE00000214FF0FF3310B50022036304460160D9
:10ADF0000171C0F80510417280F8251000F13C0384
:10AE000000F50B70D9709A60DA601A615A619A6124
:10AE1000DA611A625A629A62DA631A645A649A644C
:10AE2000DA641A655A659A65DA65DA661A675A67E6
:10AE30007C339842E6D1214604F5167004F024F8DC
:10AE4000044B1A6822B904491C60204629F0B8FB5B
:10AE5000204610BDAC5D00202838090873B5D0F835
:10AE60003C3201919942044613D0D0F840329942C5
:10AE700018D0D0F844328B4216D102200AE0D4F820
:10AE8000343253B3D4F838324BB34FF0030002B02E
:10AE900070BD002094F822308342F8D8431C84F817
:10AEA0002230F4E70120F5E7D0F83062002EE6D139
:10AEB00094F841233546B6009AB1A319C3F830126D
:10AEC000A319019AC3F83C2294F82230AB429CBFEC
:10AED0006B1C84F822302846D9E70126E8E70226D1
:10AEE000E6E704F50C7001A930442AF00BFAE7E715
:10AEF00038B504460D462AF07BF9291D201D2AF09D
:10AF000077F905F1080104F108002AF04BFA05F180
:10AF1000140104F114002AF045FA05F1200104F1AE
:10AF200020002AF03FFA05F12C0104F12C002AF050
:10AF3000F3F805F1300104F130002AF0FBF905F1D6
:10AF40003C0104F13C002AF02DFAAB6BA3636B6B60
:10AF5000636338BD2DE9F043A1B00023002500F163
:10AF60003C0706468DF80750039304930593069318
:10AF70000793089309930A930B93109311931293D9
:10AF80001393149315931693179318931C931D936F
:10AF90001E9300F50F78B94658F8043BF3B1F26EF2
:10AFA000934223D0D6F8E820934221D0D6F86421EA
:10AFB000934213D10221EBB299420FD0C1EB411160
:10AFC00009EB8104214601A8FFF792FF394620468C
:10AFD000FFF78EFF01A93846FFF78AFF0135032DE1
:10AFE00007F17C07D8D121B0BDE8F0830021E2E76A
:10AFF0000121E0E72DE9F04704460E46154680465C
:10B0000007464FF0000A31462046FFF727FF7A6FC8
:10B01000B2425FFA8AF90ED1C3B2022B0BD87C225E
:10B0200002FB0A44012084F83E0084F83F3085F892
:10B030000090BDE8F0870AF1010ABAF1030F07F1A9
:10B040007C07E0D1002731462046FFF707FFD8F8FC
:10B050006C205FFA87F912B9C3B2022B19D90137F4
:10B06000032F08F17C08EED131462046FFF7F6FEAB
:10B07000C2B2C2EB421304EB830393F83E7067B98C
:10B08000022A0BD8012083F83E0083F83F202A7063
:10B09000CFE77C2000FB0744C4E700274FF07C0982
:10B0A00004F13E0A31462046FFF7D8FE034609FB6D
:10B0B00007F05FFA87F81AF8002012B9DBB2022B0A
:10B0C00009D90137032FEDD194F8230004280BD9B7
:10B0D00014484DF0E3FE0444012084F83E0084F857
:10B0E0003F3085F80080A4E704F54377002157F846
:10B0F000043BB342CAB208D1904202D8531C84F830
:10B10000233003322A70002093E73BB9411C04EB43
:10B11000800084F82310C0F80C63F2E701310529A0
:10B12000E5D1F0E760360908C9B200EB8101D1F83A
:10B130003C3253B1026F93420AD0D0F8EC209342D4
:10B1400008D0D0F86821934206D04FF00300704732
:10B150000020704701207047022070472DE9F84316
:10B160000F469146044600F5BA7894F83E5035B93A
:10B170007C344445F9D100252846BDE8F8830023F6
:10B180004A463946012009F00FF800210646E06ED4
:10B1900009F01AF88642EBD1EEE70000012303FA2A
:10B1A00001F1D0F8083319420AD14AB190F82030A1
:10B1B000032B1FBF591C80F8201000EB8300426155
:10B1C000704700002DE9F043DFF87C8085B004462D
:10B1D00000F50F7600257C27B14656F80C3CD9F8CF
:10B1E00000209342E9B206F1040619D1C3B120460A
:10B1F000FFF79AFFC0B207FB004090F83E307BB9E2
:10B2000003A9A9F10C0003932AF07CF837F026F883
:10B2100056F8043C009342462B46012131F0ECFEE7
:10B220000135032DD8D104F16C0504F5F0742968BB
:10B2300021B9AB6813B1284628F058FC7C35A542EB
:10B24000F5D105B0BDE8F0837C36090838B5044671
:10B250001546FFF769FFC0B2022808D87C2303FB1C
:10B26000004029465030BDE838402AF08BB838BD40
:10B2700038B504461546FFF757FFC0B2022808D874
:10B280007C2303FB004029465C30BDE838402AF0AF
:10B2900079B838BD37B50D4604468DED010AFFF784
:10B2A00043FF022D07D8C0B27C2303FB004001A955
:10B2B000683029F019FF03B030BD000038B50546ED
:10B2C000FFF732FFC4B2022C13D8C4EB4414A4001D
:10B2D0003C3504F108002844002128F007FC04F163
:10B2E000340104F1300029442844BDE838402AF0F4
:10B2F00009B838BD70B505460E461446FFF714FF71
:10B30000C3B2022B0DD87C2000FB035394E8070046
:10B31000443383E8070031462846BDE87040FFF714
:10B32000CDBF70BD37B504461546FFF7FDFEC0B270
:10B33000022809D87C2303FB00400DF107014030AF
:10B340008DF8075029F054FF03B030BD1FB590F9B8
:10B350002C30044623B390F921300BB36846FFF735
:10B36000DBF9FBF7AFFE6946FBF760FCC0B1DDED32
:10B37000037A9FED0C0AF8EEE70ADDED027AF8EEAB
:10B38000E77A0123C0EE800A84F83D3387EE800A15
:10B3900003F0CCFFDFED047A20EE270A84ED0A0AE1
:10B3A00004B010BD8096184B35FA8E3C024690F9D9
:10B3B000210058B192F8400340B1114491F92C0298
:10B3C00020B192F92400033818BF01207047000013
:10B3D00038B590F8223005465BB100242346E1B22F
:10B3E0002846FFF7E3FF08B10133DBB20134032C39
:10B3F000F5D1184638BD000090ED0A0A70470000EC
:10B4000038B50C46D1ED066A11460546FFF78CFEAD
:10B41000C3B27C2000FB0353D4ED087AD3ED260A97
:10B4200094ED076AD3ED255A93ED245A26EE600A6F
:10B4300067EEA00AA5EEA70AF0EE607AE5EE867A3E
:10B44000B7EE007AA6EEE67A67EEE60AB1EE400ABB
:10B45000E5EE070A6CF02CFD9FED071ADFED070AF9
:10B4600040F658000CF0BCFCD5ED0A7ABDE8384037
:10B4700030EE270A0CF0A0BCDB0F4940DB0F49C0BF
:10B480002DE9F04190F822308B4204460D4602D25D
:10B490000020BDE8F081FFF747FEC0B204F13C0692
:10B4A000C0EB401006EB800008300FF025F9DFED0F
:10B4B000157AB0EEC00AB4EEE70AF1EE10FAE7D45E
:10B4C00029462046FFF730FEC5B27C2000FB054729
:10B4D0003B6F002BDCD0032DDAD000FB0560303051
:10B4E000D7F86C8029F042F9D7E91B32934201D199
:10B4F000984505D07C2000FB0544C4F86C80C7E764
:10B500000120C6E7000000342DE9F74F04460E463F
:10B51000174600F50F7A4FF0000B5AF8049B5FFABC
:10B520008BF8B9F1000F26D041462046FFF73EFFC9
:10B5300008B341462046FFF7F7FD7C23C0B203FB6A
:10B54000004090F83E505DB908F101031B4ADBB2A0
:10B55000394630464CF0B6FE284603B0BDE8F08FC1
:10B560005AF8102C914506D0154A394630464CF011
:10B57000A9FE0025F0E70BF1010BBBF1030FCCD1C5
:10B580004FF0000894F822305FFA88F18B420DD911
:10B5900020460191FFF774FF054620B90199204626
:10B5A000FFF704FF20B908F10108EBE70125D3E715
:10B5B000044A394630464CF085FECDE7A4360908EA
:10B5C000B9360908DE3609082DE9F0412DED048B66
:10B5D00090F842139FED348ADFED348A9FED349A60
:10B5E00082B00646FFF7A0FD06F13C07C5B27C20FD
:10B5F00000FB057554354FF0000896F822205FFADD
:10B6000088F39A424ED919463046FFF7CFFE10B95B
:10B6100008F10108F1E719463046FFF785FDC4B28D
:10B620007C2000FB0474D4ED157AF0EEE77AF4EE9A
:10B63000C87AF1EE10FA04F154040ED5D4ED017A73
:10B64000F0EEE77AF4EEC87AF1EE10FA05D50020B4
:10B6500002B0BDEC048BBDE8F081294620460FF016
:10B660005BF8B4EEE80AF1EE10FAF0DC2946204669
:10B670000EF050FBB4EEC90AF1EE10FAE7DC2146F9
:10B6800028460EF08FFA68468DED000ACDED010ACE
:10B690000EF034FBDFED077AB4EEE70AF1EE10FAB4
:10B6A000B6DDD4E70120D3E700000034DB0FC93F4B
:10B6B000920A863F00004843022910B5044608D884
:10B6C000FFF732FD7C23C0B203FB004494F83D0039
:10B6D00010BD0020FCE7000013B590F84213019163
:10B6E0000446FFF7E9FF30B10199204602B0BDE8FA
:10B6F0001040FFF75BBE02B010BD0000F7B590F937
:10B7000021500446002D73D090F84053002D6FD087
:10B7100090F84213FFF7D0FF94F83D33064613B973
:10B720002046FFF713FE002594F82020EBB29A4242
:10B7300007D904EB83030135586903689B68984770
:10B74000F2E74DF0DDFB0027224604F5BA7140F226
:10B75000F315D2F89C30C31AAB428CBF00230123EF
:10B7600082F83D307C32914247EA0307F1D194F9E7
:10B770002430032B07D194F83C33002B3BD0D4F872
:10B780003803002849D167B1236B013309D02DF06C
:10B790004FF9216B2DF016F918B12DF049F92CF065
:10B7A000D1F894F92C32002B3AD194F92D32CBBB3D
:10B7B00094F92E3213B1022384F8423394F84213E1
:10B7C0002046FFF779FF8642054611D02DF030F96B
:10B7D0004FF6FF712DF0F6F850B1002D14BF002286
:10B7E000042201922DF024F9019A03212DF07CF816
:10B7F000284603B0F0BD012384F83C330420FFF752
:10B80000AFFA054610B1214603F0DEFB94F924306F
:10B81000C4F83853032BB2D0B5E703F0EFFBB2E71F
:10B820000023C9E70123C7E738B590F92130044662
:10B83000D3B190F84053BDB1FFF776FCC0B20228F7
:10B8400012D87C2303FB0044D4ED1A7A9FED087ACA
:10B85000F4EEC77AF1EE10FA06D4B7EE087AF4EEF9
:10B86000C77AF1EE10FA00DD0025284638BD00BF8A
:10B87000ABAA2A3F70B5D0F8085315F4003504463A
:10B880000E460DD190F840335BB90A78072A07D8E5
:10B89000012303FA02F290F83F33134380F83F3359
:10B8A00070BD94F82020EBB29A42F9D904EB8303DF
:10B8B000314658690368DB6898470135F1E70000B5
:10B8C00038B505466C242B591BB10021281928F0E6
:10B8D0000DF97C34B4F5F07FF5D138BD014B186813
:10B8E000704700BFAC5D002010B50446006810B181
:10B8F00003685B689847204610BD000010B50446F9
:10B90000006810B103685B689847204610BD0000CE
:10B9100010B50446006810B103685B68984720467C
:10B9200010BD000070B51E2288B000210646FFF74A
:10B9300015FC044600B30023CDE904330025059B24
:10B9400007930622294607A8CDE9055501F05AFCC0
:10B95000294602463046FFF721FC07A8FFF7D8FF2B
:10B9600006A8FFF7D5FF05A8FFF7C8FF14B104A884
:10B97000FFF7C4FF08B070BD04230649CDE90103F9
:10B980000968054B0093024649681E2305A8FFF786
:10B9900015FAD3E7405D0020801A060070B5044612
:10B9A000002594F83F33EB40DB07E8B218D40135AB
:10B9B000082DF6D194F82330052B1ED02046FFF732
:10B9C000B1FF94F8203013B194F82230ABB90B4B8F
:10B9D0000B491B6898690368BDE870401B681847ED
:10B9E00001F088FC02460028E1D011212046FFF733
:10B9F000D5FB94F82330052BD9D170BD405D0020D4
:10BA0000F83609082DE9F04F90F9213089B0044645
:10BA1000002B00F00481012300F50C7580F8413300
:10BA2000024600F50F712B462E46D06E002859D0E5
:10BA3000002384F8413394F94030642B5BD094F9AF
:10BA4000BC30642B00F08D8094F93831642B00F009
:10BA50008A80D4F830722FBB01A9204628F02AF83A
:10BA600000B30C230593012306978DF81830714B12
:10BA700007936946BDF80430049704A8ADF8103068
:10BA80008DF8007028F0ECF99DF9001051B10229F1
:10BA900008DC38B1C9B27C2303FB01416C31284674
:10BAA00029F048FC94F841B3BBF1000F5DD0E36E80
:10BAB0006367D4F8E830C4F8F030D4F86431C4F8DF
:10BAC0006C3194F8233003F1C30204EB82020021AD
:10BAD000042B7CD852F8040B1061013342F8041C8B
:10BAE000DBB2F5E753F8040B0028A1D18B4202F139
:10BAF0007C029AD19FE7002066238DF810307C23CA
:10BB000003FB004004A9403029F058FB04A920465B
:10BB100027F0D0FF00289CD004238DF81830002394
:10BB2000CDE90133039331230593694604A828F036
:10BB300097F9059B28B108AA02EB8302009942F805
:10BB4000E01C0133332B0593EFD94AF085FF9DEDBF
:10BB5000031ADDED020A9DED010A66214AF03AFF63
:10BB600077E70120C8E70220C6E70127A94655F874
:10BB7000043B23B1AB600137042FF7D197E7AA4606
:10BB8000B8465FFA88F3022BF5D8DAF8002055F8AA
:10BB9000043C9A4205D104A95046CDF810B029F0D2
:10BBA000C9FB5AF8043B08F101020BB99046E8E7DB
:10BBB00004A906EB88000193CDF810B029F0BAFB78
:10BBC000019BAB6001A9484629F0B4FBD3E794F888
:10BBD000413313B92046FFF7BDF994F822300BB377
:10BBE000154B1B68986A036864215B689847204678
:10BBF000FFF784FD94F83E3003B9E36694F8BA3059
:10BC00000BB9C4F8E83094F836310BB9C4F8643194
:10BC1000FBF758FAFBF7C2FA0123A4F8403309B046
:10BC2000BDE8F08F2046FFF7B9FE94F82230002BD4
:10BC3000E0D0D5E7F4CD0908405D00207047000052
:10BC4000064B10B503600446FFF748FEA06004F100
:10BC50000C004CF011FB204610BD00BF303B090822
:10BC600073B505467C23AC682E7903FB0643C6EB0F
:10BC7000461604EB8604084693F8A41001900EF0D3
:10BC800027FA94F93C3001983BB9AB6893F825103A
:10BC900002B0BDE870400EF01BBA94F84010F7E710
:10BCA00037B58468057901917C2303FB054595F838
:10BCB0003F3004EB8304D4F84C325BB14DF020F9F3
:10BCC000C5F89C000199D4F84C0203B0BDE830409F
:10BCD00002F092BC03B030BD2DE9F04F90F804A003
:10BCE0008768CAEB4A144FEA840806460D4607F1F6
:10BCF0003C0B08F108018BB0594428460EF01EF9A0
:10BD00003179B0680BEB8404FFF78EFD38B17C23EA
:10BD100003FB0A7393ED1A0A28460EF043F97C23BD
:10BD200003FB0A7393ED146ADFED3A7AD3ED156ADB
:10BD3000B0EEC67AB4EEE77AF1EE10FA0FD5B0EEB7
:10BD4000E67AB4EEE77AF1EE10FA08D594ED077AC8
:10BD5000B0EEC77AB4EEE77AF1EE10FA1BD47C238A
:10BD600003FB0A73D86D196E5A6E9B6D0290039196
:10BD70000490079101A829468DED016ACDED056A71
:10BD80000692089209930CF037FA85ED000AC5ED8A
:10BD9000010A85ED021A7C2303FB0A770023C7F80A
:10BDA0008C30C7F88830C7F88430B06890F95C32BE
:10BDB00008F13C0908F14808D944D8446BB13379FB
:10BDC0005BB9414600F5167003F0CEF841462846AF
:10BDD0000BB0BDE8F04F0EF0B1B890F93430012B44
:10BDE0000BD190ED0E0A48460EF088F884ED120A49
:10BDF000C4ED130A84ED141AE8E7022BE6D1FEF72E
:10BE000095FB002201A9FEF791F80028DED09DEDF8
:10BE1000010AE8E70000003410B5037984687C2249
:10BE200002FB034407C904F1900383E807004DF0C7
:10BE300067F8C4F89C004DF057F8C4F8A00010BD96
:10BE4000F0B5054685B0A6220E4600F10C0103A808
:10BE500008F02EFBAC682F797C2303FB0743D3F853
:10BE6000B42022B903A808F045FB05B0F0BDBEB16F
:10BE700096ED007AD3ED2A7A67EE877AC3ED2A7AB7
:10BE800096ED017AD3ED2B7A67EE877AC3ED2B7AA4
:10BE900096ED027AD3ED2C7A67EE877AC3ED2C7A91
:10BEA0007C2607EE902A06FB0741A831B8EE670A08
:10BEB000084601910EF08AF801992846FFF7ACFF79
:10BEC00006FB07430022C3F8B020C3F8AC20C3F838
:10BED000A8200022C3F8B420C4E7000073B50446CC
:10BEE0008068237901917C2606FB03000D466C30A7
:10BEF00001A929F0FFF9A368227906FB02331D6727
:10BF000002B070BD70B5021D044680680E46FFF792
:10BF100071F8054618B131462046FFF7DFFF284685
:10BF200070BD000007B5826803797C2000FB032008
:10BF300090F93C0002280BD002F13C00C3EB431304
:10BF40008DF8071000EB83000DF1070129F02CF9A3
:10BF500003B05DF804FB0000836802797C2101FBDB
:10BF6000023393F93C00003818BF012070470000ED
:10BF7000836802797C2000FB023383F8A4107047A9
:10BF8000F8B5054608460F460EF07EF810B10024BD
:10BF90002046F8BD38460EF05DF804460028F6D17C
:10BFA000AB6893F934637EB138460EF0A5FB95ED8E
:10BFB000097ADFED1F7AF0EEC76AF4EEE76AF1EE78
:10BFC00010FA03D585ED090A0124E1E777EE407AFE
:10BFD00030EE076AF0EEE77AC7EE866AF6B207EE51
:10BFE000906A9FED146AF8EE677A26EE866AF4EEA0
:10BFF000C67AF1EE10FA48BFB2EE046ADFED0E7AAF
:10C0000045BFAB6A66EE866AB0EE676A87EEA66ADF
:10C0100046BF0133AB620124F7EE007A77EEC67AB1
:10C0200020EE060AA7EE270A85ED090AB0E700BF51
:10C030000000003400004843CDCCCC3D2DE9F7434F
:10C0400004460E461746FFF70BFE31462046FFF723
:10C0500027FE31462046FFF73FFE31462046FFF7D8
:10C060008FFF30B304F10C01992201A808F020FAE7
:10C07000A56894F804804FF07C0909FB0854A834A3
:10C08000314620460DF05AFF09FB0851D1F8B43073
:10C090000133C1F8B4304FB1BB4207D35B08C1F8DC
:10C0A000B430B0EE000A20460DF090FF01A808F071
:10C0B00021FA03B0BDE8F08310B50446FFF734F869
:10C0C000C0B23C34C0EB401004EB800010BD000057
:10C0D000F8B50A4E044600F5167704F5137555F8C1
:10C0E000040B08B102F0BCFDBD42F8D13368986A78
:10C0F000036801215B689847EFE700BF405D0020BF
:10C1000008B5FFF7E5FF0000F0B5144E00EB81071E
:10C1100073780446D7F84C026FF3410387B00D469D
:10C120007370C8B101F08AF968B1737843F01003F5
:10C1300073702C440023A372D7F84C0207B0BDE8FB
:10C14000F04001F0FFB8D7F84C12684601F0A6F9AC
:10C15000009B012BEDD1E8E707B0F0BD0C5E00209D
:10C1600070B506460D46002445FA04F3DB07E1B23C
:10C1700002D53046FFF7C8FF0134032CF4D170BD5F
:10C18000FF21FFF7EDBF000030B500F5137587B054
:10C1900000F5167455F8041B21B9A542FAD1002008
:10C1A00007B030BD684601F079F9009B013B022BD6
:10C1B000F3D80120F4E700002DE9F0472DED028BC4
:10C1C00088B004460D469046B0EE408AFFF774FAF8
:10C1D00030B90026304608B0BDEC028BBDE8F087D0
:10C1E00029462046FFF7E2F806460028F1D004EB86
:10C1F0008507D7F83C22D7F830329A4206D036F07D
:10C200002DF85C4A032130F0F7FEE2E7D7F84C3214
:10C2100083B94FF49870FEF7A3FD814608B101F091
:10C2200023FEC7F84C92B9F1000F03D136F016F88F
:10C23000514AE7E7B4F84A32D90711D504F082FC35
:10C2400090F8082390F8C43232B9B02202FB030000
:10C2500090F8A130012B03D836F000F8474AD1E717
:10C260002046FFF791FF20B9454A537843F0020377
:10C27000537094F9353053B329462046FFF71CFF1D
:10C2800090F90030002B53D029462046FFF714FFC9
:10C2900090F80490B9F12B0F19D829462046D7F809
:10C2A0004CA2FFF709FF94F9353090F90020022BDA
:10C2B000D4BF00210121012BD4BF00230123003A68
:10C2C000009118BF01224946504601F04FF863190A
:10C2D00000229A7275B3D4EDC10AB4F84822D7F897
:10C2E0004C0270EEA00A2B46B0EE480A414601F01F
:10C2F0005DF894F83E33002B31D1224A069412683F
:10C300000127E773906A0268156D1F4A079202932E
:10C3100009224FF40063CDE9003208AA12E90600B1
:10C320001A4BA847C8B935F099FF194A02216AE7A4
:10C330009946B2E729462046FFF7BEFE90F9003045
:10C34000002BC8D0D4EDC10AB4F84822D4F84C026E
:10C350002B46B0EE480A4146C9E784F83E730023F5
:10C360000DF1170104F124008DF8173028F026FF95
:10C3700030E700BF403B0908723B0908953B0908BC
:10C380000C5E0020405D002001C10108B33B09089C
:10C39000BE3B09082DE9F0412DED028B00244373CB
:10C3A0009DF82030837305460F469046B0EE408AD4
:10C3B000264647FA04F3DB07E1B210D5B0EE480A8F
:10C3C00042462846FFF7F8FE064640B93946284659
:10C3D000FFF7C6FEBDEC028B3046BDE8F0810134AC
:10C3E000032CE6D1F6E70000F8B500242DED028B12
:10C3F00005460F46B0EE408A427383732646E1B28B
:10C40000B0EE480A3A462846FFF7D6FE0134002827
:10C4100018BF0646032CF2D1BDEC028B3046F8BDA6
:10C42000F0B500EB81030D46D3F84C129BB00446E7
:10C4300011B900201BB0F0BD0BA801F013F863196F
:10C44000987A0028F6D10B9A002A48D0042AF0D115
:10C4500001229A720DAA07CA02AB83E8070010AA4C
:10C4600007CA05AF87E8070013AA07CA9DED180A97
:10C4700008AE86E807001A46294620468DED010AD7
:10C48000FEF738FF3A4629462046FEF7DFFE3246E1
:10C4900029462046FEF7ECFE9DED010A294620467E
:10C4A000FEF7F8FE9DF8643083B129462046FFF779
:10C4B00003FE90F900304BB194F93530012B05DDC6
:10C4C0009DF85D2029462046FEF72CFF2046FFF709
:10C4D0005BFE20B9034A537843F0040353700120F4
:10C4E000A8E700BF0C5E00202DE9F0410546884614
:10C4F00000F513770024012657F8043BE1B26BB135
:10C5000048FA04F3DB0709D52846FFF789FF00281E
:10C5100057F8040C08BF002600F014FF0134032C68
:10C52000EAD13046BDE8F0812E4B2DE9F04F1F686F
:10C53000FB6A93F89C8087B00446B8F1000F38D1AD
:10C54000DFF8A8A000F5137600F1030B054656F8B6
:10C55000040BA5EB04095FFA89F9E8B100F05AFF72
:10C5600028B19AF8013043F008038AF8013056F8F0
:10C57000040C00F063FFF8B9637B6BB1AB7A5BB975
:10C5800056F8041C684600F089FF009B042B03D179
:10C5900049462046FFF744FF01355D45D7D1124B90
:10C5A000204683F81280FFF7EFFD054630B10123E6
:10C5B000237407B0BDE8F08F8046EDE7237C002BA5
:10C5C000F7D0A37B002BF4D0B86A03684FF47A71DC
:10C5D0005B689847B86A03689B6B294607B0BDE85B
:10C5E000F04F1847405D0020ED5D00200C5E0020FC
:10C5F000F0B5002587B000F513762C46012756F8D4
:10C60000041B41B1684600F049FF009B1BB107FACB
:10C6100005F31C43E4B20135032DF0D1204607B0E9
:10C62000F0BD00002DE9F04F2DED028B03270E7CAD
:10C630009FED348A91B005468846B946AC5D013419
:10C64000E4B2B4FBF9F303EB4303E41AE4B205EB01
:10C650008403D3F84C1209B9AC554CE003A800F0A0
:10C660001DFFDDF80CB00BF1FF33022BF4D8304680
:10C670002FF09AFA8246304630F060FA00F11B0340
:10C680009A4508D2304630F0C1FE002011B0BDEC12
:10C69000028BBDE8F08FAC55284698F810A0FFF744
:10C6A000A7FFDDED057A8DF83100FCEEE77A9DF805
:10C6B00010208DF8332017EE903A8DF8343006AB09
:10C6C00003CB1B88ADF83D305C221B23CDE9003243
:10C6D000CDF83500CDF8391009AABF2150468DEDAF
:10C6E000098A8DED0A8A8DED0B8A8DF830408DF820
:10C6F00032B02FF0C3FA013F17F0FF079ED101209F
:10C70000C4E700BF000000002DE9F04F0F7CA1B08E
:10C7100006468846032500EB070999F805400134D1
:10C72000E4B20323B4FBF3F303EB4303E41AE4B2F0
:10C7300006EB8403D3F84C1211B989F805400AE0DE
:10C7400011A800F08FFEDDF844A0BAF1030F08DC59
:10C75000BAF1000FF1DA013D15F0FF05DDD101203E
:10C7600012E0AAF10402032AF5D838462FF01CFA89
:10C770008346384630F0E2F900F13602934506D29E
:10C78000384630F043FE002021B0BDE8F08F89F834
:10C790000540304698F810B0FFF72AFFDDF848E072
:10C7A000CDF80CE0DDF84CE0CDF810E0DDF850E01D
:10C7B000CDF814E0DDF854E0CDF818E0DDF858E0ED
:10C7C000CDF81CE0DDF85CE0CDF820E0DDF860E0BD
:10C7D000CDF824E03219DDF864E01C9BCDF828E0A8
:10C7E000DDF868E092F80AC09DF874109DF8752095
:10C7F000CDF82CE00E93DDF86CE01E9B8DF8350033
:10C800008DF83C108DF83D20CDF830E08DF83440A7
:10C810008DF836A08DF837C02422CDF83E3036236F
:10C82000CDE90032C0212C2303AA58462FF026FA66
:10C8300091E700007FB58A8B0B464AF2B9518A42D4
:10C8400005465FD04AF2BA518A4274D04AF2B851D2
:10C850008A420BD1474A1268D26A92F89C203AB1B8
:10C8600035F0FCFC444A052130F0C6FB042479E095
:10C87000D3ED007AF5EEC07AF1EE10FAF6D49FED22
:10C880003F7AF4EEC77AF1EE10FAEFDC93ED017A1D
:10C89000DFED3B6A1C6993ED030AB0EEC77AB4EE94
:10C8A000E67A93ED027AFCEEE77AB0EEC77AF1EE23
:10C8B00010FAB4EEE67A17EE903A54BF012600263D
:10C8C000F1EE10FA54BF01220022003C18BF0124EF
:10C8D00013F0FF0110D18DED030A0292FEF772FCF6
:10C8E0009DED030A029A234631462846FFF77CFD58
:10C8F0000028BBD0002435E0134600943246FFF7F1
:10C9000049FDF5E7D3ED007AF5EEC07AF1EE10FAC5
:10C91000ACD49FED1A7AF4EEC77AF1EE10FAA5DCEA
:10C92000FCEEE77A17EE903A13F0FF0108BFFF2103
:10C93000FFF7DAFDDCE7D3ED007AF5EEC07AF1EE31
:10C9400010FA93D49FED0D7AF4EEC77AF1EE10FA57
:10C950008CDCFCEEE77A17EE904A14F0FF0404D169
:10C96000FFF70EFC204604B070BD2146FFF7F8FB30
:10C97000C0E700BF405D0020F03B090800007F4396
:10C9800000000034F0B58BB00E4614460746FFF7A2
:10C9900093FB543007C884E8070031463846FFF758
:10C9A0008BFB90ED057ADFED267AB0EEC77AB4EE18
:10C9B000E77AF1EE10FA054611D590ED067AB0EE61
:10C9C000C77AB4EEE77AF1EE10FA08D590ED077A5F
:10C9D000B0EEC77AB4EEE77AF1EE10FA24D431461D
:10C9E0003846FFF769FB016A426A836AE869D5F84D
:10C9F00014E0D5F818C0099001A8CDF804E0029120
:10CA000003920491CDF814C00693079208930BF09B
:10CA10009FFD98B1214601A80BF0EEFB84ED000AC2
:10CA2000C4ED010A84ED021A31463846FFF744FB93
:10CA300000F1080120460DF09BFA01200BB0F0BD7B
:10CA4000000000342DE9F0472DED048BACB0B0EEC2
:10CA5000608A0546B0EE409A0F46F0EE418A904655
:10CA6000FEF7B0FBDFED8B7AB0EEC87AB4EEE77A72
:10CA7000F1EE10FA4BD5B0EEE87AB4EEE77AF1EECB
:10CA800010FA44D523AC2046FDF746FEFAF71AFB10
:10CA90002146FAF7CBF8064658BB04F053F890F855
:10CAA000083390F8C42233B1B02303FB020393F898
:10CAB000A130012B07D84FF0B00909FB020090F814
:10CAC000A130022B0BD835F0C9FB734A032130F09B
:10CAD00093FA30462CB0BDEC048BBDE8F08704F02F
:10CAE00031F890F8C43209FB0300AC300FC884E879
:10CAF0000F00DDED257A9FED691AB8EEE78ADDEDCE
:10CB0000267AF8EEE78A28EE018A68EE818A04AA7E
:10CB100003A902A8F0EE680AB0EE480A02F0F0FAA3
:10CB2000064618B935F09AFB5D4ACFE79FED5D7A6E
:10CB3000DDED027A9FED5C8ADFED5C8A8DED068A81
:10CB400067EE877A2422002111A8CDED057A8DEDBC
:10CB5000078A6DF06BFB9DED031ADDED040ADFF82B
:10CB600058A121EE281A68EEE00AB0EE480A11A892
:10CB70000BF00EFD05A911A80BF03EFB24220021AD
:10CB80001AA8CDED060A8DED071A8DED050A6DF098
:10CB90004DFBFAF797FA90ED840A8DED010AFAF74A
:10CBA00091FA29EE281AD0ED850A9DED010A1AA8FE
:10CBB0000BF0EEFC1AA923A80BF00CFC05A923A886
:10CBC0000BF01AFB4FF000098DED050ACDED060ABA
:10CBD0008DED071A95F822305FFA89F4A3427FF6AB
:10CBE00078AF1FB127FA04F3DB071AD52B1993F995
:10CBF0002C32B3B1B8F1000F0DD021462846FEF714
:10CC00005BFD88B935F02AFB294A2346032130F021
:10CC1000F3F900265DE721462846FEF7C7FB00280A
:10CC2000EBD109F10109D5E708AA214628468DED87
:10CC3000088A8DED098A8DED0A8AFFF7A3FE20B9D7
:10CC400035F00CFB1B4A2346E0E708A905A80DF0C8
:10CC50003FF90BAA214628468DED0B0ACDED0C0AB3
:10CC60008DED0D1AFEF746FB9AE807000EAB83E840
:10CC700007001A4621462846FEF7E8FA23AA21466D
:10CC800028468DED238A8DED248A8DED258AFEF7C9
:10CC9000EFFAC6E700000034143C090895BFD6330C
:10CCA0002F3C090800007A440000000035FA8E3C51
:10CCB000443C0908573C090800E408080120704773
:10CCC0000120704743689868704700004068036817
:10CCD000DB6C184710B5054B03600446C06A10B101
:10CCE00003685B689847204610BD00BF403D0908B7
:10CCF000406803689B6A184733B46C46406884E810
:10CD00000C000368DD6A94E80C00AC4602B030BC4D
:10CD10006047000010B50446FFF7DCFF2046FEF731
:10CD200027F8204610BD0000406807F00DB900004C
:10CD300090F84730DB07014602D53031FFF780B865
:10CD400070470000406807F061B9000040680123A7
:10CD500007F05CB94068002307F034B9F8B5044621
:10CD60001E460F461546FEF76BFF084B2360002357
:10CD700023636363A36394F84730E76265F3410379
:10CD800084F8466084F847302046F8BD403D0908E5
:10CD900010B50D4BC3630446C06A036898221B6933
:10CDA0000021984770B1E06A036820221B690121C5
:10CDB000984738B1E06A0368BDE810401B6901225A
:10CDC00002211847002010BDC5DC6A3F37B5044674
:10CDD000C06A03686A469D6803210623A847E0B13C
:10CDE000BDF80020BDF8041052BA95B249BAB5F5A5
:10CDF000704F0BB213D013F5805F10D0BDF8023026
:10CE00005BBA9DB2B5F5704F09D052425B42A4F8AF
:10CE10004020A4F84210A4F8443003B030BD0020F4
:10CE2000FBE70000C06A036801221B690221184762
:10CE300030B585B00446FFF7C9FF05462046FFF729
:10CE4000F1FF4DB3B4F9403094ED0F0A06EE903A7D
:10CE5000B4F9423007EE103AB4F9443007EE903A94
:10CE6000F8EEE66AB8EEC77AF8EEE77A01A8CDEDFB
:10CE7000016A8DED027ACDED037A0DF093F820462C
:10CE8000FFF76AF818B1022101A80DF021F90E226E
:10CE900001A92046FFF7D2F805B030BDFFF7C8BFA3
:10CEA00013B5C06A036801AA9C680A210323A0473E
:10CEB00038B10549032201A86DF05EF9B0FA80F09F
:10CEC000400902B010BD00BF783C09082DE9F843C5
:10CED00000252DED028BDFF888819FED5D8A0446E9
:10CEE0002E462F46E06A036811221B690021013794
:10CEF000984700287BD0D8F80090D9F8280003681C
:10CF000032215B689847E06A036860221B6901214F
:10CF1000984700286BD0E06A036801221B69022150
:10CF20009847002863D0D9F82800036832215B684D
:10CF300098472046FFF74AFF002858D00135022FB6
:10CF4000EDB256DDB4F940309FED425A9FED426A92
:10CF500007EE903AF8EEE77AC5EE276AF0EEE66A59
:10CF6000F4EEC66AF1EE10FA41DDF4EEC86AF1EEB5
:10CF700010FA3CD5B4F94230DFED385A07EE903A5A
:10CF8000F8EEE77A85EEA77AB0EEC77AB4EEC67A05
:10CF9000F1EE10FA2BDDB4EEC87AF1EE10FA26D5D8
:10CFA000B4F9443005EE903AF8EEE55AC5EE257A2C
:10CFB000F0EEE77AF4EEC67AF1EE10FA17DDF4EE51
:10CFC000C87AF1EE10FA12D594ED0C6A76EE266A64
:10CFD0000136C4ED0C6AD4ED0D6A36EE877A84ED25
:10CFE0000D7A94ED0E7A77EE277AC4ED0E7A192F2A
:10CFF00002D0052E7FF476AFE06A036810221B6929
:10D0000000219847052E18D1D4ED0C6AF1EE047A70
:10D0100086EEA77A0120D4ED0D6A84ED0C7A86EEB7
:10D02000A77AD4ED0E6A84ED0D7A86EEA77A84EDA8
:10D030000E7ABDEC028BBDE8F8834FF07E53052DD0
:10D0400023636363A36394BF00200120F1E700BF63
:10D05000CDCCAC3F00002E443333333F000022449C
:10D06000405D0020F7B50446C06A03685B699847D5
:10D07000054648B9474B48491B68986903681B68CF
:10D080009847284603B0F0BD03689B689847E06A5C
:10D0900003680A21DB6A9847E06A03689B6998473E
:10D0A00060B93C4B3D491B68986903681B68984709
:10D0B0002B682846DB6898470025E2E72046FFF703
:10D0C000EFFE0028F4D02046FFF700FF30B9314BC7
:10D0D00033491B68986903681B68E8E72046FFF737
:10D0E00057FE0028E4D0E06A0368DB69984730B94E
:10D0F000284B2C491B68986903681B68D7E794F88C
:10D100004730E06A43F0010384F8473003680321A5
:10D11000DB6A98472B682846DB68984723682046D7
:10D120009B689847E06A036807215B6A9847E06A52
:10D1300003689B6A984701462046FEF7E3FE0546D2
:10D1400000289ED094F846102046FEF711FF94F870
:10D1500047309B0703D501212046FEF7E3FEE06A36
:10D16000009403681E6A104B019302AB13E90C0094
:10D1700043F21541B047074BE06A1B689E6933686C
:10D180001F6803689B6A9847084902463046B847BB
:10D1900077E700BF405D00207C3C0908A23C0908FD
:10D1A000C83C0908ED3C09089DCE01081B3D090853
:10D1B00010B5084B036004460023086860600B60EC
:10D1C000037A03F00703022B02D1C02106F0EAFF25
:10D1D000204610BD583D090810B5044B044640F8E0
:10D1E000043BFEF795FB204610BD00BF583D0908E3
:10D1F00010B50446FFF7F0FF2046FDF7B9FD2046C5
:10D2000010BD0000F7B503680E4617461BB9002491
:10D21000204603B0F0BD0022026008200193FDF714
:10D220009FFD054610B101A9FFF7C2FF01A8FEF757
:10D230006FFB002DEBD04820FDF792FD044600283F
:10D24000E5D029463B463246FFF788FD2046FFF7EA
:10D2500009FF05460028DBD1236820465B68984714
:10D260002C46D5E77047000010B50446FDF780FD59
:10D27000204610BD0021FEF7E3BD00001FB590F869
:10D280002C200C7894421CD1B1F9052006EE902A8E
:10D29000B1F9072007EE102AB1F9092007EE902A0C
:10D2A000F8EEE66AB8EEC77AF8EEE77A90F82D2045
:10D2B000CDED016A01A98DED027ACDED037AFEF77D
:10D2C000BDFE04B010BD000038B5002390F82C203E
:10D2D00019460446052006F067FF01462046FEF782
:10D2E00011FE054618B101212046FEF71BFE284617
:10D2F00038BD000038B505463020FDF731FD044645
:10D3000078B1FEF79DFC084B84F82C502360204632
:10D31000FFF7DAFF054620B9236820465B68984787
:10D320002C46204638BD00BF903D090800224260CF
:10D330008260C260026142618261C26102624262D5
:10D340007047000013B55822044600F5807101A80B
:10D3500007F0AEF80023C4F8F830012384F8FC305D
:10D3600001A807F0C7F802B010BD0000F7B50446E9
:10D370000D46174600F580715F2201A81E4607F092
:10D3800097F8012384F858309DF8203084F85950DC
:10D3900084F85A5084F85B7084F85C6084F86D30CF
:10D3A00001A807F0A7F803B0F0BD0000F0B52DED1F
:10D3B000028B032B83B004460F46F0EE408A1646DC
:10D3C0001D46B0EE608A0CD800F580716E2201A86F
:10D3D00007F06EF8636F023B012B06D801A807F037
:10D3E00089F803B0BDEC028BF0BDA4F85E600126A5
:10D3F00084F8606084F86170C4ED198A4BF080FD98
:10D4000084F86C50A06684ED158AC4F8F86084F83E
:10D41000FC60E3E713B5044600F580718A2201A899
:10D4200007F046F8246801A8042C94BF00240124C6
:10D4300007F060F8204602B010BD000013B50446A6
:10D4400000F580719E2201A807F032F82468023CA2
:10D45000012C01A88CBF0024012407F04BF82046C2
:10D4600002B010BD73B50C460646A32201F58071CB
:10D4700001A8183407F01CF80FCC35460FC50FCCA7
:10D480000FC50FCC0FC594E8070085E8070001A879
:10D4900007F030F8304602B070BD000073B5A82226
:10D4A00006460C4601A801F5807107F001F80FCC83
:10D4B00035460FC594E8030085E8030001A807F08E
:10D4C00019F8304602B070BDF0B5044691B0084678
:10D4D000D4F8BC10D4F8C020D4F8C430D4F8B0705C
:10D4E000D4F8B460D4F8B85008910A9104F1A401BA
:10D4F00009920C930D920E9307970B960F950CF0D3
:10D50000D1FC04A907A88DED040ACDED050A8DED27
:10D51000061A0AF071FE012101A88DED010ACDED78
:10D52000020A8DED031A0AF071FB00280BDB04EBF5
:10D53000E004012300F0070003FA00F094F88D30B6
:10D54000184384F88D0011B0F0BD0000436F023B1A
:10D55000012B06D8B0F89C00A0F5967358425841AC
:10D56000704700207047000090ED347AB4EE477A9F
:10D57000F1EE10FA80F18280D0ED287ADFED406A7A
:10D58000F4EEE67AF1EE10FA78DDDFED3E6AF4EEC5
:10D59000E67AF1EE10FA71D5B0F88430D0ED296A50
:10D5A00007EE903AF8EEE77AF0EEE66AF4EEE76A14
:10D5B000F1EE10FA62D5D0ED2A6AF0EEE66AF4EEEA
:10D5C000E67AF1EE10FA59DDD0ED2B6AF0EEE66A5C
:10D5D000F4EEE67AF1EE10FA50DD90ED2C6ADFED14
:10D5E0002A6AB4EEE66AF1EE10FA47DDF1EE047A4B
:10D5F000B4EEE76AF1EE10FA40D590ED2D6AB4EE84
:10D60000E66AF1EE10FA39DDB4EEE76AF1EE10FAEF
:10D6100034D590ED2E6AB4EEE66AF1EE10FA2DDD07
:10D62000B4EEE76AF1EE10FA28D5D0ED2F6AF7EEE6
:10D63000007AF0EEE66AF4EEE76AF1EE10FA1DD534
:10D64000D0ED306AF0EEE66AF4EEE76AF1EE10FA39
:10D6500014D5D0ED316AF0EEE66AF4EEE76AF1EE49
:10D6600010FA0BD5D0ED207A67EEA77AB4EEE77A00
:10D67000F1EE10FA94BF012000207047002070479F
:10D680000000164300806D44CDCC4C3EF0B52DED2E
:10D69000028B91B00846116A09910D911146D46927
:10D6A000536A176956699569B1EC018A0C930E9318
:10D6B000079708940A940B960F950CF0F3FB01A9B9
:10D6C00007A88DED010ACDED020A8DED031A0AF0CF
:10D6D00093FD04A88DED040ACDED050A8DED061A23
:10D6E0000DF00AF838EE400A11B0BDEC028BF0BD27
:10D6F00030B52DED048BD2ED014AD1ED006AD1EDAC
:10D70000018AD2ED097AD2ED075A92ED058A92ED9F
:10D71000086A92ED047A92ED065A76EEA46AD2ED8A
:10D72000024A78EEA48A91B025EEA89A8DED0B8A74
:10D7300028EE288A67EEA88AA7EE269A084614469D
:10D74000A5EEA68A1D46E6EE268AD2ED034A8DEDA9
:10D75000077A91ED027ACDED0C7A37EE247A111D1D
:10D76000A6EE079AA7EE878AE5EE078ACDED0E7A38
:10D77000CDED085A8DED096ACDED0A5A8DED0D6A91
:10D780008DED0F5A0CF08EFB01A907A88DED010A53
:10D79000CDED020A8DED031A0AF02EFD04A88DEDE1
:10D7A000040ACDED050A8DED061A0CF0A5FF4FF029
:10D7B0007E532B60D4ED077A94ED047A68EE277AD5
:10D7C000E7EE097A94ED087AE7EE287A87EE807A18
:10D7D000F1EE477AC5ED017AD4ED057A94ED077A3A
:10D7E00068EE277AE7EE097A94ED097AE7EE287A6F
:10D7F00087EE807AF1EE477AC5ED027AD4ED097AA8
:10D8000028EE278AD4ED087AA7EE898AD4ED067A25
:10D81000A7EEA88AC8EE007AF1EE677AC5ED037A22
:10D8200011B0BDEC048B30BD70B52DED048BD2ED85
:10D83000016A91ED007AD2ED024AD2ED075AD2ED9B
:10D84000058AD2ED047A92ED098A92ED086A92ED8A
:10D85000065A37EE267AD1ED016A76EEA46A90B0C8
:10D8600025EEA69ACDED0B8A68EEA68AA7EE879ADA
:10D870000D462846E5EE878A14461E46D2ED034A39
:10D88000CDED077AD1ED027A8DED0C8A77EEA47A90
:10D890008DED0E8AE8EE278A111D28EE268AA6EE67
:10D8A000279AA6EE078ACDED085AA5EE278A8DEDB8
:10D8B000096ACDED0A5A8DED0D6A8DED0F5A0CF007
:10D8C000F1FA01A907A88DED010ACDED020A8DED4F
:10D8D000031A0AF091FC04A88DED040ACDED050AA7
:10D8E0008DED061A0CF008FFD4ED077A94ED047A5A
:10D8F00068EEA77AE7EE097A94ED087AE7EE087AFF
:10D9000087EE807AF1EE477AC6ED007AD4ED057A9B
:10D9100094ED077A68EEA77AE7EE097A94ED097A32
:10D92000E7EE087A87EE807AF1EE477AC6ED017A63
:10D93000D4ED097A94ED087A68EEA77AE7EE097AD1
:10D9400094ED067AE7EE087A87EE807AF1EE477A70
:10D95000C6ED027A94ED017AD5ED007A77EE877AFA
:10D9600069EE677A87EE807A86ED037A94ED027A23
:10D97000D5ED017A77EE877A68EEE77A87EE807ADE
:10D9800086ED047A94ED037AD5ED027A77EE877A04
:10D9900068EE677A87EE807A86ED057AD4ED027AB2
:10D9A00095ED017AD4ED016A37EE277AD5ED007A4C
:10D9B00077EEA67A67EEA87AE7EE097AF1EE677A53
:10D9C00087EE807A86ED067AD4ED037A95ED027AB9
:10D9D000D4ED016A37EE277AD5ED007A77EEA67A94
:10D9E00067EE887AE7EE097AF1EE677A87EE807A59
:10D9F00086ED077A95ED027AD4ED037AD4ED026ACA
:10DA000037EE277AD5ED017A77EEA67A27EE888A67
:10DA1000A7EE288AB1EE488AC8EE007AC6ED087AE9
:10DA200010B0BDEC048B70BDB0F9063000EE903A3A
:10DA3000B0F9083001EE103AB0F9043000EE103AB7
:10DA4000F8EEE00AB8EEC11AB8EEC00AF4EE007AB9
:10DA500020EE270A60EEA70A21EE271A88B008B048
:10DA6000704700007FB500240546C0F88D40C0F81F
:10DA70009140A0F895400A26B5F89C30A34211DDEC
:10DA8000D5F8980006FB0400FFF7CEFF01A9284651
:10DA90008DED010ACDED020A8DED031A0134FFF779
:10DAA00013FDE9E704B070BD2DE9F0412DED028BC7
:10DAB000D0F8983086B004460E46174693B3D0EDA2
:10DAC000287A9FED1C8A77EEA77A002527EE888AB0
:10DAD0004FF00A08B4F89C20ABB29A4228D99F4272
:10DAE00001D10135F6E7D4F89800ABB208FB03008A
:10DAF000FFF79AFF694630468DED000ACDED010A29
:10DB00008DED021A0CF0E4F903A88DED030ACDEDBA
:10DB1000040A8DED051A0CF0EFFDB4EEC08AF1EEAB
:10DB200010FADEDD002006B0BDEC028BBDE8F0810E
:10DB30000120F8E7D829613D1FB504460846FFF7E4
:10DB400073FF01A920468DED010ACDED020A8DED8E
:10DB5000031AFFF7A9FF04B010BD00002DE9FF4133
:10DB6000D0F898300446002B66D0B0F89C500023C3
:10DB7000013DA0F89E30ADB24FF00A0855BB0A2710
:10DB8000B4F89C30AAB2934250D9D4F898101646F3
:10DB90007E4331442046FFF7CFFFC8B9D4F8981030
:10DBA000B4F89C3007FB0313881953F80A2C8A51E8
:10DBB00053F8062C426033F8023C0381B4F89C30E1
:10DBC000013BA4F89C30B4F89E300133A4F89E3099
:10DBD0000135D5E70AF052F9D4F8982008FB05FC86
:10DBE00002EB0C060346716852F80C0001AF03C744
:10DBF00031893980691CB3FBF1F000FB113308FB5C
:10DC000003F3D018D15842F80C10416871600289B2
:10DC1000328101AAD4F898C003CA0CEB03064CF871
:10DC200003003B8871603381013DA7E7204604B0C3
:10DC3000BDE8F041FFF716BF04B0BDE8F081000079
:10DC4000F0B52DED028BD0F8983085B004460E4625
:10DC500053B3B0F89C303BB39FED158A00250A27DB
:10DC6000B4F89C30AAB2934214D9D4F8983007FB88
:10DC70000230FFF7D9FE324601A920468DED010A98
:10DC8000CDED020A8DED031AFFF700FD0135A0EE80
:10DC9000008AE5E707EE903AF8EEE77A88EE270A81
:10DCA00005B0BDEC028BF0BD9FED020AF8E700BFA6
:10DCB00000000000CAF24971B0F89C3010B504466B
:10DCC0009BB100F1A001FFF7BBFF84ED340AD4F84B
:10DCD000D030C4F8D4304FF07E53C4F8D830C4F8F4
:10DCE000DC300023A4F8CC3010BD024BC0F8D0309B
:10DCF000EDE700BFCAF24971134AC0F8A020002125
:10DD0000002210B44FF07E54C0F8B040C0F8B440C8
:10DD1000C0F8B840C0F89C105DF8044BC0F8A420CF
:10DD2000C0F8A820C0F8AC20C0F8BC20C0F8C020C3
:10DD3000C0F8C420C0F8C820C0F88D10C0F89110F9
:10DD4000A0F89510FFF7B8BF0000484338B5044667
:10DD50000D4661B1436F8B4201D1012038BD0729C7
:10DD60001ED8DFE801F004121B4A535F62622046AE
:10DD7000FFF7C2FFD4F89800002565670028ECD0B3
:10DD800067F0A6FFC4F89850E7E70125FFF7B4FF56
:10DD9000656702212046FFF7D9FFDEE7012B01D09E
:10DDA0000020DBE790F88C30012B11D0D4F89830AC
:10DDB00043B90A214FF4967067F086FFC4F89800C3
:10DDC0000028EDD02046FFF777FF02236367C4E702
:10DDD0004BF096F8D4F888309FED227AC31A07EEFC
:10DDE000903AF8EE677A67EE877A94ED1E7AF4EE51
:10DDF000C77AF1EE10FAD9D5D2E7022BD0D1FFF7CE
:10DE0000ADFE2046FFF758FF0323DFE7032BC7D102
:10DE1000D0F8980020B167F05BFF0023C4F8983079
:10DE20000423D3E79A1F012ABAD9002BB8D094F85B
:10DE30007C3023B9D4F8980068B965678DE7012173
:10DE40002046FFF783FF0028F4D094F88C3001338C
:10DE500084F88C3082E767F03BFF0023C4F89830E9
:10DE6000EBE700BF6F12833A002310B503624362F1
:10DE70008362C362036343638363C36303640A4BC4
:10DE8000C0F880300446A030FFF750FA04F58070E7
:10DE90004AF0F2F904F58C704AF0EEF900212046C0
:10DEA000FFF754FF204610BD0000A0402DE9F04FC1
:10DEB0002DED048BD0F89830C3B00546002B00F050
:10DEC000058190ED348A0CA8FFF730FA05F1A00621
:10DED00017A8FFF72BFA0FCE17AC0FC40FCE0FC445
:10DEE00096E8070017AF84E807000FCF0CAE0FC607
:10DEF0000FCF0FC694E8070086E8070040220021F4
:10DF000022A86CF093F94022002132A86CF08EF91F
:10DF1000102200210DEB02006CF088F9002705F1BA
:10DF2000A0064FF00A09B5F89C20BBB29A4244D92A
:10DF3000D5F8980009FB0300FFF776FD0DF1040BFF
:10DF400008AB0CAA594628468BED000ACBED010A16
:10DF50008BED021AFFF7CCFB0DF110080DF1200A32
:10DF6000002422AB03EB8401FAEC018A32AB03EB11
:10DF7000840208A80023D1ED007AB0EC017AE8EE23
:10DF8000877A0133DBB2042BE1EC017AD2ED007A1F
:10DF9000E8EE877AE2EC017AEDD10CAA59462846E0
:10DFA000FFF774FBD8ED007AE8EE807A0434102C89
:10DFB000E8EC017AD5D10137B5E795ED367AB2EEC6
:10DFC000049AC7EE096A0DF1880832AF3B46424613
:10DFD000002411460134042C02F1140252ED057A9A
:10DFE00077EE877AC1ED007AD3ED007A77EEA67AE4
:10DFF0001946C1ED007A03F11403EAD122A92246A1
:10E0000008460AF0A9FC002860D022463946384666
:10E010000AF0A2FC002859D00CA817A90022B0ECE5
:10E02000017AF1EC017A0DF1100E3C46C446002352
:10E03000FEEC016ABCEC016A0133A6EEC67ADBB2E3
:10E04000042BB4EC016AE6EEC67AF1D10432102A50
:10E0500000ED017A41ED017A08F1100807F110078F
:10E06000DDD10CA92846FFF7EBFD17A92846F0EEF5
:10E07000408AFFF7E5FDD5ED347AF4EEE87AF1EE6B
:10E0800010FA28D5F4EEC07AF1EE10FA23D595ED0A
:10E09000367A27EE099A85ED369AB4EE488AF1EE83
:10E0A00010FA13D6F4EEC87AF1EE10FA0EDD34460B
:10E0B0000CAE0FCE85ED348A0FC40FCE0FC496E898
:10E0C000070084E807002846FFF7CCFC43B0BDEC0E
:10E0D000048BBDE8F08FF4EEC07AF1EE10FA1CDD8F
:10E0E000F4EEC08AF1EE10FA17DD17AC0FCC95ED07
:10E0F000367AC7EE097A0CAF0FC70FCC0FC794E87A
:10E10000070087E80700C5ED367AB0EE408AB4EE26
:10E11000488AF1EE10FACAD7D8E7F4EEE87AF1EEC1
:10E1200010FABADDB0EE688AF1E700002DE9F04F91
:10E130002DED048BD0F89830ADF54F7D0546002BC2
:10E1400000F00181D0ED348A16A8FFF7EFF805F151
:10E15000A00621A8FFF7EAF80FCE21AC0FC40FCE1E
:10E160000FC496E8070021AF84E807000FCF16AE72
:10E170000FC60FCF0FC694E8070086E807004FF4DC
:10E18000A27200212CA86CF051F84FF4A272002169
:10E190007DA86CF04BF82422002104A86CF046F80E
:10E1A000002705F1A0064FF00A09B5F89C20BBB284
:10E1B0009A4244D9D5F8980009FB0300FFF734FCD4
:10E1C0000DF1040B0DAB16AA594628468BED000A3B
:10E1D000CBED010A8BED021AFFF726FB0DF11008BB
:10E1E0000DF1340A00242CAB03EB8401BAEC018A54
:10E1F0007DAB03EB84020DA80023D1ED007AB0ECD7
:10E20000017AE8EE077A0133DBB2092BE1EC017AFF
:10E21000D2ED007AE8EE077AE2EC017AEDD116AAA7
:10E2200059462846FFF732FAD8ED007AE8EE007A30
:10E230000934512CE8EC017AD5D10137B5E795EDD9
:10E24000377AB2EE049AC7EE096A0DF1B0087DAFD5
:10E250003B464246002411460134092C02F12802B3
:10E2600052ED0A7A77EE877AC1ED007AD3ED007A23
:10E2700077EEA67A1946C1ED007A03F12803EAD1B8
:10E280002CA9224608460AF067FB00285BD02246EC
:10E29000394638460AF060FB002854D017A822A956
:10E2A0000022B0EC017AF1EC017A0DF1100E3C463F
:10E2B000C4460023FEEC016ABCEC016A0133A6EE01
:10E2C000C67ADBB2092BB4EC016AE6EEC67AF1D16C
:10E2D0000932512A00ED017A41ED017A08F1240852
:10E2E00007F12407DDD116A92846FFF7A9FC21A9CB
:10E2F0002846B0EE408AFFF7A3FCD5ED347AF4EE61
:10E30000C87AF1EE10FA24D5F4EEC07AF1EE10FAE4
:10E310001FD595ED377A27EE099A85ED379AF4EEF9
:10E32000E87AF1EE10FA0EDD344616AE0FCEC5EDEA
:10E33000348A0FC40FCE0FC496E8070084E80700A4
:10E340002846FFF78FFB0DF54F7DBDEC048BBDE834
:10E35000F08FF4EEC07AF1EE10FA19DDB4EEC08A57
:10E36000F1EE10FA14DD21AC0FCC95ED377AC7EE43
:10E37000097A16AF0FC70FCC0FC794E8070087E8DC
:10E380000700C5ED377AB0EE408AF0EE488ACBE759
:10E39000F4EEC87AF1EE10FAF7DCC0E770B5044687
:10E3A00086B000F58C71EE2203A806F081F894F88F
:10E3B000FD3023B903A806F09DF806B070BD636F69
:10E3C000012B03D102212046FFF7C0FC002384F873
:10E3D000FD3004F1EC0207CA6B4603C303A81A80A0
:10E3E00006F088F8636F023B012BE6D8B4F89C3046
:10E3F000B3F5967FE1D26846FFF716FB4FF6FF7242
:10E4000003A920468DED030ACDED040A8DED051A12
:10E41000FFF74AFB0028D0D06846FFF705FB03A9A9
:10E4200020468DED030ACDED040A8DED051AFFF7A8
:10E430004BF8B4F89C20D4F898600A235A436B46F2
:10E4400003CBB518B05069601B882B81B4F89C30A1
:10E450000133A4F89C30B0E7F0B5002385B0044642
:10E4600000F1A406C0F8AC30C0F8A830C0F8A43061
:10E4700000250A27B4F89C30AAB2934211D9D4F8E7
:10E48000983007FB0230FFF7CFFA01A930468DED37
:10E49000010ACDED020A8DED031A01350BF068FD7E
